:10000000F8FF022095A2010079A2010031A20100AF
:1000100031A2010031A2010031A2010031A2010090
:1000200031A2010031A2010031A2010079A2010038
:1000300079A2010031A2010051960100C998010086
:1000400079A2010079A2010079A2010079A2010040
:1000500079A2010079A2010079A2010079A2010030
:1000600079A2010079A2010079A2010079A2010020
:1000700079A2010079A2010079A2010079A2010010
:1000800079A2010079A2010079A2010079A2010000
:1000900079A2010079A2010079A2010079A20100F0
:1000A00079840100D585010079A2010079A20100BF
:1000B00079A2010079A2010079A20100DDB301005B
:1000C00079A20100B1DB010079A201000DDD010080
:1000D00079A201003DDE010079A2010079A20100B0
:1000E00079A2010079A2010079A2010079A20100A0
:1000F00079A2010079A2010079A2010079A2010090
:1001000079A2010079A2010079A2010079A201007F
:1001100079A201008DBC010079A2010079A2010041
:1001200079A2010079A2010079A2010079A201005F
:1001300079A2010079A2010079A2010079A201004F
:100140009D93010079A201006DDF010079A20100F9
:100150009DE0010079A2010079A2010079A20100CD
:1001600079A2010079A201003187010079A2010082
:1001700079A2010079A2010079A2010079A201000F
:1001800079A20100A14F010079A2010079A201002A
:1001900079A2010079A20100FFFFFFFFFFFFFFFF2F
:1001A000FFFFFFFFFFFFFFFFFFFFFFFFFFFFFFFF5F
:1001B000FFFFFFFFFFFFFFFFFFFFFFFFFFFFFFFF4F
:1001C000FFFFFFFFFFFFFFFFFFFFFFFFFFFFFFFF3F
:1001D000FFFFFFFFFFFFFFFFFFFFFFFFFFFFFFFF2F
:10040000FFFFFFFFFFFFFFFFFFFFFFFFDEF9FFFF23
:1004100010B5054C237833B9044B13B10448AFF33E
:1004200000800123237010BDF4EB002000000000C9
:10043000CC4A0200084B10B51BB108490848AFF37D
:1004400000800848036803B910BD074B002BFBD0A0
:10045000BDE81040184700BF00000000F8EB002086
:10046000CC4A0200F4EB002000000000704700BFFF
:1004700010B54FF4097104461AF086F8204610BDF5
:1004800070B54FF06A522DED028B064642F6584386
:1004900008EE902A40F6DB72C0F202034FF20E45DE
:1004A00040F6DA70C4F24902C2F20005C3F64920F0
:1004B00008EE102A336000240FE007EE904AF8EEB1
:1004C000E77A77EE807A67EEA87A67EE887A27EE89
:1004D000800A1EF001F910EE100A21F0BFF841EC7D
:1004E000100B1DF061FF00230022CCF2900351ECB1
:1004F000100B21F007F941EC100B1DF069FF51ECD6
:10050000100B21F0D7FB0134B4F5806FB6EE000A72
:1005100025F8020FD1D14FF06A534EF60E4508EE82
:10052000103AC2F20005002407EE904AF8EEE77A8E
:10053000013467EE887A17EE900A21F08FF89FED6C
:10054000140B41EC110B1EF0C7F9002351EC100BFA
:100550000022C3F6F07320F021FF00230022C4F232
:10056000B00321F0CFF821F0C5FB21F077F841EC82
:10057000100B1DF02DFF51EC100B21F09BFBB4F57F
:10058000806F25F8020FCFD1BDEC028B304670BDD5
:100590000000000000000040704700BF10B54FF49D
:1005A0000971044619F0F0FF204610BD2DE9F04F07
:1005B0004DF66C66C2F200060A9D0B989DF83070ED
:1005C000B6F800C042F67044C0F20204C5EB000A5F
:1005D000002F18BF0C466FEA0C0B0AF1200A4DF6EB
:1005E0006C294DF66C48043A271FA1F1040E0FFA4E
:1005F0008BFB4FEAAA1AC2F20009C2F200080026D9
:1006000027E0B4F5007F02D08CB3C943C9B239F8F2
:1006100011104CEA010101EBC00080B20BEA0004AA
:10062000E143C9B2241238F8111001F58061490084
:10063000E14010EA0C0F18BFC94357F8044F09985E
:1006400009B2013604EB8131402E03444EF8041FF9
:1006500010D052F8041F1944891301F44074554412
:10066000B4F5807FC9B2A8B2CBD1C943C9B239F8B9
:100670001110D0E7BDE8F08F2DE9F04F4DF66C6515
:10068000C2F2000509982E880A9D9DF82C7042F64A
:100690007044C0F20204C0EB050E002F14BF0F46D9
:1006A00027466FEA06090EF1200E4DF66C284DF62E
:1006B0006C4C3C1F0D1F0FFA89F9FC374FEAAE1E38
:1006C000C2F20008C2F2000C2AE0BBF5007F04D0A1
:1006D000BBF1000F30D0C943C9B238F81110314313
:1006E00001EBCA0A1FFA8AFA09EA0A0B6FEA0B0140
:1006F000C9B24FEA2B2B3CF8111001F5806149007B
:100700001AEA060F21FA0BF154F804AF18BFC943D7
:1007100009B20AEB8131BC421A4445F8041F0ED0DD
:10072000911301F4407B7044BBF5807F1FFA80FA7F
:10073000C9B2CAD1C943C9B238F81110D0E7BDE86F
:10074000F08F00BF2DE9F04F4DF66C6083B0C2F220
:1007500000000D9EB0F800C00C9C9DF840A00F9FBB
:100760000E980E9D019342F6704EC0F2020EC4EB3D
:10077000060B6FEA0C06BAF1000F14BF8A46F24668
:1007800033B20BF1200B4DF66C294DF66C48AAF1F3
:10079000040600686D680093A1F1040E0AF1FC0ADA
:1007A0004FEAAB1B0137C2F20009C2F2000829E090
:1007B000B0F5007F02D098B3DB43DBB239F81330D9
:1007C0004CEA030303EBC101009B89B203EA010079
:1007D000C343DBB2001238F8133003F580635B00CB
:1007E000C34011EA0C0F18BFDB4356F8041F0198F1
:1007F0001BB29B031944564502444EF8041F284679
:1008000011D01D4643193B4113449B1303F4407020
:100810005C44B0F5807FDBB2A1B2C9D1DB43DBB26F
:1008200039F81330CEE70E9A1560536003B0BDE877
:10083000F08F00BF2DE9F04F43F6345403EB430330
:10084000C0F2020404EBC3050646144689460FCDE8
:1008500091B00AAF0FC795E80300002387E80300B3
:10086000012704F160088DF8247007978DF8253072
:100870008DF826300AAD48E00AF1FF3101EB011195
:1008800006EB0111133121F00F0194E80140C0146F
:10089000C0F500706060BEF1000F3FD0BEF5FE7F76
:1008A0003EDA10AFBA441AF81CCCBCF1000F04D0E9
:1008B00012F1000C18BF4FF0010CC3F301123AB152
:1008C00010AF07EB020B1BF81CBCBBF1000F34D1BF
:1008D00003F0C003C02B02D11B9B0F2B41DDA3688B
:1008E000E2680190CDF808C0CDF800E03046FFF78F
:1008F000C3FE9DF81C300AF81C3CE368A26803EBB9
:100900008213E3601034A04514D055F8043B13F073
:10091000030A03F00402AFD14946B6E740F2FF1ED6
:10092000B0F5FE7FBDDB002AE7D110AB9A440AF890
:100930001C2CE2E711B0BDE8F08F013A02EB021285
:10094000E368CDF80CC006EB02120290CDF804E08B
:10095000A0680090133222F00F023046FFF726FE07
:10096000C7E71F46E268A36803971A9F0190CDF876
:1009700010C00297CDF800E03046FFF7E3FEB8E77D
:1009800000207047704700BF704700BF10B5044695
:1009900018F086FC204610BD42F6EC5008B5162132
:1009A000C0F202001CF00AFF4FF20F601CF07CF84E
:1009B00042F60460C0F202000F211CF0FFFE4EF26E
:1009C0000020C2F20000BDE8084019F073B800BF73
:1009D00042F6146008B51021C0F202001CF0EEFED1
:1009E0004FF60F201CF060F842F60460C0F20200DF
:1009F0000F211CF0E3FE4EF20020C2F20000BDE821
:100A0000084019F057B800BF42F6286008B5132116
:100A1000C0F202001CF0D2FE4FF60F301CF044F87A
:100A200042F60460C0F202000F211CF0C7FE4EF235
:100A30000020C2F20000BDE8084019F03BB800BF3A
:100A400042F63C6008B50F21C0F202001CF0B6FE71
:100A50004FF60F401CF028F842F60460C0F2020086
:100A60000F211CF0ABFE4EF20020C2F20000BDE8E8
:100A7000084019F01FB800BF42F64C6008B51821B5
:100A8000C0F202001CF09AFE4FF60F601CF00CF84A
:100A900042F60460C0F202000F211CF08FFE4EF2FD
:100AA0000020C2F20000BDE8084019F003B800BF02
:100AB00042F6686008B50F21C0F202001CF07EFE0D
:100AC00040F67473C2F20103FC21986C03681B6842
:100AD000984742F67860C0F202000F211CF06EFECB
:100AE0004EF20020C2F20000BDE8084018F0E2BF5C
:100AF00042F6886008B51821C0F202001CF05EFEC4
:100B000040F67473C2F20103FE21986C03681B68FF
:100B1000984742F67860C0F202000F211CF04EFEAA
:100B20004EF20020C2F20000BDE8084018F0C2BF3B
:100B300042F6A46008B51021C0F202001CF03EFE8F
:100B400040F67473C2F20103FA21986C03681B68C3
:100B5000984742F67860C0F202000F211CF02EFE8A
:100B60004EF20020C2F20000BDE8084018F0A2BF1B
:100B700042F6B86008B51321C0F202001CF01EFE58
:100B800040F67473C2F20103FB21986C03681B6882
:100B9000984742F67860C0F202000F211CF00EFE6A
:100BA0004EF20020C2F20000BDE8084018F082BFFB
:100BB00038B542F6CC604EF2002540F66454102160
:100BC000C2F20104C2F20005C0F202001CF0F6FD00
:100BD000284618F06FFF20680FF00CF820680EF020
:100BE00015FF20680EF026FF42F6E0601621C0F2E5
:100BF00002001CF0E3FD4FF60F701BF055FF42F6AC
:100C00000460C0F202000F211CF0D8FD2846BDE8A8
:100C1000384018F04FBF00BF38B542F6CC604EF2F6
:100C2000002540F664541021C2F20104C2F200050E
:100C3000C0F202001CF0C2FD284618F03BFF2068FD
:100C40000EF0D8FF20680EF0E1FE20680EF0F2FEF4
:100C500042F6F8601621C0F202001CF0AFFD40F62B
:100C60007473C2F20103FF21986C03681B689847F4
:100C700042F67860C0F202000F211CF09FFD28466A
:100C8000BDE8384018F016BF10B5044642F61070A3
:100C90001521C0F202001CF091FD200400F4FE00BA
:100CA00040F4734040F002001BF0FEFE42F6046088
:100CB000C0F202000F211CF081FD4EF20020C2F2B2
:100CC0000000BDE8104018F0F5BE00BF10B50446A6
:100CD00042F628701F21C0F2020004F00F041CF03D
:100CE0006DFD44F010044FF2021040EA04401BF086
:100CF000DBFE42F60460C0F202000F211CF05EFD34
:100D00004EF20020C2F20000BDE8104018F0D2BE42
:100D100042F6487008B51621C0F202001CF04EFDE4
:100D200040F67473C2F20103F621986C0368DB6C21
:100D3000984742F67860C0F202000F211CF03EFD99
:100D40004EF20020C2F20000BDE8084018F0B2BE2A
:100D50001F2938B50C46054608D84DF67063C2F217
:100D6000000318790FF0B8FE0BF050FD42F66070EA
:100D70000D21C0F202001CF021FD2304681E03F4C3
:100D8000FE0343F44043000243F00C0300F47060A0
:100D900018431BF089FE42F60460C0F202000F21E6
:100DA0001CF00CFD4EF20020C2F20000BDE83840FD
:100DB00018F080BE70B5064642F670700C46C0F260
:100DC0000200122115461CF0F9FC6EB9681E0002E3
:100DD000240400F4706004F4FE04204340F4504006
:100DE00040F00D001BF060FE42F60460C0F202000D
:100DF0000F211CF0E3FC4EF20020C2F20000BDE81F
:100E0000704018F057BE00BF38B540F67474054600
:100E1000C2F2010442F684701F21C0F202001CF0ED
:100E2000CDFCA06C0368F1211B689847A06C036897
:100E300029461B68984742F67860C0F202000F21ED
:100E40001CF0BCFC4EF20020C2F20000BDE83840AD
:100E500018F030BE38B540F674740546C2F201048D
:100E600042F6A4701521C0F202001CF0A7FCA06C91
:100E70000368F3211B689847A06C036805F07F01A5
:100E8000DB6C984742F67860C0F202000F211CF03C
:100E900095FC4EF20020C2F20000BDE8384018F088
:100EA00009BE00BFF0B548F21C52C2F2010283B085
:100EB00040F2442311680091C2F2010300991E68B8
:100EC0001268019240F65C55C2F2010540F62852C4
:100ED000C2F20102891B42F6BC704EF20024C2F23B
:100EE0000004019F298000260C21C0F20200167028
:100EF0001F601CF063FC2B8820464EF6602191FB9E
:100F0000F3F118F079FD42F6CC700521C0F2020031
:100F10001CF054FC2988204618F06EFD42F6D4706F
:100F20000F21C0F202001CF049FC204618F0C2FD5F
:100F300003B0F0BD08B540F62851C2F201014AF6EF
:100F4000AB230A780132D2B2CAF6AA23A3FB02036A
:100F50001B0903EB4303A2EBC30313F0FF0F0A705B
:100F600001D1FFF79FFF42F6E4701021C0F20200AA
:100F70001CF024FC4FF60F001BF096FD42F60460B7
:100F8000C0F202000F211CF019FC4EF20020C2F248
:100F90000000BDE8084018F08DBD00BF08B540F660
:100FA0002851C2F201014AF6AB230A780132D2B2CB
:100FB000CAF6AA23A3FB02031B0903EB4303A2EB1C
:100FC000C30313F0FF0F0A7001D1FFF76BFF42F666
:100FD000F8701021C0F202001CF0F0FB40F67473B0
:100FE000C2F20103F821986C03681B68984742F627
:100FF0007860C0F202000F211CF0E0FB4EF20020EE
:10100000C2F20000BDE8084018F054BD38B540F603
:101010006453C2F2010301F500521B6805460C46F9
:1010200043F20C00C3F884200D21C0F2020004F347
:101030000D041CF0C3FB04F50054681E23040002D9
:1010400003F4FE0300F47060184340F4604064044D
:1010500004F0FE4440F00E0020431BF025FD42F654
:101060000460C0F202000F211CF0A8FB4EF2002029
:10107000C2F20000BDE8384018F01CBD1F2938B589
:101080000D46044608D84DF67063C2F20003187985
:101090000FF022FD0BF0BAFB43F21C000D21C0F251
:1010A00002001CF08BFB611EC9B20F290FD840F65D
:1010B0007474C2F2010441F0C001A06C03681B68A3
:1010C0009847A06C036805F07F011B68984742F6BB
:1010D0007860C0F202000F211CF070FB4EF200207D
:1010E000C2F20000BDE8384018F0E4BC48F290338A
:1010F000C2F2010310B49A6B13685068197804782F
:10110000507A137A044201EA03011AD0937A03F069
:10111000030309B143F0040343F008039910082BBB
:1011200091722AD8072B22D2032B2ED011D9042B4F
:1011300013D0062B14D1D3685DF8044B023BD36067
:101140007047937A03F003030029E7D043F00403C8
:10115000E4E7012B0BD0022B02D1D368013BD36013
:101160005DF8044B70470D2BF7D00E2BF8D1D368E8
:101170005DF8044B0133D36070470C2B05D0F2D8D7
:10118000092BD8D00B2BE8D0EAE7D3685DF8044BE5
:101190000233D360704700BF48F29033C2F20103BC
:1011A00010B4DA6B1368506819780478507A137A9F
:1011B000044201EA03011AD0937A03F0030309B150
:1011C00043F0040343F008039910082B91722AD8C6
:1011D000072B22D2032B2ED011D9042B13D0062B90
:1011E00014D1D3685DF8044B023BD3607047937A07
:1011F00003F003030029E7D043F00403E4E7012BE5
:101200000BD0022B02D1D368013BD3605DF8044BB5
:1012100070470D2BF7D00E2BF8D1D3685DF8044B37
:101220000133D36070470C2B05D0F2D8092BD8D0EE
:101230000B2BE8D0EAE7D3685DF8044B0233D360A8
:10124000704700BF48F29033C2F2010310B41A6C29
:101250001368506819780478507A137A044201EAC6
:1012600003011AD0937A03F0030309B143F0040396
:1012700043F008039910082B91722AD8072B22D229
:10128000032B2ED011D9042B13D0062B14D1D368E5
:101290005DF8044B023BD3607047937A03F003037D
:1012A0000029E7D043F00403E4E7012B0BD0022B25
:1012B00002D1D368013BD3605DF8044B70470D2B1E
:1012C000F7D00E2BF8D1D3685DF8044B0133D3600F
:1012D00070470C2B05D0F2D8092BD8D00B2BE8D0B7
:1012E000EAE7D3685DF8044B0233D360704700BF70
:1012F00048F29033C2F2010310B45A6C136850687C
:1013000019780478507A137A044201EA03011AD05A
:10131000937A03F0030309B143F0040343F0080395
:101320009910082B91722AD8072B22D2032B2ED08A
:1013300011D9042B13D0062B14D1D3685DF8044BBC
:10134000023BD3607047937A03F003030029E7D090
:1013500043F00403E4E7012B0BD0022B02D1D36846
:10136000013BD3605DF8044B70470D2BF7D00E2B7B
:10137000F8D1D3685DF8044B0133D36070470C2B70
:1013800005D0F2D8092BD8D00B2BE8D0EAE7D368E8
:101390005DF8044B0233D360704700BF48F29033CE
:1013A000C2F2010310B49A6C13685068197804787B
:1013B000507A137A044201EA03011AD0937A03F0B7
:1013C000030309B143F0040343F008039910082B09
:1013D00091722AD8072B22D2032B2ED011D9042B9D
:1013E00013D0062B14D1D3685DF8044B023BD360B5
:1013F0007047937A03F003030029E7D043F0040316
:10140000E4E7012B0BD0022B02D1D368013BD36060
:101410005DF8044B70470D2BF7D00E2BF8D1D36835
:101420005DF8044B0133D36070470C2B05D0F2D824
:10143000092BD8D00B2BE8D0EAE7D3685DF8044B32
:101440000233D360704700BF48F29033C2F2010309
:1014500010B4DA6C1368506819780478507A137AEB
:10146000044201EA03011AD0937A03F0030309B19D
:1014700043F0040343F008039910082B91722AD813
:10148000072B22D2032B2ED011D9042B13D0062BDD
:1014900014D1D3685DF8044B023BD3607047937A54
:1014A00003F003030029E7D043F00403E4E7012B32
:1014B0000BD0022B02D1D368013BD3605DF8044B03
:1014C00070470D2BF7D00E2BF8D1D3685DF8044B85
:1014D0000133D36070470C2B05D0F2D8092BD8D03C
:1014E0000B2BE8D0EAE7D3685DF8044B0233D360F6
:1014F000704700BF48F29033C2F2010310B41A6D76
:101500001368506819780478507A137A044201EA13
:1015100003011AD0937A03F0030309B143F00403E3
:1015200043F008039910082B91722AD8072B22D276
:10153000032B2ED011D9042B13D0062B14D1D36832
:101540005DF8044B023BD3607047937A03F00303CA
:101550000029E7D043F00403E4E7012B0BD0022B72
:1015600002D1D368013BD3605DF8044B70470D2B6B
:10157000F7D00E2BF8D1D3685DF8044B0133D3605C
:1015800070470C2B05D0F2D8092BD8D00B2BE8D004
:10159000EAE7D3685DF8044B0233D360704700BFBD
:1015A00048F29033C2F2010310B45A6D13685068C8
:1015B00019780478507A137A044201EA03011AD0A8
:1015C000937A03F0030309B143F0040343F00803E3
:1015D0009910082B91722AD8072B22D2032B2ED0D8
:1015E00011D9042B13D0062B14D1D3685DF8044B0A
:1015F000023BD3607047937A03F003030029E7D0DE
:1016000043F00403E4E7012B0BD0022B02D1D36893
:10161000013BD3605DF8044B70470D2BF7D00E2BC8
:10162000F8D1D3685DF8044B0133D36070470C2BBD
:1016300005D0F2D8092BD8D00B2BE8D0EAE7D36835
:101640005DF8044B0233D360704700BF48F290331B
:10165000C2F2010310B49A6D1368506819780478C7
:10166000507A137A044201EA03011AD0937A03F004
:10167000030309B143F0040343F008039910082B56
:1016800091722AD8072B22D2032B2ED011D9042BEA
:1016900013D0062B14D1D3685DF8044B023BD36002
:1016A0007047937A03F003030029E7D043F0040363
:1016B000E4E7012B0BD0022B02D1D368013BD360AE
:1016C0005DF8044B70470D2BF7D00E2BF8D1D36883
:1016D0005DF8044B0133D36070470C2B05D0F2D872
:1016E000092BD8D00B2BE8D0EAE7D3685DF8044B80
:1016F0000233D360704700BF48F29033C2F2010357
:1017000010B4DA6D1368506819780478507A137A37
:10171000044201EA03011AD0937A03F0030309B1EA
:1017200043F0040343F008039910082B91722AD860
:10173000072B22D2032B2ED011D9042B13D0062B2A
:1017400014D1D3685DF8044B023BD3607047937AA1
:1017500003F003030029E7D043F00403E4E7012B7F
:101760000BD0022B02D1D368013BD3605DF8044B50
:1017700070470D2BF7D00E2BF8D1D3685DF8044BD2
:101780000133D36070470C2B05D0F2D8092BD8D089
:101790000B2BE8D0EAE7D3685DF8044B0233D36043
:1017A000704700BF48F29033C2F2010310B41A6EC2
:1017B0001368506819780478507A137A044201EA61
:1017C00003011AD0937A03F0030309B143F0040331
:1017D00043F008039910082B91722AD8072B22D2C4
:1017E000032B2ED011D9042B13D0062B14D1D36880
:1017F0005DF8044B023BD3607047937A03F0030318
:101800000029E7D043F00403E4E7012B0BD0022BBF
:1018100002D1D368013BD3605DF8044B70470D2BB8
:10182000F7D00E2BF8D1D3685DF8044B0133D360A9
:1018300070470C2B05D0F2D8092BD8D00B2BE8D051
:10184000EAE7D3685DF8044B0233D360704700BF0A
:1018500048F29033C2F2010310B45A6E1368506814
:1018600019780478507A137A044201EA03011AD0F5
:10187000937A03F0030309B143F0040343F0080330
:101880009910082B91722AD8072B22D2032B2ED025
:1018900011D9042B13D0062B14D1D3685DF8044B57
:1018A000023BD3607047937A03F003030029E7D02B
:1018B00043F00403E4E7012B0BD0022B02D1D368E1
:1018C000013BD3605DF8044B70470D2BF7D00E2B16
:1018D000F8D1D3685DF8044B0133D36070470C2B0B
:1018E00005D0F2D8092BD8D00B2BE8D0EAE7D36883
:1018F0005DF8044B0233D360704700BF48F2903369
:10190000C2F2010310B49A6E136850681978047813
:10191000507A137A044201EA03011AD0937A03F051
:10192000030309B143F0040343F008039910082BA3
:1019300091722AD8072B22D2032B2ED011D9042B37
:1019400013D0062B14D1D3685DF8044B023BD3604F
:101950007047937A03F003030029E7D043F00403B0
:10196000E4E7012B0BD0022B02D1D368013BD360FB
:101970005DF8044B70470D2BF7D00E2BF8D1D368D0
:101980005DF8044B0133D36070470C2B05D0F2D8BF
:10199000092BD8D00B2BE8D0EAE7D3685DF8044BCD
:1019A0000233D360704700BF48F29033C2F20103A4
:1019B00010B4DA6E1368506819780478507A137A84
:1019C000044201EA03011AD0937A03F0030309B138
:1019D00043F0040343F008039910082B91722AD8AE
:1019E000072B22D2032B2ED011D9042B13D0062B78
:1019F00014D1D3685DF8044B023BD3607047937AEF
:101A000003F003030029E7D043F00403E4E7012BCC
:101A10000BD0022B02D1D368013BD3605DF8044B9D
:101A200070470D2BF7D00E2BF8D1D3685DF8044B1F
:101A30000133D36070470C2B05D0F2D8092BD8D0D6
:101A40000B2BE8D0EAE7D3685DF8044B0233D36090
:101A5000704700BF48F29033C2F2010310B41A6F0E
:101A60001368506819780478507A137A044201EAAE
:101A700003011AD0937A03F0030309B143F004037E
:101A800043F008039910082B91722AD8072B22D211
:101A9000032B2ED011D9042B13D0062B14D1D368CD
:101AA0005DF8044B023BD3607047937A03F0030365
:101AB0000029E7D043F00403E4E7012B0BD0022B0D
:101AC00002D1D368013BD3605DF8044B70470D2B06
:101AD000F7D00E2BF8D1D3685DF8044B0133D360F7
:101AE00070470C2B05D0F2D8092BD8D00B2BE8D09F
:101AF000EAE7D3685DF8044B0233D360704700BF58
:101B000048F29033C2F2010310B45A6F1368506860
:101B100019780478507A137A044201EA03011AD042
:101B2000937A03F0030309B143F0040343F008037D
:101B30009910082B91722AD8072B22D2032B2ED072
:101B400011D9042B13D0062B14D1D3685DF8044BA4
:101B5000023BD3607047937A03F003030029E7D078
:101B600043F00403E4E7012B0BD0022B02D1D3682E
:101B7000013BD3605DF8044B70470D2BF7D00E2B63
:101B8000F8D1D3685DF8044B0133D36070470C2B58
:101B900005D0F2D8092BD8D00B2BE8D0EAE7D368D0
:101BA0005DF8044B0233D360704700BF48F29033B6
:101BB000C2F2010310B49A6F136850681978047860
:101BC000507A137A044201EA03011AD0937A03F09F
:101BD000030309B143F0040343F008039910082BF1
:101BE00091722AD8072B22D2032B2ED011D9042B85
:101BF00013D0062B14D1D3685DF8044B023BD3609D
:101C00007047937A03F003030029E7D043F00403FD
:101C1000E4E7012B0BD0022B02D1D368013BD36048
:101C20005DF8044B70470D2BF7D00E2BF8D1D3681D
:101C30005DF8044B0133D36070470C2B05D0F2D80C
:101C4000092BD8D00B2BE8D0EAE7D3685DF8044B1A
:101C50000233D360704700BF48F29033C2F20103F1
:101C600010B4DA6F1368506819780478507A137AD0
:101C7000044201EA03011AD0937A03F0030309B185
:101C800043F0040343F008039910082B91722AD8FB
:101C9000072B22D2032B2ED011D9042B13D0062BC5
:101CA00014D1D3685DF8044B023BD3607047937A3C
:101CB00003F003030029E7D043F00403E4E7012B1A
:101CC0000BD0022B02D1D368013BD3605DF8044BEB
:101CD00070470D2BF7D00E2BF8D1D3685DF8044B6D
:101CE0000133D36070470C2B05D0F2D8092BD8D024
:101CF0000B2BE8D0EAE7D3685DF8044B0233D360DE
:101D0000704700BF48F29033C2F2010310B4D3F819
:101D100080201368506819780478507A137A044246
:101D200001EA03011AD0937A03F0030309B143F0E7
:101D3000040343F008039910082B91722AD8072B4B
:101D400022D2032B2ED011D9042B13D0062B14D161
:101D5000D3685DF8044B023BD3607047937A03F07D
:101D600003030029E7D043F00403E4E7012B0BD081
:101D7000022B02D1D368013BD3605DF8044B70475E
:101D80000D2BF7D00E2BF8D1D3685DF8044B01333F
:101D9000D36070470C2B05D0F2D8092BD8D00B2B71
:101DA000E8D0EAE7D3685DF8044B0233D3607047AC
:101DB00048F29033C2F2010310B4D3F884201368C0
:101DC000506819780478507A137A044201EA0301C2
:101DD0001AD0937A03F0030309B143F0040343F0EC
:101DE00008039910082B91722AD8072B22D2032BB3
:101DF0002ED011D9042B13D0062B14D1D3685DF843
:101E0000044B023BD3607047937A03F0030300292D
:101E1000E7D043F00403E4E7012B0BD0022B02D1FF
:101E2000D368013BD3605DF8044B70470D2BF7D0AE
:101E30000E2BF8D1D3685DF8044B0133D3607047A3
:101E40000C2B05D0F2D8092BD8D00B2BE8D0EAE721
:101E5000D3685DF8044B0233D360704748F2903387
:101E6000C2F2010310B4D3F88820136850681978BF
:101E70000478507A137A044201EA03011AD0937A63
:101E800003F0030309B143F0040343F0080399107E
:101E9000082B91722AD8072B22D2032B2ED011D9CE
:101EA000042B13D0062B14D1D3685DF8044B023BEE
:101EB000D3607047937A03F003030029E7D043F01F
:101EC0000403E4E7012B0BD0022B02D1D368013BC2
:101ED000D3605DF8044B70470D2BF7D00E2BF8D173
:101EE000D3685DF8044B0133D36070470C2B05D0E9
:101EF000F2D8092BD8D00B2BE8D0EAE7D3685DF8ED
:101F0000044B0233D360704748F29033C2F20103AE
:101F100010B4D3F88C201368506819780478507A7C
:101F2000137A044201EA03011AD0937A03F00303FF
:101F300009B143F0040343F008039910082B917290
:101F40002AD8072B22D2032B2ED011D9042B13D041
:101F5000062B14D1D3685DF8044B023BD360704765
:101F6000937A03F003030029E7D043F00403E4E786
:101F7000012B0BD0022B02D1D368013BD3605DF85B
:101F8000044B70470D2BF7D00E2BF8D1D3685DF8BA
:101F9000044B0133D36070470C2B05D0F2D8092BCA
:101FA000D8D00B2BE8D0EAE7D3685DF8044B0233B6
:101FB000D360704748F29033C2F2010310B4D3F8F3
:101FC00090201368506819780478507A137A044284
:101FD00001EA03011AD0937A03F0030309B143F035
:101FE000040343F008039910082B91722AD8072B99
:101FF00022D2032B2ED011D9042B13D0062B14D1AF
:10200000D3685DF8044B023BD3607047937A03F0CA
:1020100003030029E7D043F00403E4E7012B0BD0CE
:10202000022B02D1D368013BD3605DF8044B7047AB
:102030000D2BF7D00E2BF8D1D3685DF8044B01338C
:10204000D36070470C2B05D0F2D8092BD8D00B2BBE
:10205000E8D0EAE7D3685DF8044B0233D3607047F9
:1020600048F29033C2F2010310B4D3F894201368FD
:10207000506819780478507A137A044201EA03010F
:102080001AD0937A03F0030309B143F0040343F039
:1020900008039910082B91722AD8072B22D2032B00
:1020A0002ED011D9042B13D0062B14D1D3685DF890
:1020B000044B023BD3607047937A03F0030300297B
:1020C000E7D043F00403E4E7012B0BD0022B02D14D
:1020D000D368013BD3605DF8044B70470D2BF7D0FC
:1020E0000E2BF8D1D3685DF8044B0133D3607047F1
:1020F0000C2B05D0F2D8092BD8D00B2BE8D0EAE76F
:10210000D3685DF8044B0233D360704748F29033D4
:10211000C2F2010310B4D3F89820136850681978FC
:102120000478507A137A044201EA03011AD0937AB0
:1021300003F0030309B143F0040343F008039910CB
:10214000082B91722AD8072B22D2032B2ED011D91B
:10215000042B13D0062B14D1D3685DF8044B023B3B
:10216000D3607047937A03F003030029E7D043F06C
:102170000403E4E7012B0BD0022B02D1D368013B0F
:10218000D3605DF8044B70470D2BF7D00E2BF8D1C0
:10219000D3685DF8044B0133D36070470C2B05D036
:1021A000F2D8092BD8D00B2BE8D0EAE7D3685DF83A
:1021B000044B0233D360704748F29033C2F20103FC
:1021C00010B4D3F89C201368506819780478507ABA
:1021D000137A044201EA03011AD0937A03F003034D
:1021E00009B143F0040343F008039910082B9172DE
:1021F0002AD8072B22D2032B2ED011D9042B13D08F
:10220000062B14D1D3685DF8044B023BD3607047B2
:10221000937A03F003030029E7D043F00403E4E7D3
:10222000012B0BD0022B02D1D368013BD3605DF8A8
:10223000044B70470D2BF7D00E2BF8D1D3685DF807
:10224000044B0133D36070470C2B05D0F2D8092B17
:10225000D8D00B2BE8D0EAE7D3685DF8044B023303
:10226000D360704748F29033C2F2010310B4D3F840
:10227000A0201368506819780478507A137A0442C1
:1022800001EA03011AD0937A03F0030309B143F082
:10229000040343F008039910082B91722AD8072BE6
:1022A00022D2032B2ED011D9042B13D0062B14D1FC
:1022B000D3685DF8044B023BD3607047937A03F018
:1022C00003030029E7D043F00403E4E7012B0BD01C
:1022D000022B02D1D368013BD3605DF8044B7047F9
:1022E0000D2BF7D00E2BF8D1D3685DF8044B0133DA
:1022F000D36070470C2B05D0F2D8092BD8D00B2B0C
:10230000E8D0EAE7D3685DF8044B0233D360704746
:1023100048F29033C2F2010310B4D3F8A42013683A
:10232000506819780478507A137A044201EA03015C
:102330001AD0937A03F0030309B143F0040343F086
:1023400008039910082B91722AD8072B22D2032B4D
:102350002ED011D9042B13D0062B14D1D3685DF8DD
:10236000044B023BD3607047937A03F003030029C8
:10237000E7D043F00403E4E7012B0BD0022B02D19A
:10238000D368013BD3605DF8044B70470D2BF7D049
:102390000E2BF8D1D3685DF8044B0133D36070473E
:1023A0000C2B05D0F2D8092BD8D00B2BE8D0EAE7BC
:1023B000D3685DF8044B0233D360704748F2903322
:1023C000C2F2010310B4D3F8A8201368506819783A
:1023D0000478507A137A044201EA03011AD0937AFE
:1023E00003F0030309B143F0040343F00803991019
:1023F000082B91722AD8072B22D2032B2ED011D969
:10240000042B13D0062B14D1D3685DF8044B023B88
:10241000D3607047937A03F003030029E7D043F0B9
:102420000403E4E7012B0BD0022B02D1D368013B5C
:10243000D3605DF8044B70470D2BF7D00E2BF8D10D
:10244000D3685DF8044B0133D36070470C2B05D083
:10245000F2D8092BD8D00B2BE8D0EAE7D3685DF887
:10246000044B0233D360704748F29033C2F2010349
:1024700010B4D3F8AC201368506819780478507AF7
:10248000137A044201EA03011AD0937A03F003039A
:1024900009B143F0040343F008039910082B91722B
:1024A0002AD8072B22D2032B2ED011D9042B13D0DC
:1024B000062B14D1D3685DF8044B023BD360704700
:1024C000937A03F003030029E7D043F00403E4E721
:1024D000012B0BD0022B02D1D368013BD3605DF8F6
:1024E000044B70470D2BF7D00E2BF8D1D3685DF855
:1024F000044B0133D36070470C2B05D0F2D8092B65
:10250000D8D00B2BE8D0EAE7D3685DF8044B023350
:10251000D360704748F29033C2F2010310B4D3F88D
:10252000B0201368506819780478507A137A0442FE
:1025300001EA03011AD0937A03F0030309B143F0CF
:10254000040343F008039910082B91722AD8072B33
:1025500022D2032B2ED011D9042B13D0062B14D149
:10256000D3685DF8044B023BD3607047937A03F065
:1025700003030029E7D043F00403E4E7012B0BD069
:10258000022B02D1D368013BD3605DF8044B704746
:102590000D2BF7D00E2BF8D1D3685DF8044B013327
:1025A000D36070470C2B05D0F2D8092BD8D00B2B59
:1025B000E8D0EAE7D3685DF8044B0233D360704794
:1025C00048F29033C2F2010310B4D3F8B420136878
:1025D000506819780478507A137A044201EA0301AA
:1025E0001AD0937A03F0030309B143F0040343F0D4
:1025F00008039910082B91722AD8072B22D2032B9B
:102600002ED011D9042B13D0062B14D1D3685DF82A
:10261000044B023BD3607047937A03F00303002915
:10262000E7D043F00403E4E7012B0BD0022B02D1E7
:10263000D368013BD3605DF8044B70470D2BF7D096
:102640000E2BF8D1D3685DF8044B0133D36070478B
:102650000C2B05D0F2D8092BD8D00B2BE8D0EAE709
:10266000D3685DF8044B0233D360704748F290336F
:10267000C2F2010310B41A6813685068197804781C
:10268000507A137A044201EA03011AD0937A03F0D4
:10269000030309B143F0040343F008039910082B26
:1026A00091722AD8072B22D2032B2ED011D9042BBA
:1026B00013D0062B14D1D3685DF8044B023BD360D2
:1026C0007047937A03F003030029E7D043F0040333
:1026D000E4E7012B0BD0022B02D1D368013BD3607E
:1026E0005DF8044B70470D2BF7D00E2BF8D1D36853
:1026F0005DF8044B0133D36070470C2B05D0F2D842
:10270000092BD8D00B2BE8D0EAE7D3685DF8044B4F
:102710000233D360704700BF48F29033C2F2010326
:1027200010B45A681368506819780478507A137A8C
:10273000044201EA03011AD0937A03F0030309B1BA
:1027400043F0040343F008039910082B91722AD830
:10275000072B22D2032B2ED011D9042B13D0062BFA
:1027600014D1D3685DF8044B023BD3607047937A71
:1027700003F003030029E7D043F00403E4E7012B4F
:102780000BD0022B02D1D368013BD3605DF8044B20
:1027900070470D2BF7D00E2BF8D1D3685DF8044BA2
:1027A0000133D36070470C2B05D0F2D8092BD8D059
:1027B0000B2BE8D0EAE7D3685DF8044B0233D36013
:1027C000704700BF48F29033C2F2010310B49A6818
:1027D0001368506819780478507A137A044201EA31
:1027E00003011AD0937A03F0030309B143F0040301
:1027F00043F008039910082B91722AD8072B22D294
:10280000032B2ED011D9042B13D0062B14D1D3684F
:102810005DF8044B023BD3607047937A03F00303E7
:102820000029E7D043F00403E4E7012B0BD0022B8F
:1028300002D1D368013BD3605DF8044B70470D2B88
:10284000F7D00E2BF8D1D3685DF8044B0133D36079
:1028500070470C2B05D0F2D8092BD8D00B2BE8D021
:10286000EAE7D3685DF8044B0233D360704700BFDA
:1028700048F29033C2F2010310B4DA68136850686A
:1028800019780478507A137A044201EA03011AD0C5
:10289000937A03F0030309B143F0040343F0080300
:1028A0009910082B91722AD8072B22D2032B2ED0F5
:1028B00011D9042B13D0062B14D1D3685DF8044B27
:1028C000023BD3607047937A03F003030029E7D0FB
:1028D00043F00403E4E7012B0BD0022B02D1D368B1
:1028E000013BD3605DF8044B70470D2BF7D00E2BE6
:1028F000F8D1D3685DF8044B0133D36070470C2BDB
:1029000005D0F2D8092BD8D00B2BE8D0EAE7D36852
:102910005DF8044B0233D360704700BF48F2903338
:10292000C2F2010310B41A69136850681978047868
:10293000507A137A044201EA03011AD0937A03F021
:10294000030309B143F0040343F008039910082B73
:1029500091722AD8072B22D2032B2ED011D9042B07
:1029600013D0062B14D1D3685DF8044B023BD3601F
:102970007047937A03F003030029E7D043F0040380
:10298000E4E7012B0BD0022B02D1D368013BD360CB
:102990005DF8044B70470D2BF7D00E2BF8D1D368A0
:1029A0005DF8044B0133D36070470C2B05D0F2D88F
:1029B000092BD8D00B2BE8D0EAE7D3685DF8044B9D
:1029C0000233D360704700BF48F29033C2F2010374
:1029D00010B45A691368506819780478507A137AD9
:1029E000044201EA03011AD0937A03F0030309B108
:1029F00043F0040343F008039910082B91722AD87E
:102A0000072B22D2032B2ED011D9042B13D0062B47
:102A100014D1D3685DF8044B023BD3607047937ABE
:102A200003F003030029E7D043F00403E4E7012B9C
:102A30000BD0022B02D1D368013BD3605DF8044B6D
:102A400070470D2BF7D00E2BF8D1D3685DF8044BEF
:102A50000133D36070470C2B05D0F2D8092BD8D0A6
:102A60000B2BE8D0EAE7D3685DF8044B0233D36060
:102A7000704700BF48F29033C2F2010310B49A6964
:102A80001368506819780478507A137A044201EA7E
:102A900003011AD0937A03F0030309B143F004034E
:102AA00043F008039910082B91722AD8072B22D2E1
:102AB000032B2ED011D9042B13D0062B14D1D3689D
:102AC0005DF8044B023BD3607047937A03F0030335
:102AD0000029E7D043F00403E4E7012B0BD0022BDD
:102AE00002D1D368013BD3605DF8044B70470D2BD6
:102AF000F7D00E2BF8D1D3685DF8044B0133D360C7
:102B000070470C2B05D0F2D8092BD8D00B2BE8D06E
:102B1000EAE7D3685DF8044B0233D360704700BF27
:102B200048F29033C2F2010310B4DA6913685068B6
:102B300019780478507A137A044201EA03011AD012
:102B4000937A03F0030309B143F0040343F008034D
:102B50009910082B91722AD8072B22D2032B2ED042
:102B600011D9042B13D0062B14D1D3685DF8044B74
:102B7000023BD3607047937A03F003030029E7D048
:102B800043F00403E4E7012B0BD0022B02D1D368FE
:102B9000013BD3605DF8044B70470D2BF7D00E2B33
:102BA000F8D1D3685DF8044B0133D36070470C2B28
:102BB00005D0F2D8092BD8D00B2BE8D0EAE7D368A0
:102BC0005DF8044B0233D360704700BF48F2903386
:102BD000C2F2010310B41A6A1368506819780478B5
:102BE000507A137A044201EA03011AD0937A03F06F
:102BF000030309B143F0040343F008039910082BC1
:102C000091722AD8072B22D2032B2ED011D9042B54
:102C100013D0062B14D1D3685DF8044B023BD3606C
:102C20007047937A03F003030029E7D043F00403CD
:102C3000E4E7012B0BD0022B02D1D368013BD36018
:102C40005DF8044B70470D2BF7D00E2BF8D1D368ED
:102C50005DF8044B0133D36070470C2B05D0F2D8DC
:102C6000092BD8D00B2BE8D0EAE7D3685DF8044BEA
:102C70000233D360704700BF48F29033C2F20103C1
:102C800010B45A6A1368506819780478507A137A25
:102C9000044201EA03011AD0937A03F0030309B155
:102CA00043F0040343F008039910082B91722AD8CB
:102CB000072B22D2032B2ED011D9042B13D0062B95
:102CC00014D1D3685DF8044B023BD3607047937A0C
:102CD00003F003030029E7D043F00403E4E7012BEA
:102CE0000BD0022B02D1D368013BD3605DF8044BBB
:102CF00070470D2BF7D00E2BF8D1D3685DF8044B3D
:102D00000133D36070470C2B05D0F2D8092BD8D0F3
:102D10000B2BE8D0EAE7D3685DF8044B0233D360AD
:102D2000704700BF48F29033C2F2010310B49A6AB0
:102D30001368506819780478507A137A044201EACB
:102D400003011AD0937A03F0030309B143F004039B
:102D500043F008039910082B91722AD8072B22D22E
:102D6000032B2ED011D9042B13D0062B14D1D368EA
:102D70005DF8044B023BD3607047937A03F0030382
:102D80000029E7D043F00403E4E7012B0BD0022B2A
:102D900002D1D368013BD3605DF8044B70470D2B23
:102DA000F7D00E2BF8D1D3685DF8044B0133D36014
:102DB00070470C2B05D0F2D8092BD8D00B2BE8D0BC
:102DC000EAE7D3685DF8044B0233D360704700BF75
:102DD00048F29033C2F2010310B4DA6A1368506803
:102DE00019780478507A137A044201EA03011AD060
:102DF000937A03F0030309B143F0040343F008039B
:102E00009910082B91722AD8072B22D2032B2ED08F
:102E100011D9042B13D0062B14D1D3685DF8044BC1
:102E2000023BD3607047937A03F003030029E7D095
:102E300043F00403E4E7012B0BD0022B02D1D3684B
:102E4000013BD3605DF8044B70470D2BF7D00E2B80
:102E5000F8D1D3685DF8044B0133D36070470C2B75
:102E600005D0F2D8092BD8D00B2BE8D0EAE7D368ED
:102E70005DF8044B0233D360704700BF48F29033D3
:102E8000C2F2010310B41A6B136850681978047801
:102E9000507A137A044201EA03011AD0937A03F0BC
:102EA000030309B143F0040343F008039910082B0E
:102EB00091722AD8072B22D2032B2ED011D9042BA2
:102EC00013D0062B14D1D3685DF8044B023BD360BA
:102ED0007047937A03F003030029E7D043F004031B
:102EE000E4E7012B0BD0022B02D1D368013BD36066
:102EF0005DF8044B70470D2BF7D00E2BF8D1D3683B
:102F00005DF8044B0133D36070470C2B05D0F2D829
:102F1000092BD8D00B2BE8D0EAE7D3685DF8044B37
:102F20000233D360704700BF48F29033C2F201030E
:102F300010B45A6B1368506819780478507A137A71
:102F4000044201EA03011AD0937A03F0030309B1A2
:102F500043F0040343F008039910082B91722AD818
:102F6000072B22D2032B2ED011D9042B13D0062BE2
:102F700014D1D3685DF8044B023BD3607047937A59
:102F800003F003030029E7D043F00403E4E7012B37
:102F90000BD0022B02D1D368013BD3605DF8044B08
:102FA00070470D2BF7D00E2BF8D1D3685DF8044B8A
:102FB0000133D36070470C2B05D0F2D8092BD8D041
:102FC0000B2BE8D0EAE7D3685DF8044B0233D360FB
:102FD000704700BF48F29033C2F2010310B4D3F837
:102FE000E8201368506819780478507A137A0442FC
:102FF00001EA03011AD0937A03F0030309B143F005
:10300000040343F008039910082B91722AD8072B68
:1030100022D2032B2ED011D9042B13D0062B14D17E
:10302000D3685DF8044B023BD3607047937A03F09A
:1030300003030029E7D043F00403E4E7012B0BD09E
:10304000022B02D1D368013BD3605DF8044B70477B
:103050000D2BF7D00E2BF8D1D3685DF8044B01335C
:10306000D36070470C2B05D0F2D8092BD8D00B2B8E
:10307000E8D0EAE7D3685DF8044B0233D3607047C9
:1030800048F29033C2F2010310B4D3F8EC20136875
:10309000506819780478507A137A044201EA0301DF
:1030A0001AD0937A03F0030309B143F0040343F009
:1030B00008039910082B91722AD8072B22D2032BD0
:1030C0002ED011D9042B13D0062B14D1D3685DF860
:1030D000044B023BD3607047937A03F0030300294B
:1030E000E7D043F00403E4E7012B0BD0022B02D11D
:1030F000D368013BD3605DF8044B70470D2BF7D0CC
:103100000E2BF8D1D3685DF8044B0133D3607047C0
:103110000C2B05D0F2D8092BD8D00B2BE8D0EAE73E
:10312000D3685DF8044B0233D360704748F29033A4
:10313000C2F2010310B4D3F8D8201368506819788C
:103140000478507A137A044201EA03011AD0937A80
:1031500003F0030309B143F0040343F0080399109B
:10316000082B91722AD8072B22D2032B2ED011D9EB
:10317000042B13D0062B14D1D3685DF8044B023B0B
:10318000D3607047937A03F003030029E7D043F03C
:103190000403E4E7012B0BD0022B02D1D368013BDF
:1031A000D3605DF8044B70470D2BF7D00E2BF8D190
:1031B000D3685DF8044B0133D36070470C2B05D006
:1031C000F2D8092BD8D00B2BE8D0EAE7D3685DF80A
:1031D000044B0233D360704748F29033C2F20103CC
:1031E00010B4D3F8DC201368506819780478507A4A
:1031F000137A044201EA03011AD0937A03F003031D
:1032000009B143F0040343F008039910082B9172AD
:103210002AD8072B22D2032B2ED011D9042B13D05E
:10322000062B14D1D3685DF8044B023BD360704782
:10323000937A03F003030029E7D043F00403E4E7A3
:10324000012B0BD0022B02D1D368013BD3605DF878
:10325000044B70470D2BF7D00E2BF8D1D3685DF8D7
:10326000044B0133D36070470C2B05D0F2D8092BE7
:10327000D8D00B2BE8D0EAE7D3685DF8044B0233D3
:10328000D360704748F29033C2F2010310B4D3F810
:10329000E0201368506819780478507A137A044251
:1032A00001EA03011AD0937A03F0030309B143F052
:1032B000040343F008039910082B91722AD8072BB6
:1032C00022D2032B2ED011D9042B13D0062B14D1CC
:1032D000D3685DF8044B023BD3607047937A03F0E8
:1032E00003030029E7D043F00403E4E7012B0BD0EC
:1032F000022B02D1D368013BD3605DF8044B7047C9
:103300000D2BF7D00E2BF8D1D3685DF8044B0133A9
:10331000D36070470C2B05D0F2D8092BD8D00B2BDB
:10332000E8D0EAE7D3685DF8044B0233D360704716
:1033300048F29033C2F2010310B4D3F8E4201368CA
:10334000506819780478507A137A044201EA03012C
:103350001AD0937A03F0030309B143F0040343F056
:1033600008039910082B91722AD8072B22D2032B1D
:103370002ED011D9042B13D0062B14D1D3685DF8AD
:10338000044B023BD3607047937A03F00303002998
:10339000E7D043F00403E4E7012B0BD0022B02D16A
:1033A000D368013BD3605DF8044B70470D2BF7D019
:1033B0000E2BF8D1D3685DF8044B0133D36070470E
:1033C0000C2B05D0F2D8092BD8D00B2BE8D0EAE78C
:1033D000D3685DF8044B0233D360704748F29033F2
:1033E000C2F2010310B4D3F8B820136850681978FA
:1033F0000478507A137A044201EA03011AD0937ACE
:1034000003F0030309B143F0040343F008039910E8
:10341000082B91722AD8072B22D2032B2ED011D938
:10342000042B13D0062B14D1D3685DF8044B023B58
:10343000D3607047937A03F003030029E7D043F089
:103440000403E4E7012B0BD0022B02D1D368013B2C
:10345000D3605DF8044B70470D2BF7D00E2BF8D1DD
:10346000D3685DF8044B0133D36070470C2B05D053
:10347000F2D8092BD8D00B2BE8D0EAE7D3685DF857
:10348000044B0233D360704748F29033C2F2010319
:1034900010B4D3F8BC201368506819780478507AB7
:1034A000137A044201EA03011AD0937A03F003036A
:1034B00009B143F0040343F008039910082B9172FB
:1034C0002AD8072B22D2032B2ED011D9042B13D0AC
:1034D000062B14D1D3685DF8044B023BD3607047D0
:1034E000937A03F003030029E7D043F00403E4E7F1
:1034F000012B0BD0022B02D1D368013BD3605DF8C6
:10350000044B70470D2BF7D00E2BF8D1D3685DF824
:10351000044B0133D36070470C2B05D0F2D8092B34
:10352000D8D00B2BE8D0EAE7D3685DF8044B023320
:10353000D360704748F29033C2F2010310B4D3F85D
:10354000C0201368506819780478507A137A0442BE
:1035500001EA03011AD0937A03F0030309B143F09F
:10356000040343F008039910082B91722AD8072B03
:1035700022D2032B2ED011D9042B13D0062B14D119
:10358000D3685DF8044B023BD3607047937A03F035
:1035900003030029E7D043F00403E4E7012B0BD039
:1035A000022B02D1D368013BD3605DF8044B704716
:1035B0000D2BF7D00E2BF8D1D3685DF8044B0133F7
:1035C000D36070470C2B05D0F2D8092BD8D00B2B29
:1035D000E8D0EAE7D3685DF8044B0233D360704764
:1035E00048F29033C2F2010310B4D3F8C420136838
:1035F000506819780478507A137A044201EA03017A
:103600001AD0937A03F0030309B143F0040343F0A3
:1036100008039910082B91722AD8072B22D2032B6A
:103620002ED011D9042B13D0062B14D1D3685DF8FA
:10363000044B023BD3607047937A03F003030029E5
:10364000E7D043F00403E4E7012B0BD0022B02D1B7
:10365000D368013BD3605DF8044B70470D2BF7D066
:103660000E2BF8D1D3685DF8044B0133D36070475B
:103670000C2B05D0F2D8092BD8D00B2BE8D0EAE7D9
:10368000D3685DF8044B0233D360704748F290333F
:10369000C2F2010310B4D3F8C82013685068197837
:1036A0000478507A137A044201EA03011AD0937A1B
:1036B00003F0030309B143F0040343F00803991036
:1036C000082B91722AD8072B22D2032B2ED011D986
:1036D000042B13D0062B14D1D3685DF8044B023BA6
:1036E000D3607047937A03F003030029E7D043F0D7
:1036F0000403E4E7012B0BD0022B02D1D368013B7A
:10370000D3605DF8044B70470D2BF7D00E2BF8D12A
:10371000D3685DF8044B0133D36070470C2B05D0A0
:10372000F2D8092BD8D00B2BE8D0EAE7D3685DF8A4
:10373000044B0233D360704748F29033C2F2010366
:1037400010B4D3F8CC201368506819780478507AF4
:10375000137A044201EA03011AD0937A03F00303B7
:1037600009B143F0040343F008039910082B917248
:103770002AD8072B22D2032B2ED011D9042B13D0F9
:10378000062B14D1D3685DF8044B023BD36070471D
:10379000937A03F003030029E7D043F00403E4E73E
:1037A000012B0BD0022B02D1D368013BD3605DF813
:1037B000044B70470D2BF7D00E2BF8D1D3685DF872
:1037C000044B0133D36070470C2B05D0F2D8092B82
:1037D000D8D00B2BE8D0EAE7D3685DF8044B02336E
:1037E000D360704748F29033C2F2010310B4D3F8AB
:1037F000D0201368506819780478507A137A0442FC
:1038000001EA03011AD0937A03F0030309B143F0EC
:10381000040343F008039910082B91722AD8072B50
:1038200022D2032B2ED011D9042B13D0062B14D166
:10383000D3685DF8044B023BD3607047937A03F082
:1038400003030029E7D043F00403E4E7012B0BD086
:10385000022B02D1D368013BD3605DF8044B704763
:103860000D2BF7D00E2BF8D1D3685DF8044B013344
:10387000D36070470C2B05D0F2D8092BD8D00B2B76
:10388000E8D0EAE7D3685DF8044B0233D3607047B1
:1038900048F29033C2F2010310B4D3F8D420136875
:1038A000506819780478507A137A044201EA0301C7
:1038B0001AD0937A03F0030309B143F0040343F0F1
:1038C00008039910082B91722AD8072B22D2032BB8
:1038D0002ED011D9042B13D0062B14D1D3685DF848
:1038E000044B023BD3607047937A03F00303002933
:1038F000E7D043F00403E4E7012B0BD0022B02D105
:10390000D368013BD3605DF8044B70470D2BF7D0B3
:103910000E2BF8D1D3685DF8044B0133D3607047A8
:103920000C2B05D0F2D8092BD8D00B2BE8D0EAE726
:10393000D3685DF8044B0233D3607047F0B540F6AE
:103940006453C2F201034DF20A721B68C3F62342AC
:1039500006EE102A93F89D2093F89F6007EE102A38
:1039600093F89620B8EEC77A07EE902A27EE067AEB
:10397000F8EEE76A83B067EE267A0D46FCEEE77A4A
:103980000021CDED017A044683F893509DF8042080
:1039900083F8921083F8911083F890100EB183F899
:1039A000902093F89E1009B183F8912093F8A0100D
:1039B00009B183F8922093F8A52093F8A70007EEA9
:1039C000102A4DF20A72C3F6234206EE102A93F82B
:1039D0009420B8EEC77A07EE902A27EE067AF8EE22
:1039E000E76A67EE267AFCEEE77ACDED017A9DF87C
:1039F000042030B193F89000904238BF104683F80D
:103A0000900093F8A60030B193F89100904238BF2F
:103A1000104683F8910093F8A80030B193F89260B3
:103A2000B24238BF324683F8922093F8A12093F82F
:103A3000A36007EE102A4DF20A72C3F6234206EE87
:103A4000102A93F89520B8EEC77A07EE902A27EE51
:103A5000067AF8EEE76A67EE267AFCEEE77ACDEDB5
:103A6000017A9DF8042036B193F89060964238BFF1
:103A7000164683F8906093F8A26036B193F891608F
:103A8000964238BF164683F8916093F8A46036B129
:103A900093F89270BA4238BF3A4683F8922093F86E
:103AA000A92093F8AB7007EE902A4DF20A72C3F684
:103AB000234207EE102AF8EEE77A67EE877A07EEE0
:103AC000105AB8EEC77A67EE877AFCEEE77ACDED4A
:103AD000017A9DF8042037B193F89070974238BF6F
:103AE000174683F8907093F8AA7037B193F89170E5
:103AF000974238BF174683F8917093F8AC7037B18E
:103B000093F892E0724538BF724683F8922029B943
:103B100026B918B917B97F2283F8922043F22C00F6
:103B20000D21C0F2020019F049FE611EC9B20F2931
:103B30000FD840F67474C2F2010441F0D001A06CB9
:103B400003681B689847A06C036805F07F011B6839
:103B5000984742F678600F21C0F2020019F02EFE5D
:103B60004EF20020C2F2000003B0BDE8F04015F0B4
:103B7000A1BF00BFF0B540F66453C2F201034DF29D
:103B80000A721B68C3F6234206EE102A93F89D20A2
:103B900093F89F6007EE102A93F89620B8EEC77A44
:103BA00007EE902A27EE067AF8EEE76A83B067EE12
:103BB000267A0C46FCEEE77A0021CDED017A054627
:103BC00083F893409DF8042083F8921083F89110B5
:103BD00083F890100EB183F8902093F89E1009B1ED
:103BE00083F8912093F8A01009B183F8922093F8FC
:103BF000A52093F8A70007EE102A4DF20A72C3F62B
:103C0000234206EE102A93F89420B8EEC77A07EE06
:103C1000902A27EE067AF8EEE76A67EE267AFCEE3F
:103C2000E77ACDED017A9DF8042030B193F8900049
:103C3000904238BF104683F8900093F8A60030B148
:103C400093F89100904238BF104683F8910093F8A2
:103C5000A80030B193F89260B24238BF324683F880
:103C6000922093F8A12093F8A36007EE102A4DF25A
:103C70000A72C3F6234206EE102A93F89520B8EE96
:103C8000C77A07EE902A27EE067AF8EEE76A67EE23
:103C9000267AFCEEE77ACDED017A9DF8042036B164
:103CA00093F89060964238BF164683F8906093F878
:103CB000A26036B193F89160964238BF164683F8F9
:103CC000916093F8A46036B193F89270BA4238BF0D
:103CD0003A4683F8922093F8A92093F8AB7007EE48
:103CE000902A4DF20A72C3F6234207EE102AF8EE2C
:103CF000E77A67EE877A07EE104AB8EEC77A67EE82
:103D0000877AFCEEE77ACDED017A9DF8042037B191
:103D100093F89070974238BF174683F8907093F8E5
:103D2000AA7037B193F89170974238BF174683F85D
:103D3000917093F8AC7037B193F892E0724538BF48
:103D4000724683F8922029B926B918B917B97F228B
:103D500083F8922043F23C000D21C0F202002404BB
:103D600019F02CFD04F4FE04681E44F450440002D3
:103D700044F00D0400F47060204318F095FE42F604
:103D800004600F21C0F2020019F018FD4EF200206D
:103D9000C2F2000003B0BDE8F04015F08BBE00BFDA
:103DA00070B5044643F24C000E46C0F202001221E8
:103DB000154619F003FD611EC9B20F2915D840F64A
:103DC0007474C2F2010441F0A001A06C03681B6886
:103DD0009847A06C036806F07F011B689847A06CA9
:103DE000036805F07F011B68984743F26000C0F24A
:103DF00002000A2119F0E2FC4EF20020C2F200009B
:103E0000BDE8704015F056BEF8B54DF67067C2F2C9
:103E1000000705463B7C0E4614467BB398422DD0E6
:103E200043F26C001E21C0F2020019F0C7FC4EF2F2
:103E3000002000230A222946C2F2000015F04CFEA1
:103E400043F28C000E21C0F2020019F0B7FC4EF2D2
:103E50000020397C00230A22C2F2000015F03CFE4B
:103E600043F29C000121C0F2020019F0A7FC4EF2BF
:103E70000020C2F2000015F01DFE08E040F6645379
:103E8000C2F201032246186831460BF009FB43F2E7
:103E9000A0001121C0F2020019F090FC230603F0EB
:103EA000FE43300443F41043013D43F0090300F4A2
:103EB000FE002D02184305F47065284318F0F4FD48
:103EC00042F60460C0F202000F2119F077FC4EF2B6
:103ED0000020C2F20000BDE8F84015F0EBBD00BFC5
:103EE000F8B54DF67067C2F2000705463B7C0E46FA
:103EF00014467BB398422DD043F26C001E21C0F2D1
:103F0000020019F05BFC4EF2002000230A22294631
:103F1000C2F2000015F0E0FD43F28C000E21C0F269
:103F2000020019F04BFC4EF20020397C00230A22DB
:103F3000C2F2000015F0D0FD43F29C000121C0F256
:103F4000020019F03BFC4EF20020C2F2000015F016
:103F5000B1FD07E040F66453C2F201033146186830
:103F60000BF066FC43F2B4001221C0F2020019F01B
:103F700025FC230603F0FE43300443F40043013DD7
:103F800043F0080300F4FE002D02184305F47065A9
:103F9000284318F089FD42F60460C0F202000F21A8
:103FA00019F00CFC4EF20020C2F20000BDE8F8400F
:103FB00015F080BDF8B54DF67065C2F200050446F7
:103FC0002B7C0E4617467BB398422DD043F26C00F3
:103FD0001E21C0F2020019F0F1FB4EF20020002376
:103FE0000A222146C2F2000015F076FD43F28C0051
:103FF0000E21C0F2020019F0E1FB4EF20020297CF4
:1040000000230A22C2F2000015F066FD43F29C0074
:104010000121C0F2020019F0D1FB4EF20020C2F2E1
:10402000000015F047FD07E040F66453C2F20103BB
:10403000314618680BF0FCFB43F2C8001221C0F2B5
:104040000200013C19F0BAFBE1B20F2915D840F685
:104050007475C2F2010541F08001A86C03681B6809
:104060009847A86C036806F07F011B689847A86C06
:10407000036807F07F011B68984742F67860C0F23A
:1040800002000F2119F09AFB4EF20020C2F200004C
:10409000BDE8F84015F00EBDF8B54DF67065C2F2FA
:1040A000000504462B7C0E4617467BB398422DD064
:1040B00043F26C001E21C0F2020019F07FFB4EF2A9
:1040C000002000230A222146C2F2000015F004FD60
:1040D00043F28C000E21C0F2020019F06FFB4EF289
:1040E0000020297C00230A22C2F2000015F0F4FC13
:1040F00043F29C000121C0F2020019F05FFB4EF276
:104100000020C2F2000015F0D5FC08E040F6645330
:10411000C2F201033A46186831460BF0C1F943F286
:10412000DC001121C0F20200013C19F047FBE1B2B2
:104130000F2915D840F67475C2F2010541F09001BF
:10414000A86C03681B689847A86C036806F07F0199
:104150001B689847A86C036807F07F011B689847A5
:1041600042F67860C0F202000F2119F027FB4EF2F0
:104170000020C2F20000BDE8F84015F09BBC00BF73
:1041800038B540F66453C2F2010304461B6801F5DA
:10419000005543F2F0000D21C3F88450C0F2020034
:1041A00019F00CFB611EC9B20F2915D840F67474C2
:1041B000C2F2010441F0E001A06C03681B6898475B
:1041C000A06C036805F07F011B689847A06C03682A
:1041D000C5F3C6111B68984742F67860C0F202002A
:1041E0000F2119F0EBFA4EF20020C2F20000BDE8F8
:1041F000384015F05FBC00BF10B442F69054002365
:10420000C0F202044172026104600372C36041B1F2
:10421000194600E0026942F82310427A01339A42BB
:10422000F8DC48F29043C2F201031A680AB90CE0C4
:104230001A465369002BFBD15061002343618380F0
:10424000C38083725DF8044B70471860F5E700BFC8
:10425000F8B540F67474C2F2010447F61221A06C5E
:104260000368DB69984743F6E167032043F6096377
:1042700046F6990143F6753641F20D0284F8640062
:10428000C0F20003C0F20007C0F20001C0F2000655
:10429000C0F2000240F6515063602760E160666141
:1042A000A261C0F2000045F6853340F6CD4740F6E6
:1042B000B55140F6894640F699122061C0F20003DC
:1042C000C0F20007C0F20001C0F20006C0F2000216
:1042D00040F63570E3612762A160A662E262C0F237
:1042E000000040F6D11340F6092740F6412140F680
:1042F000792640F6B132C0F200022063C0F200031A
:10430000C0F20007C0F20001C0F200064EF2002524
:1043100043F200106264C2F200056363A7630023E6
:104320004FF6FF77E16326641721C0F2020084F89C
:104330004C3084F84E3084F84D30A365636584F8C2
:10434000E93084F8663084F8653084F8673084F8A2
:104350006830E765276619F031FA284615F0AAFBA0
:1043600048F27071C2F2010144F2990EC0F2000EDF
:1043700048F26874C1F800E0C2F2010443F6B57E69
:10438000C0F2000E48F26C73C4F800E0C2F2010300
:1043900046F2BD7EC0F2000E48F24077C3F800E05E
:1043A000C2F2010743F63D1EC0F2000E48F2307023
:1043B000C7F800E0C2F2010044F2811EC0F2000E14
:1043C00048F22C76C0F800E0C2F2010641F27D0E00
:1043D000C0F2000E48F25072C6F800E0C2F20102CC
:1043E00045F6C53EC0F2000E48F24871C2F800E042
:1043F000C2F2010140F6096EC0F2000E48F23C74B0
:10440000C1F800E0C2F2010443F6A15EC0F2000E62
:1044100048F26473C4F800E0C2F2010340F6556E3E
:10442000C0F2000E48F24C77C3F800E0C2F2010778
:1044300040F6115EC0F2000E48F21470C7F800E0BA
:10444000C2F2010040F69D77C0F2000748F24476C0
:104450000760C2F2010648F2247240F63137C2F218
:104460000102C0F2000748F25C7140F6713037601B
:10447000C2F20101C0F2000048F21C7448F2187345
:1044800040F6B127C2F201031060C2F20104C0F28B
:10449000000740F6F12640F6194243F218100F606B
:1044A000C0F20006C0F20002C0F20200182126602D
:1044B0001A6019F083F92846BDE8F84015F0FABAF9
:1044C0001D2810B50B4600F0E983024622D92C289E
:1044D00000F064813FD8242800F0EE8340F2A880E9
:1044E000282800F0748300F2D680262800F0F58199
:1044F00040F2D58248F29034C2F2010442F2B9117E
:10450000C0F2000104222720C4F89C3016F06EF897
:10451000012010BD0E2800F097833AD8062800F03D
:10452000A1836CD90A2800F0058300F207810828CE
:1045300000F07E8140F2758248F29034C2F20104AC
:1045400042F67941C0F2000104220920636216F0AC
:104550004DF8012010BD342800F0BD8336D8302836
:1045600000F0638300F2D6802E2800F0528140F2E2
:10457000018248F29034C2F2010443F28941C0F250
:10458000000104222F20C4F8BC3016F02FF80120BF
:1045900010BD152800F0748364D9192800F0FA8141
:1045A00000F2A580172800F08A8140F2D18248F2FB
:1045B0009034C2F2010441F2A571C0F2000104225C
:1045C0001820236616F012F8012010BD382800F0DC
:1045D000CE8275D8362800F0398140F27F8248F2C9
:1045E0009034C2F2010443F2D911C0F20001042256
:1045F0003720C4F8DC3015F0F9FF012010BD022887
:1046000000F0018240F27881042800F04B8140F2F2
:10461000BD8248F29034C2F2010442F6C911C0F2E0
:10462000000104220520636115F0E0FF012010BDA8
:10463000202800F0448240F28981222800F0238162
:1046400040F2D48248F29034C2F2010441F609717A
:10465000C0F2000104222320C4F88C3015F0C6FFFC
:10466000012010BD112800F0B18140F25A811328B9
:1046700000F0FB8040F2B88148F29034C2F20104AD
:1046800041F2F541C0F2000104221420236515F027
:10469000ADFF012010BD2A2800F0AC8040F2E0817F
:1046A00048F29034C2F2010442F26941C0F20001C2
:1046B00004222B20C4F8AC3015F098FF012010BD67
:1046C0003A2800F08880C0F072823B2840F06D826A
:1046D00048F29034C2F2010443F28101C0F20001B9
:1046E0000422C4F8EC3015F081FF012010BD1B2816
:1046F00063D040F28B8248F29034C2F2010441F65A
:104700005521C0F2000104221C20236715F06EFF22
:10471000012010BD322824D040F2928148F290341A
:10472000C2F2010443F23971C0F2000104223320C5
:10473000C4F8CC3015F05AFF012010BD0C281FD052
:1047400040F29E8148F29034C2F2010442F629718F
:10475000C0F2000104220D20636315F047FF012021
:1047600010BD48F29034C2F2010443F28D61C0F2F0
:1047700000010422C4F8C83015F038FF012010BD34
:1047800048F29034C2F2010442F67D61C0F20001A9
:104790000422236315F02AFF012010BD48F2903453
:1047A000C2F2010442F21551C0F200010422C4F821
:1047B000B03015F01BFF012010BD48F29034C2F25A
:1047C000010441F6A911C0F200010422E36615F0CC
:1047D0000DFF012010BD48F29034C2F2010442F6F0
:1047E000D571C0F200010422C4F8E83015F0FEFED5
:1047F000012010BD48F29034C2F2010442F2BD31F2
:10480000C0F200010422C4F8A83015F0EFFE012028
:1048100010BD48F29034C2F2010443F2DD31C0F21F
:1048200000010422C4F8B83015F0E0FE012010BDEC
:1048300048F29034C2F2010442F6CD31C0F20001D8
:104840000422236215F0D2FE012010BD48F29034FC
:10485000C2F2010443F22D11C0F200010422C4F897
:10486000D83015F0C3FE012010BD48F29034C2F2DA
:10487000010441F24941C0F200010422E36415F051
:10488000B5FE012010BD48F29034C2F2010441F699
:104890005D61C0F200010422C4F8883015F0A6FE64
:1048A000012010BD48F29034C2F2010442F61D11FD
:1048B000C0F20001236115F099FE012010BD48F2FD
:1048C0009034C2F2010441F2F961C0F20001042205
:1048D000E36515F08BFE012010BD48F29034C2F262
:1048E000010442F20D11C0F200010422C4F8983014
:1048F00015F07CFE012010BD002800F0FF8001288B
:1049000040F0538148F29034C2F2010442F219712E
:10491000C0F2000104220120636015F067FE01204F
:1049200010BD0F2800F0F880102840F03E8148F2BA
:104930009034C2F2010441F24521C0F20001042288
:104940001020236415F052FE012010BD1E282FD028
:104950001F2840F02A8148F29034C2F2010441F647
:104960005941C0F2000104221F20E36715F03EFE0A
:10497000012010BD48F29034C2F2010442F2C1514C
:10498000C0F2000104222D20C4F8B43015F02EFE30
:10499000012010BD48F29034C2F2010441F65101E9
:1049A000C0F200010422636615F020FE012010BD54
:1049B00048F29034C2F2010441F6AD31C0F2000178
:1049C0000422A36715F012FE012010BD48F29034B6
:1049D000C2F2010441F2F121C0F200010422636439
:1049E00015F004FE012010BD48F29034C2F201041B
:1049F00041F29D31C0F2000104221220A36415F09F
:104A0000F5FD012010BD48F29034C2F2010442F2DB
:104A1000C571C0F200010422A36015F0E7FD01207A
:104A200010BD48F29034C2F2010442F62131C0F2C6
:104A3000000104220720E36115F0D8FD012010BD1C
:104A400048F29034C2F2010443F2E151C0F2000195
:104A500004223120C4F8C43015F0C8FD012010BD77
:104A600048F29034C2F2010442F21131C0F2000166
:104A700004222920C4F8A43015F0B8FD012010BD8F
:104A800048F29034C2F2010442F6D151C0F2000162
:104A900004220B20E36215F0A9FD012010BD48F2AD
:104AA0009034C2F2010442F26101C0F2000104221A
:104AB0002520C4F8943015F099FD012010BD48F26E
:104AC0009034C2F2010441F60551C0F20001042203
:104AD000C4F8803015F08AFD012010BD48F29034F2
:104AE000C2F2010443F69101C0F200010422352014
:104AF000C4F8D43015F07AFD012010BD48F290348E
:104B0000C2F2010442F26D61C0F20001042223608E
:104B100015F06CFD012010BD48F29034C2F2010482
:104B200041F29911C0F200010422E36315F05EFD29
:104B3000012010BD48F29034C2F2010442F6255122
:104B4000C0F200010422A36215F050FD012010BD47
:104B500048F29034C2F2010441F24D61C0F200010A
:104B600004221620A36515F041FD012010BD48F276
:104B70009034C2F2010443F28521C0F20001042204
:104B8000C4F8E03015F032FD012010BD48F2903439
:104B9000C2F2010442F67101C0F2000104220320B6
:104BA000E36015F023FD012010BD002010BD48F288
:104BB0009034C2F2010443F23131C0F20001042208
:104BC0003920C4F8E43015F011FD012010BD48F281
:104BD0009034C2F2010442F26521C0F200010422C5
:104BE000C4F8A03015F002FD012010BD48F2903449
:104BF000C2F2010441F6B151C0F2000104222120A9
:104C0000C4F8843015F0F2FC012010BD48F2903455
:104C1000C2F2010441F6FD01C0F2000104221A2093
:104C2000A36615F0E3FC012010BD48F29034C2F2F7
:104C3000010443F23551C0F200010422C4F8C0302F
:104C400015F0D4FC012010BD48F29034C2F20104EA
:104C500041F2ED01C0F200010422A36315F0C6FC8D
:104C6000012010BD48F29034C2F2010442F67521D1
:104C7000C0F200010422A36115F0B8FC012010BDB0
:104C800048F29034C2F2010441F2A151C0F2000195
:104C90000422636515F0AAFC012010BD48F290348F
:104CA000C2F2010441F60131C0F20001042263673F
:104CB00015F09CFC012010BD48F29034C2F20104B2
:104CC00041F6B571C0F200010422C4F8903015F02D
:104CD0008DFC012010BD48F29034C2F2010443F271
:104CE000E571C0F200010422C4F8D03015F07EFC5A
:104CF000012010BDF8B5044616460D4608460221AF
:104D000015F0B8FE3046022115F0B4FE44F26C33C3
:104D1000C0F20203012253F83500227200F500713F
:104D2000216053F8361062724FF4625301F5007738
:104D300062F31F4300226760E260013BFDD190F8FF
:104D4000003291F8002203F00103D20744BF43F080
:104D50000203DBB21D2DA37200F00F8422D92C2D8B
:104D600000F070813FD8242D00F0168440F2A88016
:104D7000282D00F0968300F2D680262D00F00D82BB
:104D800040F2F28248F29033C2F2010342F2B911CA
:104D9000C0F2000104222720C3F89C4015F026FC35
:104DA000012326E10E2D00F0BB833AD8062D00F03A
:104DB000C6836CD90A2D00F0258300F20881082DE6
:104DC00000F08F8140F2928248F29033C2F20103E8
:104DD00042F67941C0F20001042209205C6215F01C
:104DE00005FC012305E1342D00F0E68336D8302D93
:104DF00000F0868300F2D7802E2D00F0628140F211
:104E00001A8248F29033C2F2010343F28941C0F2A0
:104E1000000104222F20C3F8BC4015F0E7FB01235A
:104E2000E7E0152D00F09A8364D9192D00F0138264
:104E300000F2A680172D00F0A18140F2F28248F224
:104E40009033C2F2010341F2A571C0F200010422C5
:104E500018201C6615F0CAFB0123CAE0382D00F0AB
:104E6000EF8275D8362D00F04B8140F29D8248F2DA
:104E70009033C2F2010343F2D911C0F200010422BF
:104E80003720C3F8DC4015F0B1FB0123B1E0022D5F
:104E900000F01D8240F29181042D00F0608140F20B
:104EA000DF8248F29033C2F2010342F6C911C0F228
:104EB0000001042205205C6115F098FB012398E0B5
:104EC000202D00F0618240F2A281222D00F0378176
:104ED00040F2F78248F29033C2F2010341F60971C1
:104EE000C0F2000104222320C3F88C4015F07EFBA1
:104EF00001237EE0112D00F0CC8140F27381132D4F
:104F000000F00E8140F2D48148F29033C2F20103E6
:104F100041F2F541C0F20001042214201C6515F095
:104F200065FB012365E02A2D00F0BB8040F2FD8186
:104F300048F29033C2F2010342F26941C0F200012B
:104F400004222B20C3F8AC4015F050FB012350E0A5
:104F50003A2D00F09680C0F094823B2D40F08F8275
:104F600048F29033C2F2010343F281012846C0F2B5
:104F700000010422C3F8EC4015F038FB012338E0AF
:104F80001B2D6FD040F2AD8248F29033C2F2010384
:104F900041F65521C0F2000104221C201C6715F0C7
:104FA00025FB012325E0322D2DD040F2AE8148F2C1
:104FB0009033C2F2010343F23971C0F200010422BE
:104FC0003320C3F8CC4015F011FB012311E00C2D68
:104FD00029D040F2BA8148F29033C2F2010342F67E
:104FE0002971C0F2000104220D205C6315F0FEFA65
:104FF0000123237430462146FFF762FA237C1844CC
:1050000020742046F8BD48F29033C2F2010343F207
:105010008D612846C0F200010422C3F8C84015F093
:10502000E5FA0123E5E748F29033C2F2010342F6C4
:105030007D612846C0F2000104221C6315F0D6FAF7
:105040000123D6E748F29033C2F2010342F2155130
:105050002846C0F200010422C3F8B04015F0C6FA99
:105060000123C6E748F29033C2F2010341F6A911C9
:105070002846C0F200010422DC6615F0B7FA0123CD
:10508000B7E748F29033C2F2010342F6D5712846E1
:10509000C0F200010422C3F8E84015F0A7FA01238A
:1050A000A7E748F29033C2F2010342F2BD3128462D
:1050B000C0F200010422C3F8A84015F097FA0123BA
:1050C00097E748F29033C2F2010343F2DD312846FC
:1050D000C0F200010422C3F8B84015F087FA01239A
:1050E00087E748F29033C2F2010342F6CD312846F9
:1050F000C0F2000104221C6215F078FA012378E75F
:1051000048F29033C2F2010343F22D112846C0F257
:1051100000010422C3F8D84015F068FA012368E7BB
:1051200048F29033C2F2010341F249412846C0F2ED
:1051300000010422DC6415F059FA012359E748F212
:105140009033C2F2010341F65D612846C0F20001CE
:105150000422C3F8884015F049FA012349E748F2D0
:105160009033C2F2010342F61D11C0F200012A463B
:1051700028461C6115F03AFA01233AE748F29033C9
:10518000C2F2010341F2F9612846C0F20001042293
:10519000DC6515F02BFA01232BE748F29033C2F2BD
:1051A000010342F20D112846C0F200010422C3F8A7
:1051B000984015F01BFA01231BE7002D00F0048135
:1051C000012D40F05C8148F29033C2F2010342F2BB
:1051D0001971C0F20001042201205C6015F006FA8A
:1051E000012306E70F2D00F0FE80102D40F04781CF
:1051F00048F29033C2F2010341F24521C0F20001AE
:10520000042210201C6415F0F1F90123F1E61E2D93
:1052100030D01F2D40F0338148F29033C2F20103A9
:1052200041F65941C0F2000104221F20DC6715F04D
:10523000DDF90123DDE648F29033C2F2010342F2C8
:10524000C151C0F2000104222D20C3F8B44015F072
:10525000CDF90123CDE648F29033C2F2010341F6C5
:1052600051012846C0F2000104225C6615F0BEF927
:105270000123BEE648F29033C2F2010341F6AD319C
:105280002846C0F2000104229C6715F0AFF9012303
:10529000AFE648F29033C2F2010341F2F121284611
:1052A000C0F2000104225C6415F0A0F90123A0E61D
:1052B00048F29033C2F2010341F29D31C0F2000185
:1052C000042212209C6415F091F9012391E648F222
:1052D0009033C2F2010342F2C5712846C0F20001C8
:1052E00004229C6015F082F9012382E648F2903393
:1052F000C2F2010342F62131C0F20001042207206C
:10530000DC6115F073F9012373E648F29033C2F2C1
:10531000010343F2E151C0F2000104223120C3F83D
:10532000C44015F063F9012363E648F29033C2F2FA
:10533000010342F21131C0F2000104222920C3F816
:10534000A44015F053F9012353E648F29033C2F21A
:10535000010342F6D151C0F2000104220B20DC62AD
:1053600015F044F9012344E648F29033C2F20103F8
:1053700042F26101C0F2000104222520C3F89440EA
:1053800015F034F9012334E648F29033C2F20103F8
:1053900041F605512846C0F200010422C3F88040BE
:1053A00015F024F9012324E648F29033C2F20103F8
:1053B00043F69101C0F2000104223520C3F8D44025
:1053C00015F014F9012314E648F29033C2F20103F8
:1053D00042F26D612846C0F2000104221C6015F003
:1053E00005F9012305E648F29033C2F2010341F2C8
:1053F00099112846C0F200010422DC6315F0F6F88A
:105400000123F6E548F29033C2F2010342F625513A
:105410002846C0F2000104229C6215F0E7F801233F
:10542000E7E548F29033C2F2010341F24D61C0F268
:105430000001042216209C6515F0D8F80123D8E558
:1054400048F29033C2F2010343F285212846C0F2AC
:1054500000010422C3F8E04015F0C8F80123C8E5B4
:1054600048F29033C2F2010342F67101C0F200012A
:1054700004220320DC6015F0B9F80123B9E500230C
:10548000B7E548F29033C2F2010343F23131C0F282
:10549000000104223920C3F8E44015F0A7F80123E5
:1054A000A7E548F29033C2F2010342F26521284693
:1054B000C0F200010422C3F8A04015F097F80123C0
:1054C00097E548F29033C2F2010341F6B151C0F2C0
:1054D000000104222120C3F8844015F087F801233D
:1054E00087E548F29033C2F2010341F6FD01C0F2B4
:1054F000000104221A209C6615F078F8012378E553
:1055000048F29033C2F2010343F235512846C0F20B
:1055100000010422C3F8C04015F068F8012368E5D3
:1055200048F29033C2F2010341F2ED012846C0F285
:10553000000104229C6315F059F8012359E548F253
:105540009033C2F2010342F675212846C0F20001F1
:1055500004229C6115F04AF801234AE548F2903391
:10556000C2F2010341F2A1512846C0F20001042217
:105570005C6515F03BF801233BE548F29033C2F23D
:10558000010341F601312846C0F2000104225C67A4
:1055900015F02CF801232CE548F29033C2F20103F8
:1055A00041F6B5712846C0F200010422C3F89040CC
:1055B00015F01CF801231CE548F29033C2F20103F8
:1055C00043F2E5712846C0F200010422C3F8D0403E
:1055D00015F00CF801230CE52DE9F04F044643F2D9
:1055E000341089B00F46C0F202000B2118F0E6F823
:1055F0004EF200203946C2F2000000230A2214F0C5
:105600006BFA43F24010C0F20200012118F0D6F804
:10561000B7B10026354643F240400121C0F20200F6
:1056200018F0CCF801354EF20020A15DEDB2C2F2C7
:10563000000000230A2214F04FFAAF422E46EAD8A7
:105640004DF670654EF20020C2F20005C2F2000075
:1056500014F030FA2B7CC3B3A67806F00F0601369F
:10566000B34232D043F26C001E21C0F2020018F0A7
:10567000A5F84EF2002000230A223146C2F20000B3
:1056800014F02AFA43F28C000E21C0F2020018F046
:1056900095F84EF2002000230A22297CC2F2000075
:1056A00014F01AFA43F29C000121C0F2020018F033
:1056B00085F84EF20020C2F2000014F0FBF943F22C
:1056C0004410C0F202001B2107E06378432B0FD087
:1056D00043F26010C0F202001B2118F06FF84EF286
:1056E0000020C2F2000009B0BDE8F04F14F0E2B9AA
:1056F00043F27C100C21C0F2020018F05FF8A17890
:105700004EF20020C1F30211C2F2000014F074F94D
:1057100043F240100121C0F2020018F04FF84EF29F
:105720000020C2F2000014F0C5F9072F05D043F2A3
:105730001C20C0F202002021CFE7E378C3F38403EA
:10574000002B00F0AA81022B40F01582A379F72BE1
:1057500040F0A68140F66453C2F201034AF6AB2042
:1057600021791B686279C3F6AA5005EE900A4DF2C2
:105770000A7001F07F01C3F6234006EE100A5818A4
:1057800002F07F022171627180F88C2193F8CE11B2
:1057900093F8CF7193F8D421019793F8D1710092C7
:1057A00093F8CB6193F8CD21029701F00407049799
:1057B0000592C3F88860009A93F8D00193F8D2510B
:1057C00093F8CCB193F8D3E1CDF80CE001F00206E8
:1057D00016F100090696049EC3F88CB002F0020C84
:1057E000624600F0020A18BF4FF0010916F1000CE2
:1057F00000F0040E18BF4FF0010C1AF1000B05F079
:10580000020818BF4FF0010B83F89F901EF10009AA
:1058100005F0040718BF4FF0010983F8A0C018F184
:10582000000C18BF4FF0010C01F0010100F0010065
:1058300083F8A3B017F1000B18BF4FF0010B83F8EA
:105840009E1083F8A20083F8A49012F1000918BFFB
:105850004FF0010983F8AB9093F8D59183F8A8B085
:10586000DDF814B007924FEA496907EE10BA07EE67
:10587000909A93F896909DF80420009E83F8A120BA
:10588000F8EEC76AF8EEE77A07EE109A67EEA57AA7
:1058900066EE866AB8EEC77A9DF8082083F8A520E0
:1058A000C9B29DF80C200091FDEEE77A079983F8C4
:1058B000A92026EE877A06F004020AF0FF0A83F890
:1058C000A7C083F89DB006F0010C12F1000B049EF6
:1058D000C3ED267ACDF810A0FCEEC77A01F0FF0ADE
:1058E000069983F8AAC04FF0000905F0010518BF1A
:1058F0004FF0010B83F8A65083F8ACB006F0FF061A
:10590000C0B20EF0FF0E08F0FF08EDB207F0FF077F
:105910005FFA8CFC02F0FF0217EE90BA83F89290C7
:1059200083F8919083F8909009B183F890B0009932
:1059300009B183F891B00EB183F892B0029907EEE5
:10594000901A4DF20A71C3F6234106EE901A93F8AD
:105950009410B8EEE77A07EE901A27EE267AF8EE62
:10596000E77A67EE277AFCEEE77ACDED007A9DF8CC
:105970000010B8F1000F06D093F89080884538BF2A
:10598000884683F8908035B193F891508D4238BFA6
:105990000D4683F8915037B193F89250A94238BF21
:1059A000294683F892100199049D07EE901A4DF252
:1059B0000A71C3F6234106EE901A93F89510B8EEDB
:1059C000E77A07EE901A27EE267AF8EEE77A67EE86
:1059D000277AFCEEE77ACDED007A9DF8001035B11C
:1059E00093F890508D4238BF0D4683F8905030B1F7
:1059F00093F89100884238BF084683F89100BEF1C1
:105A0000000F06D093F89200814238BF014683F818
:105A10009210039907EE901A4DF20A71C3F62341D2
:105A200006EE901A93F89310B8EEE77A07EE901A04
:105A300027EE267AF8EEE77A67EE277AFCEEE77A29
:105A4000CDED007A9DF80010BAF1000F06D093F862
:105A50009000884238BF084683F89000BCF1000FE0
:105A600006D093F89100884238BF084683F8910029
:105A700032B193F89200814238BF014683F8921008
:105A80003EB9BEF1000F04D11FB912B97F2283F8CD
:105A9000922025795C35EDB22AE0A379F72B05D069
:105AA00043F2C410C0F20200262116E6227963797F
:105AB00040F66455C2F2010502F07F0203F07F0355
:105AC0002868227163710AF095F8E27823792868D2
:105AD000617902F0030203EBC213034483F830112F
:105AE00009F07CFFE578237903EBC51505F0FF0588
:105AF00043F2EC10C0F20200052117F05FFEE378DC
:105B000013F07C0F06D143F2F410C0F20200092119
:105B100017F054FE43F200200B21C0F2020017F0F0
:105B20004DFE4EF2002000230A222179C2F200002D
:105B300013F0D2FF43F218200321C0F2020017F045
:105B40003DFE4EF20020617900230A22C2F20000DD
:105B500013F0C2FF43F20C200F21C0F2020017F035
:105B60002DFE4EF20020294600230A22C2F2000038
:105B700013F0B2FFB3E543F28C10C0F202003621FD
:105B8000ABE500BF38B504460D46FFF725FD43F2EF
:105B900040201021C0F2020017F010FE29462046D6
:105BA000002216F0D5FF42F60460C0F202000F2179
:105BB00017F004FE4EF20020C2F20000BDE83840AB
:105BC00013F078BF70B540F674750E460446C2F205
:105BD0000105FFF701FD43F254201021C0F202003D
:105BE00017F0ECFDA86C0368F021DB6C984746B118
:105BF0002644A86C14F8011B03681B689847A6424A
:105C0000F7D1A86C0368F721DB6C984742F67860FF
:105C1000C0F202000F2117F0D1FD4EF20020C2F2B7
:105C20000000BDE8704013F045BF00BFFFFFFFFF5D
:105C300038B543F2682010EE105A4DF670642DED21
:105C4000048BC2F200041421C0F20200B0EE608A9C
:105C5000C4ED030A84ED020A17F0B0FD28461BF0DC
:105C6000FDFC41EC100B4EF200200A21C2F20000B4
:105C700013F072FF43F280200121C0F2020017F0FE
:105C80009DFD40F6DB73C4F24903A06809EE103AAB
:105C90001BF0E4FC41EC100B4EF200200A21C2F292
:105CA000000013F059FF43F284200621C0F20200E5
:105CB00017F084FD43F280200121C0F2020017F0AA
:105CC0007DFDE0681BF0CAFC41EC100B4EF2002099
:105CD0000A21C2F2000013F03FFF43F28C200221A0
:105CE000C0F2020017F06AFDE36807EE903A27EE73
:105CF000890AF6EE008A20EE280A18F0EDFCA36867
:105D000007EE903A60EE277A17EE900A1BF0A6FC99
:105D10009FED511B41EC100B18F0DEFD4EF2002000
:105D20000321C2F2000013F017FF43F2902001217B
:105D3000C0F2020017F042FDE36807EE903A27EE4A
:105D4000890A20EE280A18F077FCA36807EE903A3B
:105D500060EE277A17EE900A1BF080FC9FED3E1B49
:105D600041EC100B18F0B8FD4EF200200321C2F2F6
:105D7000000013F0F1FE4EF20020C2F2000013F01A
:105D800099FE40F6645328EE098AC2F2010328EE18
:105D9000288A1B68B0EE480AC3F82C5118F09CFC06
:105DA0004FF47E43C4F2FF6307EE903AB4EEE70A85
:105DB000F1EE10FA0EDC4FF47E43CCF2FF6307EEF7
:105DC000903AB4EEE70AF1EE10FA30D50023C8F2AB
:105DD000010302E00023C7F6FF7340F60852C2F247
:105DE0000102B0EE480A936118F026FC4FF47E439E
:105DF000C4F2FF6307EE903AB4EEE70AF1EE10FA50
:105E000023DC4FF47E43CCF2FF6307EE903AB4EE0E
:105E1000E70AF1EE10FA11D50023C8F20103BDEC38
:105E2000048B40F63842C2F20102936138BDF0EEB5
:105E3000407AFEEEC87A17EE903ACEE7F0EE407A5E
:105E4000FEEEC87A17EE903AE9E70023C7F6FF7333
:105E5000E5E700BFAFF300800000002085EBB13F15
:105E60002DE9F041054643F2942082B00C46C0F281
:105E70000200032117F0A2FC4EF2002000230A22A8
:105E80002946C2F2000013F027FE43F298200121B8
:105E9000C0F2020017F092FC4EF2002021460023CF
:105EA0000A22C2F2000013F017FE4EF20020C2F2E6
:105EB000000013F0FFFD672D00F093824DD9782D7F
:105EC00000F0A08000F28980692D00F0C180C0F050
:105ED000DE836A2D00F0A0836B2D40F0FC8100234F
:105EE00001EE903A04EB44040023C4F2482304EB8F
:105EF000041401EE103AC4F3C71307EE903A40F6CB
:105F00007072C2F20102B8EE670AF0EE610AB7EEF3
:105F1000002A137004F0DAF84FF47E43C4F2FF63F2
:105F200007EE903AB4EEE70AF1EE10FA00F3D883E8
:105F30004FF47E43CCF2FF6307EE903AB4EEE70AEB
:105F4000F1EE10FA40F126840023C8F2010340F676
:105F50009042C2F20102D36167E2042D00F06A822E
:105F600040F2C5800A2D61D040F2C481202D00F09E
:105F7000DE81402D40F0AF8140F66456C2F201064A
:105F80003F2C94BF00210121306809F033FD3068B7
:105F900009F038FD0546002840F09D8130683746FD
:105FA00009F092FEEBB203EB430498424FEA8404FB
:105FB00040F29181306803190135DA78002AEFD078
:105FC00093F80280B8F1000FEAD198680BF08CF9D1
:105FD0003868044484F80380E2E77B2D1CD040F24B
:105FE0007D817E2D00F09D817F2D40F0748140F6F3
:105FF0006453C2F201030021186802B0BDE8F04109
:1060000009F0F0BC40F66453C2F20103186802B014
:10601000BDE8F04109F0FABC40F66453C2F2010356
:10602000186802B0BDE8F04109F0E4BD4DF67063B8
:10603000C2F2000300EE904A9A68FBEEEC0A00EE12
:10604000102AC3ED030A02B0BDE8F041FFF7F0BD2E
:10605000002301EE903A0023C4F2964302EE103A78
:1060600004EB44040023C4F2482304EB041401EEBF
:10607000103AC4F3C71307EE903A40F24012C2F24E
:106080000102B8EE670AF0EE610A137004F01EF820
:10609000B5EEC00AF1EE10FA00F1268347F6790357
:1060A000C4F2302307EE103AF6EE007AE0EE077AFB
:1060B0004FF4FC53C0F20103FCEEE77A17EE902A8E
:1060C0009A4240F276831A464FF4107040F2F4235D
:1060D000C2F20103197ECC0700F10983DC8B1A623E
:1060E000A04241F0010188BFD88319769DE1012DBE
:1060F00000F02B81C0F02181022D40F0EC8040F6B1
:106100006453C2F201034DF20A721B68C3F62342C4
:1061100006EE102A93F89D2093F89F0083F8944090
:1061200007EE902A93F89620B8EEE77A06EE902ACA
:1061300067EE067AF8EEE66A002167EEA67A83F843
:106140009210FCEEE77A83F89110CDED017A9DF87C
:10615000042083F8901008B183F8902093F89E10E3
:1061600009B183F8912093F8A01009B183F8922027
:1061700093F8A52093F8A70007EE902A4DF20A7233
:10618000B8EEE77A07EE904AC3F6234206EE102AED
:10619000F8EEE76A67EE067A67EEA67AFCEEE77A33
:1061A000CDED017A9DF8042030B193F89000904233
:1061B00038BF104683F8900093F8A60030B193F8EA
:1061C0009100904238BF104683F8910093F8A840A0
:1061D00034B193F89200824238BF024683F892208D
:1061E00093F8A12093F8A30007EE902A4DF20A72CB
:1061F000C3F6234206EE102A93F89520B8EEE77A0C
:1062000006EE902A67EE067AF8EEE66A67EEA67A60
:10621000FCEEE77ACDED017A9DF8042030B193F8D9
:106220009000904238BF104683F8900093F8A20087
:1062300030B193F89100904238BF104683F8910036
:1062400093F8A40030B193F89250AA4238BF2A467E
:1062500083F8922093F8A92093F8AB5007EE902A88
:106260004DF20A72C3F6234206EE102A93F89320E9
:10627000B8EEE77A06EE902A67EE067AF8EEE66A5E
:1062800067EEA67AFCEEE77ACDED017A9DF8042060
:1062900035B193F89050954238BF154683F8905029
:1062A00093F8AA5035B193F89150954238BF1546EE
:1062B00083F8915093F8AC5035B193F89260B242A4
:1062C00038BF324683F8922029B920B91CB915B9D4
:1062D0007F2283F8922002B0BDE8F081792DFAD1B7
:1062E00040F66453C2F20103186802B0BDE8F04101
:1062F00009F0A0BB072DEED107EE904A0023C4F2AF
:10630000FE23B8EE677A07EE903A87EE270A4DF63D
:106310007063C2F20003DA6800EE902A83ED020A8D
:1063200091E640F66453C2F20103012164E64DF6A2
:106330007063C2F200031C71CDE7632CCBD84DF61D
:106340007063C2F200031C716FE040F66453C2F246
:1063500001034DF20A721B68C3F6234206EE102AAF
:1063600093F89D2093F89F0083F8964007EE902ABB
:10637000B8EEE77A07EE904AF8EEE76A67EE067A3B
:10638000002167EEA67A83F89210FCEEE77A83F894
:106390009110CDED017A9DF8042083F8901008B19A
:1063A00083F8902093F89E1009B183F8912093F818
:1063B000A01009B183F8922093F8A52093F8A700C4
:1063C00007EE902A4DF20A72C3F6234206EE102A17
:1063D00093F8942006EE902AB8EEE77AF8EEE66A93
:1063E000D8E624B204EB840303EB830304EB8304B9
:1063F000C4F3C71407EE904A0023C4F2C823F8EE92
:10640000676A07EE903A86EEA77A40F66452C2F2C7
:10641000010240F6ED531268C2F201031C70F7EE60
:10642000007A77EEC77AC2ED4A7A02B0BDE8F04151
:1064300006F0ECB940F66453C2F201034DF20A7261
:106440001B68C3F6234206EE102A93F89D2093F8AA
:106450009F0083F8954007EE902A93F89620B8EEB7
:10646000E77A06EE902A67EE067AF8EEE66A0021F1
:1064700067EEA67A83F89210FCEEE77A83F8911023
:10648000CDED017A9DF8042083F8901008B183F8CF
:10649000902093F89E1009B183F8912093F8A010F2
:1064A00009B183F8922093F8A52093F8A70007EE8E
:1064B000902A4DF20A72C3F6234206EE102A93F890
:1064C0009420B8EEE77A06EE902A67EE067AF8EEA8
:1064D000E66A67EEA67AFCEEE77ACDED017A9DF8E2
:1064E000042030B193F89000904238BF104683F8F2
:1064F000900093F8A60030B193F89100904238BF15
:10650000104683F8910093F8A85035B193F89200A3
:10651000824238BF024683F8922093F8A12093F874
:10652000A30007EE902A4DF20A72C3F6234206EE4C
:10653000102AB8EEE77A07EE904AF8EEE76A67EEBF
:10654000067A67EEA67AFCEEE77ACDED017A9DF841
:10655000042030B193F89000904238BF104683F881
:10656000900093F8A20030B193F89100904238BFA8
:10657000104683F8910093F8A40030B193F892404C
:10658000A24238BF224683F8922093F8A92093F8BC
:10659000AB4007EE902A4DF20A72C3F6234206EE94
:1065A000102A93F89320B8EEE77A06EE902A67EE69
:1065B000067AF8EEE66A67EEA67AFCEEE77ACDEDAB
:1065C000017A9DF8042034B193F89040944238BF8A
:1065D000144683F8904093F8AA4034B193F8914060
:1065E000944238BF144683F8914093F8AC4034B1DC
:1065F00093F89260B24238BF324683F89220002965
:106600007FF469AE00287FF466AE002D7FF463AEA0
:10661000002C3FF45DAE5EE604EBC4040022C4F33C
:10662000471401EE902A07EE904A40F6EC53002200
:10663000C2F20103C4F20C22B8EE670A01EE102A7E
:10664000F0EE610AB7EE002A1C7003F03FFD4FF434
:106650007E43C4F2FF6307EE903AB4EEE70AF1EE30
:1066600010FA39DC4FF47E43CCF2FF6307EE903A28
:10667000B4EEE70AF1EE10FA40F194800023C8F27C
:10668000010340F65842C2F20102D361CDE624B2C2
:1066900004EB840303EB830304EB8304C4F3C71408
:1066A00007EE904A0023C4F2C823F8EE676A07EEAB
:1066B000903A86EEA77A40F66452C2F201024FF693
:1066C00010431268C2F200031C70F7EE007A77EEF6
:1066D000C77AC2ED497AA8E60023C7F6FF73D0E770
:1066E0000023C7F6FF7332E401200022EEE41C6AA7
:1066F000A24205D9D98B1A62884288BFD88394E612
:1067000002F17F00C009013000281A62024638BF3A
:106710000022880706D5586A7F30C00901308242BE
:1067200038BF02464F0706D5986A7F30C00901304E
:10673000824238BF02460E0706D5D86A7F30C009AC
:106740000130824238BF0246CD0606D5186B7F3035
:10675000C0090130824238BF02468C0606D5586B0C
:106760007F30C0090130824238BF0246480606D554
:10677000986B7F30C0090130824238BF0246C90998
:1067800006D0D96B7F31C90901318A4238BF0A4628
:10679000DA834AE6F0EE407AFEEEC87A17EE903AD7
:1067A000FFF7D5BBF0EE407AFEEEC87A17EE903ACE
:1067B00067E702F17F00C009013087E4F8B54DF6C4
:1067C0007065C2F2000504462B7C0E4617467BB36B
:1067D00098422DD043F26C001E21C0F2020016F048
:1067E000EDFF4EF2002000230A222146C2F20000F3
:1067F00013F072F943F28C000E21C0F2020016F081
:10680000DDFF4EF20020297C00230A22C2F20000A4
:1068100013F062F943F29C000121C0F2020016F06D
:10682000CDFF4EF20020C2F2000013F043F903E066
:1068300039463046FFF714FB43F29C200D21C0F28D
:106840000200013C16F0BAFFE1B20F2915D840F65C
:106850007475C2F2010541F0B001A86C03681B68B1
:106860009847A86C036806F07F011B689847A86CDE
:10687000036807F07F011B68984742F67860C0F212
:1068800002000F2116F09AFF4EF20020C2F2000023
:10689000BDE8F84013F00EB9F8B54DF67067C2F2D6
:1068A000000705463B7C0E4614467BB398422DD02C
:1068B00043F26C001E21C0F2020016F07FFF4EF280
:1068C000002000230A222946C2F2000013F004F936
:1068D00043F28C000E21C0F2020016F06FFF4EF260
:1068E0000020397C00230A22C2F2000013F0F4F8E1
:1068F00043F29C000121C0F2020016F05FFF4EF24D
:106900000020C2F2000013F0D5F803E02146304623
:10691000FFF7A6FA43F2AC200D21C0F2020016F0F8
:106920004DFF230603F0FE43681E43F43043360454
:1069300006F4FE0643F00B030002334300F47060DC
:10694000184316F0B1F842F60460C0F202000F21BD
:1069500016F034FF4EF20020C2F20000BDE8F8400D
:1069600013F0A8B848F21C53C2F2010382B01B68AE
:10697000019340F66C72C2F2010240F2A013C2F21F
:1069800001030199116001221A7002B0704700BF23
:1069900042F6AC532DE9F04FC0F202031C460FCC77
:1069A000B1B020AD0FC50FCC0FC50FCC0FC594E80B
:1069B0000F0010944DF6706740F2A014C2F2000769
:1069C000C2F201044FF0000E84F800E01F9585E844
:1069D0000F00BD7A0395FD7A3B7904953D7B0595C3
:1069E0007D7B06956FEA0309BD7B079509F00F09CA
:1069F00030AD05EB8909BA7997F80580787A02906D
:106A00001D1159F8403C11951146FA79139183F004
:106A100070431446DB433A7A019283EA05020DF192
:106A2000C00E02F00F020EEB82024FEA281E52F84F
:106A3000402C82EA1313DB4383EA0802754602F016
:106A40000F020DF1C00E0EEB82020DF1C00E52F8D6
:106A5000402C129582EA131383EA050202F00F021A
:106A60000EEB82020DF1C00E52F8402C82EA131395
:106A7000DB4383EA010202F00F020EEB82020811EF
:106A800052F8402C0199064682EA131383EA060263
:106A90000DF1C00E02F00F020EEB820208111496E7
:106AA0000990029852F8402C159482EA1313DB43A4
:106AB00083EA04020DF1C00E02F00F020EEB820217
:106AC000251152F8402C039C169582EA131383EA91
:106AD00005020DF1C00E02F00F020EEB82020DF165
:106AE000C00E52F8402C82EA13136FEA030C8CEAB2
:106AF000010202F00F0205990EEB82020B1152F80F
:106B0000402C0C93099B82EA1C1C8CEA03020DF1B9
:106B1000C00E02F00F020EEB8202069B52F8402CD0
:106B20001B110D9382EA1C13DB4383EA000206115A
:106B300002F00F0207980A960DF1C00E0EEB820EBE
:106B400002110E925EF8402C82EA13130A9A5A4000
:106B500002F00F020DF1C00E0EEB820E109AA2F1A0
:106B6000300C5EF8402C82EA1313DB4383EA040204
:106B70000DF1C00E02F00F020EEB820226110B96F1
:106B800052F8402C0B9C049E82EA131383EA040201
:106B90000DF1C00A02F00F020AEB8202351152F821
:106BA000402C179582EA1313DB4383EA060202F0B6
:106BB0000F020AEB82020DF1C00A52F8402C0C9E23
:106BC00082EA131383EA050202F00F020AEB820243
:106BD0000DF1C00A52F8402C82EA1313DB4383EA1A
:106BE000010202F00F020AEB82020DF1C00A52F814
:106BF000402C82EA131383EA060202F00F020AEB2A
:106C000082020DF1C00A52F8402C069E0E9D97F8A4
:106C100013B082EA1313DB4383EA060202F00F0289
:106C20000AEB82020D9E52F8402C82EA131383EA8B
:106C300006020DF1C00A02F00F020AEB82020DF10A
:106C4000C00A52F8402C82EA1313DB4383EA0002A5
:106C500002F00F020AEB82020DF1C00A52F8402C3A
:106C600082EA131383EA050202F00F020AEB8202A2
:106C700097F80FA052F8402C564697F810A0189697
:106C8000514697F811A01A9182EA13135046DB433C
:106C900097F812A083EA0602554602F00F020DF1A2
:106CA000C00A0AEB8202361152F8402C199682EA89
:106CB000131383EA06020DF1C00A02F00F020AEB79
:106CC00082020DF1C00A52F8402C1D9582EA13137E
:106CD000DB4383EA010202F00F020AEB82020E118B
:106CE00052F8402C0F9682EA13130F9A5A400DF176
:106CF000C00A02F00F020AEB8202064652F8402C4C
:106D00001B9682EA1313DB4383EA06020DF1C00AE5
:106D100002F00F020AEB8202011152F8402C1C9182
:106D200082EA131383EA01024FEA2B1ACDF820A05E
:106D300002F00F020DF1C00A0AEB82020DF1C00A47
:106D400052F8402C82EA1313DB4383EA050202F077
:106D50000F020AEB8202281152F8402C1E9082EAA0
:106D6000131383EA00020DF1C00A02F00F020AEBCE
:106D7000820230AE52F8402C82EA1313DB438BEAD6
:106D8000030202F00F020AEB82020DF1800E52F8AC
:106D9000402C82EA131A089B55468AEA030ABCE88B
:106DA0000F000AF00F0A06EB8A0A3C465AF840AC7C
:106DB000AEE80F00BCE80F00AEE80F00BCE80F0023
:106DC000AEE80F0059F8402C8AEA151A82F070429A
:106DD000119DD24382EA050303F00F0306EB830300
:106DE0000DF1C00E53F8403C83EA1212D24382EAFE
:106DF000080303F00F0306EB83036FEA0A0A53F854
:106E0000403CC7F800A083EA1212129B534003F0E3
:106E10000F030EEB83030DF1C00E53F8403C1398A3
:106E2000019983EA1212D24382EA000303F00F03AE
:106E30000EEB8303149853F8403C83EA121282EA63
:106E400000030DF1C00E03F00F030EEB8303159842
:106E500053F8403C83EA1212D24382EA00030DF158
:106E6000C00E03F00F030EEB8303169853F8403C5B
:106E700083EA121282EA00030DF1C00E03F00F0341
:106E80000EEB83030DF1C00E53F8403C099883EAE2
:106E90001212D24382EA010303F00F030EEB8303C5
:106EA0000DF1C00E53F8403C059983EA121282EAB4
:106EB000000303F00F030EEB8303029853F8403CEA
:106EC00083EA1212D24382EA00030DF1C00E03F0EE
:106ED0000F030EEB83030A9853F8403C83EA121227
:106EE00082EA00030DF1C00E03F00F030EEB8303E3
:106EF0000DF1C00E53F8403C0B9883EA1212039B2D
:106F0000D243534003F00F030EEB83030DF1C00E89
:106F100053F8403C83EA121282EA000303F00F03A5
:106F20000EEB83030DF1C00E53F8403C179883EA33
:106F30001212049BD243534003F00F030EEB830362
:106F40000DF1C00E53F8403C83EA121282EA0003AE
:106F500003F00F030EEB83030DF1C00E53F8403C1A
:106F60000C9883EA1212D24382EA010303F00F0362
:106F70000EEB83030DF1C00E53F8403C83EA12126E
:106F800082EA000303F00F030EEB83030DF1C00E42
:106F900053F8403C0D9883EA1212069BD2435340AB
:106FA00003F00F030EEB83030DF1C00E53F8403CCA
:106FB00083EA121282EA000303F00F030EEB83034D
:106FC0000DF1C00E53F8403C07981A9983EA12124B
:106FD000D24382EA000303F00F030EEB83030E9803
:106FE00053F8403C83EA121282EA00030DF1C00E0E
:106FF00003F00F030EEB83030DF1C00E53F8403C7A
:10700000199883EA1212189BD243534003F00F03DE
:107010000EEB83030DF1C00E53F8403C83EA1212CD
:1070200082EA000303F00F030EEB83030DF1C00EA1
:1070300053F8403C1E9883EA1212D24382EA0103BD
:1070400003F00F030EEB83030F9953F8403C83EAE0
:10705000121282EA01030DF1C00E03F00F030EEBD2
:1070600083030DF1C00E53F8403C1C9983EA1212C1
:107070001B9BD243534003F00F030EEB830307F136
:10708000140553F8403C83EA121282EA010303F02C
:107090000F030EEB8303FE4353F8403C83EA1212C6
:1070A0001D9BD243534003F00F030EEB830353F8B1
:1070B000403C83EA121282EA000303F00F030EEB56
:1070C000830353F8403C83EA1212D2438BEA020353
:1070D00003F00F030EEB830353F8403C83EA1212D4
:1070E000089B534003F00F030EEB830353F8403C1F
:1070F00083EA1213DB433B7014F8018BA71938465F
:1071000012F028FF80454146384601D012F07EFF3C
:10711000AC42F1D143F2BC202721C0F2020016F0AC
:107120004DFB4EF20020C2F2000031B0BDE8F04F3E
:1071300012F0C0BCF0B597B001AD2C4606AE601B96
:1071400012F008FF04F8010BB442F8D142F6AC5536
:10715000C0F202050FCD0FC40FCD0FC40FCD0FC469
:1071600095E80F0084E80F009DF808609DF809502D
:107170009DF80A409DF80B209DF80C309DF80D00FD
:107180009DF80E10F7430DF1580E07F00F070EEBA8
:10719000870757F8407C87F07047FF4387EA161649
:1071A00006F00F060EEB860656F8406C86EA1716B8
:1071B000F64385EA060707F00F070EEB870757F837
:1071C000407C87EA161787EA151606F00F060EEBC5
:1071D00086069DF80F5056F8406C86EA1716F6435F
:1071E00084EA060707F00F070EEB870757F8407C85
:1071F00087EA161787EA141606F00F060EEB8606C6
:107200009DF8104056F8406C86EA1716F64382EA5D
:10721000060707F00F070EEB870757F8407C87EA51
:10722000161787EA121606F00F060EEB86069DF873
:10723000112056F8406C86EA1716F64383EA0607D3
:1072400007F00F070EEB870757F8407C87EA161701
:1072500087EA131606F00F060EEB86069DF812302D
:1072600056F8406C86EA1716F64380EA060707F0E0
:107270000F070EEB870757F8407C87EA161787EA57
:10728000101606F00F060EEB860643F2E42056F8C1
:10729000406C86EA1716F64381EA060707F00F07E7
:1072A0000EEB8707C0F2020057F8407C87EA1617FA
:1072B00087EA111606F00F060EEB8606132156F824
:1072C000406C86EA1716F64385EA060707F00F07B3
:1072D0000EEB870757F8407C87EA161686EA1515E5
:1072E00005F00F050EEB850555F8405C85EA16158F
:1072F000ED4384EA050606F00F060EEB860656F807
:10730000406C86EA151585EA141404F00F040EEBA0
:10731000840454F8404C84EA1514E44382EA0405DA
:1073200005F00F050EEB850555F8405C85EA141451
:1073300084EA121202F00F020EEB820252F8402C85
:1073400082EA1412D24383EA020404F00F040EEB23
:10735000840454F8406C86EA121787EA131303F08A
:107360000F030EEB830353F8406C9DF813309DF828
:1073700014509DF815409DF8162086EA1716F6431E
:1073800083EA060707F00F070EEB870757F8407CE4
:1073900087EA161787EA131606F00F060EEB860625
:1073A0009DF8173056F8406C86EA1716F64385EAC2
:1073B000060707F00F070EEB870757F8407C87EAB0
:1073C000161686EA151505F00F050EEB850555F81E
:1073D000405C85EA1615ED4384EA050606F00F06C3
:1073E0000EEB860656F8406C86EA151585EA1414ED
:1073F00004F00F040EEB840454F8404C84EA151496
:10740000E44382EA040505F00F050EEB850555F807
:10741000405C85EA141484EA121202F00F020EEBAB
:10742000820252F8402C82EA1412D24383EA020408
:1074300004F00F040EEB840454F8404C84EA121458
:1074400084EA131303F00F030EEB830353F8403C5D
:1074500083EA141416F0B2F9019D4EF200200023C5
:1074600010222946C2F2000012F036FB43F2F82047
:107470000521C0F2020016F0A1F9E4434EF200200B
:107480002146C2F200000023102212F025FBA54283
:107490001DD14DF67065C2F2000505F114062C46AB
:1074A000601B12F057FD04F8010BB442F8D143F20F
:1074B0002430C0F202000F2116F080F94EF20020B5
:1074C000C2F2000017B0BDE8F04012F0F3BA43F288
:1074D00000302321C0F2020016F070F9FFF758FACD
:1074E000ECE700BF2DE9F84348F2F649C2F2010982
:1074F00043F234302DED028B0521C0F2020016F06C
:107500005DF9B9F8003007EE103A49F69A13C4F263
:10751000D92308EE903AB8EEC77A49F69A13C4F226
:10752000593308EE103A37EE287A4EF20024C7EEAF
:10753000087AC2F2000448F2F047C2F2010748F2AA
:10754000F448C2F2010848F29446C2F201064FF62E
:107550002045C2F2000517EE900A1AF07FF841ECC0
:10756000100B0221204612F0F7FA43F23C300D21B5
:10757000C0F2020016F022F93B8807EE903AF8EECE
:10758000E77A77EEA87A87EE887A17EE100A1AF073
:1075900065F841EC100B0221204612F0DDFA43F2AF
:1075A0004C300821C0F2020016F008F9B8F80010BB
:1075B000204612F021FA43F258300C21C0F20200AA
:1075C00016F0FCF83188204612F016FA43F26830C3
:1075D0001421C0F2020016F0F1F82988204612F0BA
:1075E0000BFA43F280300921C0F2020016F0E6F8EF
:1075F00040F60453C2F201030A2219682046002310
:1076000012F06AFA43F28C300D21C0F2020016F03B
:10761000D5F84FF61443C2F200030A221968204637
:10762000002312F059FA43F29C300921C0F2020003
:1076300016F0C4F840F69C53C2F201030A221968FE
:107640002046002312F048FA43F2A8300C21C0F281
:10765000020016F0B3F88021204612F0CDF943F273
:10766000B8301021C0F2020016F0A8F840F6C95355
:10767000C2F201030A2219782046002312F02CFAE4
:10768000204612F017FABDEC028BB9F80030B8F8BA
:1076900000203B80002332802B80BDE8F88300BFB0
:1076A00070B584B0002440F6645502940194CDF87E
:1076B0000B40C2F20105062643F2CC300221C0F293
:1076C000020016F07BF84EF200203146C2F20000B4
:1076D00012F092F943F22C500221C0F2020016F08F
:1076E0006DF84EF20020C2F2000012F0E3F943F20E
:1076F000D0305621C0F2020016F060F84EF20020A1
:10770000C2F2000012F0D6F92B6823444EF200209A
:1077100093F830110A220023C2F2000012F0DCF9C3
:1077200043F240400121C0F2020016F047F82B68F6
:1077300023444EF2002093F831110A220023C2F2B2
:10774000000012F0C9F943F240400121C0F20200EA
:1077500016F034F82B6823444EF2002093F83211CF
:107760000A220023C2F2000012F0B6F943F24040B0
:107770000121C0F2020016F021F82B6823444EF2DA
:10778000002093F833110A220023C2F2000012F005
:10779000A3F943F240400121C0F2020016F00EF8B6
:1077A0002B6823444EF2002093F834110A22002360
:1077B000C2F2000012F090F943F240400121C0F201
:1077C000020015F0FBFF2B6823444EF2002093F8D3
:1077D00035110A220023C2F2000012F07DF943F2B3
:1077E00040400121C0F2020015F0E8FF2B6823445D
:1077F0004EF2002093F836110A220023C2F2000054
:1078000012F06AF943F240400121C0F2020015F083
:10781000D5FF2B6823444EF2002093F837110A223B
:107820000023C2F2000012F057F943F22840082169
:10783000C0F2020015F0C2FF2B6823444EF2002074
:1078400093F838110A220023C2F2000012F044F922
:1078500043F234400D21C0F2020015F0AFFF2B6857
:1078600023444EF2002093F839110A220023C2F279
:10787000000012F031F943F234400D21C0F2020051
:1078800015F09CFF2B6823444EF200200A2293F847
:107890003A11C2F20000002312F01EF94EF200204D
:1078A000C2F2000012F006F943F244405C21C0F23B
:1078B000020015F083FF4EF20020C2F2000012F029
:1078C000F9F843F2A4400621C0F2020015F076FF59
:1078D0002B6823444EF2002093F83B110A22002328
:1078E000C2F2000012F0F8F843F238400921C0F269
:1078F000020015F063FF2B6823444EF2002093F83A
:107900003C110A220023C2F2000012F0E5F843F213
:1079100038400921C0F2020015F050FF2B682344C3
:107920004EF2002093F83D110A220023C2F200001B
:1079300012F0D2F843F228400821C0F2020015F0FC
:107940003DFF2B6823444EF2002093F83E110A229B
:107950000023C2F2000012F0BFF843F23C400521C0
:10796000C0F2020015F02AFF2B6823444EF20020DB
:1079700093F83F110A220023C2F2000012F0ACF883
:1079800043F2A4400621C0F2020015F017FF2B6855
:1079900023444EF2002093F840110A220023C2F241
:1079A000000012F099F843F2A4400621C0F2020050
:1079B00015F004FF2B6823444EF2002093F8411188
:1079C0000A220023C2F2000012F086F843F22C4093
:1079D0000421C0F2020015F0F1FE2B6823444EF2A0
:1079E000002093F842110A220023C2F2000012F094
:1079F00073F843F23C400521C0F2020015F0DEFEB0
:107A00002B6823444EF2002093F843110A220023EE
:107A1000C2F2000012F060F843F23C400521C0F2CF
:107A2000020015F0CBFE2B6823444EF2002093F8A1
:107A300044110A220023C2F2000012F04DF84EF267
:107A400000201534C2F2000012F034F87E2C06F14A
:107A5000FF367FF431AE43F2AC402D21C0F202007C
:107A600015F0ACFE4EF20020C2F2000012F022F837
:107A700043F24040C0F20200012115F09FFE2B6846
:107A800023444EF2002093F830110A220023C2F260
:107A9000000012F021F843F2A8400134C0F20200C5
:107AA000022140F6645615F089FE862CC2F20106CA
:107AB000E5D14EF20020C2F2000011F0FBFF43F2CC
:107AC000DC400521C0F2020015F078FE33684EF26A
:107AD000002093F8B6110A220023C2F2000011F030
:107AE000FBFF4EF20020C2F2000011F0E3FF43F270
:107AF000E4400421C0F2020015F060FE33684EF24B
:107B0000002093F8B7110A220023C2F2000011F0FE
:107B1000E3FF4EF20020C2F2000011F0CBFF43F26F
:107B2000EC400521C0F2020015F048FE33684EF229
:107B3000002093F8B8110A220023C2F2000011F0CD
:107B4000CBFF4EF20020C2F2000011F0B3FF43F26F
:107B5000F4400921C0F2020015F030FE33684EF205
:107B6000002093F8B9110A220023C2F2000011F09C
:107B7000B3FF4EF20020C2F2000011F09BFF43F26F
:107B800000500921C0F2020015F018FE33684EF2D1
:107B9000002093F8BA110A220023C2F2000011F06B
:107BA0009BFF4EF20020C2F2000011F083FF43F26F
:107BB0000C500921C0F2020015F000FE33684EF2AD
:107BC000002093F8BB110A220023C2F2000011F03A
:107BD00083FF4EF20020C2F2000011F06BFF43F26F
:107BE00018500921C0F2020015F0E8FD33684EF28A
:107BF000002093F8BC110A220023C2F2000011F009
:107C00006BFF4EF20020C2F2000011F053FF43F26E
:107C100024500A21C0F2020015F0D0FD33684EF264
:107C2000002093F8BD110A220023C2F2000011F0D7
:107C300053FF4EF20020C2F2000011F03BFF43F26E
:107C400030500D21C0F2020015F0B8FD33684EF23D
:107C5000002093F8BE110A220023C2F2000011F0A6
:107C60003BFF4EF20020C2F2000011F023FF43F26E
:107C700040500921C0F2020015F0A0FD33684EF219
:107C8000002093F8BF110A220023C2F2000011F075
:107C900023FF4EF20020C2F2000011F00BFF43F26E
:107CA0004C500921C0F2020015F088FD33684EF2F5
:107CB000002093F8C0110A220023C2F2000011F044
:107CC0000BFF4EF20020C2F2000011F0F3FE43F26F
:107CD00058500621C0F2020015F070FD31680A22EA
:107CE00001F2C11101A81AF059FD43F280200121CF
:107CF000C0F2020015F062FD01A81AF0E1FC014695
:107D000001A815F05BFD43F240100121C0F2020012
:107D100015F054FD4EF20020C2F2000011F0CAFE30
:107D20009B244EF2002000230A222146C2F20000CA
:107D300011F0D2FE43F22C500221C0F2020015F0E5
:107D40003DFD2B6823444EF2002093F830110A22A7
:107D50000023C2F2000011F0BFFE4EF200200134F9
:107D6000C2F2000011F0A6FEAD2CDAD14EF20020D6
:107D7000C2F2000011F09EFE04B070BD2DE9F0418A
:107D80002DED028B40F65C7086B0C2F2010011F05E
:107D9000E3F840F65C70C2F2010010F059FF40F6C3
:107DA0005C70C2F2010010F04BFF40F65C70C2F252
:107DB000010010F0E3FD40F65C70C2F2010010F02B
:107DC0004FFF40F65C70C2F2010010F051FF40F628
:107DD0005C70C2F2010010F02BFF43F26053C0F25E
:107DE000020393E8070000244FF020376B46029708
:107DF00003940494CDF80B708DF8144003C340F63F
:107E00005C701A8021462246C2F2010010F0ECFE9E
:107E100068461AF055FC024640F65C706946C2F2AC
:107E2000010011F0D3FD4EF2002023460A22214624
:107E3000C2F2000011F050FE43F290200121C0F286
:107E4000020015F0BBFC4EF2002023460A22214618
:107E5000C2F2000011F040FE43F26C500321C0F268
:107E6000020015F0ABFC68461AF02AFC0146684691
:107E700015F0A4FC43F240100121C0F2020015F0FD
:107E80009DFC43F270564EF20020C0F20206C2F290
:107E9000000011F00FFE96E80300009040F65C70C1
:107EA000019722468DF80410C2F201000B210297BF
:107EB00003940494CDF80B708DF8144010F094FEE8
:107EC00068461AF0FDFB024640F65C706946C2F255
:107ED000010011F07BFD4EF2002023460A222146CC
:107EE000C2F2000011F0F8FD43F290200121C0F22F
:107EF000020015F063FC4EF2002023460A220B21FB
:107F0000C2F2000011F0E8FD43F26C500321C0F210
:107F1000020015F053FC68461AF0D2FB0146684691
:107F200015F04CFC43F240100121C0F2020015F0A4
:107F300045FC4EF20020C2F2000011F0BBFD43F2FE
:107F40007853C0F202030FCB8DE80F0040F65C704F
:107F500021460122C2F2010004948DF8144010F071
:107F600043FE68461AF0ACFB024640F65C70694678
:107F7000C2F2010011F02AFD4EF2002023460A222F
:107F80000121C2F2000011F0A7FD43F2902001216F
:107F9000C0F2020015F012FC4EF200200A22234625
:107FA0002146C2F2000011F097FD43F26C5003210C
:107FB000C0F2020015F002FC68461AF081FB01468F
:107FC000684615F0FBFB43F240100121C0F20200AD
:107FD00015F0F4FB4EF20020C2F2000011F06AFD31
:107FE0000221042012F046FD02211E2012F042FD63
:107FF000DC2012F0A1FD43F28C503421C0F20200CB
:1080000015F0DCFB4EF20020C2F2000011F052FD30
:1080100043F2C4502E21C0F2020015F0CFFB4EF205
:108020000020C2F2000011F045FD43F2F450292176
:10803000C0F2020015F0C2FB4EF20020C2F20000B6
:1080400011F038FD43F220600921C0F2020015F062
:10805000B5FB0521304615F0B1FB4EF20020C2F20F
:10806000000011F027FD43F22C600D21C0F2020048
:1080700015F0A4FB4EF20020C2F2000011F01AFD30
:10808000FFF758F8FCF7E4F84EF28813CEF200033D
:10809000012740F2002040F26C15C2F201051F607A
:1080A0004FF4E171C1F6FF7010F068FF28460BF045
:1080B000FFF928460AF04CFDEA88242122F010023C
:1080C00028460AF011FBEA88242122F4807228460F
:1080D0000AF00AFB28460AF0BBFCF6EE000AB0EEF6
:1080E000600A28460AF0DEFF4CF6CD461D212846E0
:1080F0000AF01EFEC3F64C5628460BF031F801EE8E
:10810000106A4DF20A76C3F6234600EE906A46F2F4
:108110006666C3F666763B4600EE106A3A46394616
:1081200028460BF065F828460AF08EFB28460AF030
:108130000DFC0222072128460AF080FD28460AF09D
:1081400001FB4CF6CD43C3F64C63022200EE903A9D
:10815000B7EE000A394628460AF06EFE43F23C604C
:108160001B21C0F2020015F029FB4EF20020C2F2E2
:10817000000011F09FFC4DF6A060C2F200000B2140
:108180000CF0D6FB4DF6A060C2F200000D210CF001
:1081900037FC48F21010C2F20100FE210CF06EFD17
:1081A000002840F0A18043F258601721C0F202007D
:1081B00015F004FB4EF20020C2F2000011F07AFC30
:1081C00043F27063C0F2020393E8030040F6A0524A
:1081D00040F65073C2F20102C2F2010382E80300CA
:1081E00083E803004DF67066C2F2000640F6EC54D8
:1081F000C2F20104002301EE903A237800EE103A17
:108200000023C4F2964302EE103A0023C4F248233E
:1082100001EE103AB8EE400AF0EE610A01F056FFA6
:10822000B5EEC00AF1EE10FA00F1388347F6790393
:10823000C4F2302307EE103AF6EE007AE0EE077A49
:108240004FF4FC53C0F20103FCEEE77A17EE902ADC
:108250009A4240F226831A464FF4107140F2F423FA
:10826000C2F20103187EC50700F12481DD8B1A627A
:10827000A94240F0010088BFD9831876237800EE28
:10828000103A002301EE903A40F658440023C4F21D
:108290000C23C2F2010401EE103AB8EE400A4FF48A
:1082A0008033F0EE610AB7EE002AA36101F00EFF01
:1082B0004FF47E43C4F2FF6307EE903AB4EEE70A50
:1082C000F1EE10FA00F3BC804FF47E43CCF2FF6372
:1082D00007EE903AB4EEE70AF1EE10FA40F1D782D9
:1082E0000023C8F20103AEE043F278600E21C0F231
:1082F000020015F063FA4EF20020C2F2000011F005
:10830000D9FB4DF6706640F63053C2F20103C2F25B
:1083100000061F7008F04CFA327940F6C85EC2F2CF
:10832000010E02EB42034FF6244802EB8302C2F235
:10833000000840F6A0518EF80000C2F2010108EBDF
:10834000020008F0C3F8307908F0DEF843F28860E4
:108350000621C0F2020015F031FA337903EB430530
:1083600003EB850308EB030528461AF0A9F901463B
:10837000284615F023FA43F290203946C0F2020055
:1083800015F01CFA40F6A050C2F201001AF098F95C
:10839000014640F6A050C2F2010015F00FFA43F278
:1083A00040103946C0F2020015F008FA4EF20020E3
:1083B000C2F2000040F6F05511F07CFBC2F201055C
:1083C0002FE043F290600321C0F2020015F0F6F9AD
:1083D0004EF2002000230A222146C2F2000011F0D2
:1083E0007BFB43F280200121C0F2020015F0E6F988
:1083F00028461AF065F90146284615F0DFF943F2E0
:1084000040100121C0F2020015F0D8F94EF2002010
:108410000134C2F2000011F04DFB202C05F10B05D8
:1084200009D0092CCDD843F240400121C0F202000E
:1084300015F0C4F9C5E77179307908F04DFBD5E640
:108440000023C7F6FF7340F67075C2F201050022E3
:1084500001EE902A2A78E36100EE102A0022C4F28D
:10846000482201EE102AB8EE400AF0EE610AB7EE9B
:10847000002A01F02BFE4FF47E43F7EE007AC4F29F
:10848000FF6337EEC00A07EE903AB4EEE70AF1EE6A
:1084900010FA19DC4FF47E43CCF2FF6307EE903AFA
:1084A000B4EEE70AF1EE10FA40F1EA810023C8F2D7
:1084B00001030CE01D6AAA4240F29881D88B1A622F
:1084C000814288BFD983D9E60023C7F6FF732A7893
:1084D00000EE102A002201EE902A40F6904400227D
:1084E000C4F24822C2F2010401EE102AB8EE400A9A
:1084F000F0EE610AB7EE002AA36101F0E7FD4FF448
:108500007E43C4F2FF6307EE903AB4EEE70AF1EE61
:1085100010FA0FDC4FF47E43CCF2FF6307EE903A83
:10852000B4EEE70AF1EE10FA40F159810023C8F2E7
:10853000010302E00023C7F6FF732A78E36100EE2F
:10854000102A002201EE902A0022C4F2482201EEF5
:10855000102AB8EE400AF0EE610AB7EE002A01F0E8
:10856000B5FD4FF47E43C4F2FF6307EE903AB4EEDC
:10857000E70AF1EE10FA0FDC4FF47E43CCF2FF6312
:1085800007EE903AB4EEE70AF1EE10FA40F12081DE
:108590000023C8F2010302E00023C7F6FF7340F690
:1085A000ED514FF61042C2F20101C2F20002097809
:1085B0001278236207EE901A07EE102A0022C4F206
:1085C000C82208EE102AF8EE677AB8EE477AC7EEAE
:1085D000886A40F66453F268C2F201031B68C7EE72
:1085E000087AB7EE007A77EE666A77EE677A00EE81
:1085F000902AB268C3ED4A6A00EE102A83ED4B7AE6
:10860000C3ED497AFDF714FB0023C4F22C2307EED7
:10861000903A002306EE903AB36807EE103A27EE40
:10862000087A27EE277AC7EE087A77EEA67AFDEE6B
:10863000E77A17EE902A920072B640F6C843C2F26B
:108640000103DA6062B61A7C012A40F22F8172B609
:10865000DA6862B64FF61841002AC2F20001B8BFCC
:10866000033292100A60717972B640F6C8428900EE
:108670001962C2F2010262B693F82410012940F295
:108680003A8172B6126A62B64FF61843002AB8BF32
:108690000332C2F2000340F6CC509210C2F2010045
:1086A0005A6010F00BF940F6DC50C2F2010010F0F5
:1086B00005F948F2F64448F2F441C2F20104C2F26C
:1086C000010148F2F04248F29443C2F20102C2F2C0
:1086D000010343F2946025880C8815801821C0F2AC
:1086E00002001C8015F06AF84EF2002000230A22D6
:1086F0003179C2F2000011F0EFF943F2902001212C
:10870000C0F2020015F05AF84EF2002000230A22AF
:108710007179C2F2000011F0DFF943F2401001213B
:10872000C0F2020015F04AF84EF20020C2F200003A
:1087300011F0C0F9FEF7B4FF43F2B0601421C0F2AB
:10874000020015F03BF84EF200208021C2F200003A
:1087500011F052F943F2C8601121C0F2020015F085
:108760002DF84EF2002040F65A31C2F2000011F00E
:1087700043F943F2DC600321C0F2020015F01EF859
:108780004EF20020C2F2000011F094F9FEF7AAFEAA
:1087900040F65C70C2F2010010F06AFA01F0D6FEF9
:1087A0004EF20813CEF20003012243F2E0601A6099
:1087B0000B21C0F2020015F001F84EF20020C2F2C7
:1087C000000011F077F906B0BDEC028BBDE8F08136
:1087D000F0EE407AFEEEC87A17EE903ADFE6F0EE61
:1087E000407AFEEEC87A17EE903AA6E602F17F01D3
:1087F000C909013100291A620A4638BF00228707D9
:1088000006D5596A7F31C90901318A4238BF0A4603
:10881000450706D5996A7F31C90901318A4238BFB7
:108820000A46010706D5D96A7F31C90901318A4252
:1088300038BF0A46C70606D5196B7F31C909013111
:108840008A4238BF0A46850606D5596B7F31C90969
:1088500001318A4238BF0A46410606D5996B7F31FD
:10886000C90901318A4238BF0A46C10906D0D96B0D
:108870007F31C90901318A4238BF0A46DA83FDE4F3
:10888000F0EE407AFEEEC87A17EE903A1FE6F0EE70
:10889000407AFEEEC87A17EE903AD4E50121002224
:1088A000DCE402F17F01C9090131D7E472B61A682C
:1088B000586811780478587A1A7A044201EA020159
:1088C0003AD09A7A02F00302002940F0818042F007
:1088D00008029110082A997236D8072A62D2032A10
:1088E0004CD046D9042A37D0062A7FF4B1AEDA68D4
:1088F000023ADA60ADE672B6516990690D78047893
:10890000507F117F044201EA050129D1927F02F0D4
:10891000030200295FD19110082A997732D8072ADB
:1089200052D2032A48D041D9042A32D0062A41D152
:108930001A6A023A1A62A6E69A7A02F0030200293B
:10894000C7D042F00402C4E70C2A17D025D8092A60
:10895000CDD00B2A7FF47CAEDA68013ADA6078E693
:10896000927F02F0030209B142F0040242F00802D1
:10897000D1E7012A16D0022AEED069E6DA6802327F
:10898000DA6066E60C2A17D01AD8092AD0D00B2A4A
:1089900010D11A6A013A1A6275E60D2ADCD00E2A45
:1089A0007FF456AEDA680132DA6052E6012A0BD063
:1089B000022AEED01A6A66E61A6A02321A6262E681
:1089C0000D2AE6D00E2AF5D11A6A01321A625AE649
:1089D00042F004027BE742F004029CE72DE9F047F5
:1089E0009DF82040013CE4B20F2C03D84EB2002E7B
:1089F0000D4601DBBDE8F087E0290FD9F729F9D949
:108A00000835EDB2012303FA05F515F0DD0FF1D0BD
:108A1000806C0368BDE8F0471B6818478146806C8E
:108A20001F46036846EA0401C9B21B68904698478E
:108A3000D9F84800036808F07F011B6805F0EF05CE
:108A40009847C02DD6D0D9F84800036807F07F01B9
:108A50001B68BDE8F0471847F8B50446806C03680A
:108A60001B69984708B90020F8BDA06C03685B69D2
:108A70009847C3B203F0FB01F929F4D0A26D82B983
:108A800094F84D2084F84F30150600F19C8040B2D8
:108A90000028C0F25081002084F84D00A065606578
:108AA000F8BD010667D494F84F10F02904EB0201D9
:108AB00040D081F84F30616D4B1E9A4240D394F8FC
:108AC0004F20F02AE7D013063DD4002384F8663007
:108AD000B02B4CD0A02B4AD0D02B48D0E02B46D086
:108AE000C02B44D0002094F8505084F867500329DC
:108AF00008BF94F8515084F8650018BF0025002184
:108B00000120B02B84F86850A165616584F8E90004
:108B100000F0B58000F2AC80902B00F0B080A02B6C
:108B200000F0AD80802B00F0AA80002384F84D3047
:108B30000120F8BD81F86930636D013B9A42AAD2E9
:108B40000132A2658FE702F10C03DBB2012BBCD925
:108B500002F0FB03F92BB8D0EF2A00F2DB8002F021
:108B6000F003802B84F8663001D0902BB0D102F056
:108B70000F000130B7E7A3F1F701082993D80125C9
:108B800005FA01F010F4DD7F40F0968000298AD1CB
:108B900094F86930F02B7FF47EAF561C2244F72006
:108BA000370A82F8690084F8676084F8687084F88E
:108BB000651084F84D10284684F8663084F8E95032
:108BC000A1656165F8BD02F10C05EEB2012E7FF6DC
:108BD0005EAF02F0FB0EBEF1F90F3FF458AFEF2A83
:108BE0002DD802F0F007802F2AD140B20028FFF6DE
:108BF0004FAF012184F84F2084F85030A165EDB2C9
:108C0000012D7FF648AFBEF1F90F3FF444AFEF2AD4
:108C10005FD802F0F003B02B26D01ED9D02B04D0A1
:108C2000E02B21D0C02B7FF436AF022363650121F6
:108C3000A36D994227D90133A3650020F8BD1746DB
:108C400007F0DF06902ED0D007F0BF06A02ECCD0C4
:108C500007F0EF07C02FC8D019E7902B04D0A02B46
:108C600002D0802B7FF417AF032363650221DFE777
:108C7000D02B04D0E02B02D0C02B7FF456AF84F869
:108C80004D200120F8BDEF2A94BF02F0F0051546F3
:108C900002F00F020023013294F8501084F865208E
:108CA000012084F8671084F8683084F86650A36562
:108CB000636584F8E900F8BD002284F8672084F831
:108CC000682084F8652084F8663084F8E9502846E6
:108CD000F8BDF62A0FD007D8F12AA6D01CD9F22A5F
:108CE000C2D0F32AA1D0D6E6FC2A21D8FA2A02D291
:108CF000F82A7FF4D0AE0023012084F8653084F890
:108D0000673084F8683084F86620A365636584F86A
:108D1000E900F8BD1346D9E6F02A7FF4BCAE802105
:108D20000023616584F8692084F84D307F217FE756
:108D3000FE2AE0D2AFE61A468E4603F10C055EE746
:108D400090F86630F12B7CD00ED9FA2B2BD01FD89F
:108D5000F32B38D0C0F08180F62B7AD0F82B40F07E
:108D60008B80036BF3B11847B02B6ED031D9D02B69
:108D700021D03ED9E02B42D0F02B7ED1C3698BB1FC
:108D8000B0F86710802900F1690028BF80211847DA
:108D9000FC2B0CD051D3FE2B4BD0FF2B6BD1436C53
:108DA000002BE0D17047436B002BDCD1FAE7C36B9B
:108DB000002BD8D1F6E74369002BF3D090F8671069
:108DC00090F865001847836A002BEBD090F8670095
:108DD0001847902B29D0A02B23D0802BE2D10368F9
:108DE000002BDFD090F8682090F8671090F86500AD
:108DF0001847C02B42D10369002BDFD1D2E782692B
:108E0000002ACFD090F8681090F8673090F865008D
:108E1000C90101F47E5103F07F031943A1F500510C
:108E200010478368002BDDD1BCE74368002BD9D104
:108E3000B8E7036C002B96D1B4E7836B002B92D17B
:108E4000B0E7036A002BC1D1ACE7C368002BC9D1DE
:108E5000A8E7C36A002B86D1A4E7426A002AA1D002
:108E600090F8683090F86700DB0103F47E5300F05F
:108E70007F0018431047704770477047704700BF26
:108E800090F86430DA0725D513F0FE0F22D070B5C4
:108E900090F8665085F08002602A82B004461AD9A4
:108EA000F62D6ED067D8F12D7ED04FD9F22D2DD072
:108EB000F32D1AD1806C94F86760036829461B680B
:108EC0009847A06C0368DB6C06F07F0102B0BDE838
:108ED00070401847704790F865608E4207D031B1F6
:108EE0005B08012B08D0032B27D002B070BD5B08B4
:108EF000012B01D0022BF8D194F8683094F8672048
:108F0000009629462046FFF769FDEEE7806C94F84D
:108F10006730026894F868601268294643EAC6150B
:108F20009047A06C036805F07F019B6C9847A06C8C
:108F30000368C5F3C6119B6CC8E794F8683094F8D1
:108F4000672000962946FFF749FDCEE7F02DCCD1EA
:108F5000B0F86760802E28BF802600F16905002EDA
:108F6000C3D02E44A06C15F8011B03681B689847FA
:108F7000AE42F7D1B9E7FC2D26D8FA2D01D2F82D53
:108F8000B3D105F10803DBB2072BAED8012202FAF8
:108F900003F313F0DD0FA8D0A06C03681B6829460B
:108FA00002B0BDE870401847806C94F8672094F8D0
:108FB000683006681201294603F00F0302F07005BD
:108FC00032681D439047E7E7FE2D8ED3D9E700BFF7
:108FD000F0B540F2A41087B0C2F201000BF076FBAE
:108FE000002840F0F88048F21C54C2F2010440F618
:108FF0006C7223680193C2F20102019B116841F275
:1090000087325B1A934206D940F6C953C2F2010374
:109010001B78002B3AD040F67475C2F2010595F822
:109020004C60102E43D9002013F0E0FF40F62C5383
:1090300022680292C2F20103029A1868121A48F2D8
:109040001C51322AC2F201014ED840F66053226808
:109050000492C2F20103049A1968521A632A00F2B8
:10906000B58040F2842322680592C2F20103059A7A
:10907000196841F28730521A824205D901F59C5194
:1090800008311960FEF72EFA07B0F0BD40F2A013C8
:10909000C2F201031B78002BBDD040F67475C2F2FA
:1090A0000105FDF775FC95F84C60102EBBD82846DD
:1090B000FFF7D2FC0028B6D095F86630902B00F070
:1090C0000E8183F08003602B40F20C8140F67470B7
:1090D000C2F20100FFF734FE40F674703146C2F26E
:1090E0000100FFF7CDFE9EE740F664560A68039242
:1090F000C2F2010640F63455039A30681A60C2F293
:10910000010506F0E5FD40F6C953C2F20103AA8845
:109110001870002A40F0438140F23815C2F2010570
:10912000AB88002B40F0F08040F2C425C2F201056C
:10913000AB88002B89D03268D2F8241107EE901A40
:10914000296807EE101A77EE877A43F26470C2ED51
:10915000497A013B0F21C0F20200AB8014F02EFBD4
:109160003368D3F8240118F079FA41EC100B4EF271
:1091700000200521C2F2000010F0EEFC43F27470F2
:109180001521C0F2020014F019FB4EF20020A9884C
:10919000C2F2000010F030FC43F28C701521C0F2D6
:1091A000020014F00BFB286818F058FA41EC100B81
:1091B0004EF200200521C2F2000010F0CDFC4EF26C
:1091C0000020C2F2000010F075FC3EE76431196027
:1091D00003F01CFB45E740F27814C2F2010411F0E1
:1091E00085FC2368C01AB0F5356F7FF6FCAE11F030
:1091F0007DFC206040F2A410C2F201000BF076FA70
:10920000044611F073FC40F66453C2F201030546B4
:1092100022461868802106F049F811F067FC40F6F4
:109220005A33401B984252D84FF6204411F05EFC4E
:10923000C2F20004401B2388834260D372B640F21E
:109240007C13C2F201031A7F02F0FF010AB100226F
:109250001A7762B6A1B372B647F6FF744FF40040B6
:10926000B3F91E50B3F92020DC83188462B685EA76
:10927000E57182EAE273A3EBE273A1EBE5718B4245
:10928000B8BF0B4607EE903A4FF47E43C4F2FF633B
:1092900006EE103AF8EEE77A47F2A403C7EE866AC4
:1092A000C3F67D7307EE103AF4EEC76AF1EE10FADA
:1092B00006DD40F69C53C2F201031A6801321A60BF
:1092C00040F2A410C2F201000BF022FA8BE640F645
:1092D0000453C2F201031A6801321A60A4E795F838
:1092E000683043B195F865309E423FF4EFAE002EF2
:1092F0003FF4ECAEF0E6802385F86630F2E711F03B
:10930000F5FB401B208099E73268D2F8281107EE60
:10931000901A296807EE101A77EE877A43F21870D0
:10932000C2ED4A7A013B1221C0F20200AB8014F078
:1093300045FA3368D3F8280118F090F941EC100B86
:109340004EF200200521C2F2000010F005FC43F2AD
:109350002C701821C0F2020014F030FA4EF20020F6
:10936000A988C2F2000010F047FB43F248701821B0
:10937000C0F2020014F022FA286818F06FF941ECEC
:10938000100B4EF200200521C2F2000010F0E4FBA9
:109390004EF20020C2F2000010F08CFBC4E64DF645
:1093A0007067C2F20007013AFB68AA8000EE903AAB
:1093B000BB6807EE903A2B6807EE103A37EE870A43
:1093C000FCF736FC43F2EC600821C0F2020014F016
:1093D000F5F9B86818F042F941EC100B4EF2002094
:1093E0000521C2F2000010F0B7FB43F2F8600E2135
:1093F000C0F2020014F0E2F94EF20020A988C2F295
:10940000000010F0F9FA43F208700E21C0F20200D9
:1094100014F0D4F9286818F021F941EC100B4EF241
:1094200000200521C2F2000010F096FB4EF2002051
:10943000C2F2000010F03EFB6EE600BF2DE9F04FD7
:1094400040F67475C2F201058DB010F035FD95F847
:109450006430002401264EF2200743F001034FF64A
:10946000FF7E66F34703214685F8654085F8664030
:1094700085F8674085F8684085F8E940C2F2000742
:1094800005F169008022C5F85CE0C5F860E085F868
:109490006430AF6485F84C4085F84D4085F84E4007
:1094A0006C65AC6540F65C7718F0C2FF4DF668223B
:1094B00040F689112846C2F20002C0F20001C2F251
:1094C00001072C606C60AC60EC602C616C61AC617D
:1094D000EC612C626C62AC62EC622C636C63AC631A
:1094E000EC632C646C6418F055FC022310222721D5
:1094F00038460FF033FA40F6C84042F69C53C0F2AB
:10950000020302220321C2F201003B60FBF7F2FBDF
:1095100040F6DC401D221C21C2F20100FBF7EAFBF1
:1095200048F21C5340F6CC50C2F20103142204212D
:10953000C2F201001D4602930FF0A8F940F6DC507C
:1095400014221E21C2F201000FF0A0F92B6806932D
:1095500040F66053C2F2010340F2A419C2F20109BD
:10956000069A1A602146224640F27C1B4846FAF7CA
:1095700043FEC2F2010B44F25C13C0F202030BF192
:1095800018023146584689F89C40C9F8984089F835
:109590009D40C9F8003040F2F425FAF72DFE4FF453
:1095A0000041C2F2010547F6FF7244F20413ABF822
:1095B000201042F69051C0F20203ABF81E20C0F218
:1095C000020105F51462CBF800302C722346EC60E2
:1095D00020466E722A6129602C4600E0226942F81A
:1095E0002300697A013340F2F4229942C2F2010267
:1095F000F4DC48F29043C2F201030393196809B9FD
:10960000A8E219464B69002BFBD14D614FF00004D5
:10961000002140F6584844F22C1340F23430C2F294
:109620000108C0F2020369614FF41062AC80EC8063
:10963000AC722C76C2F201004FF000042B606C83F8
:10964000AC83EC8318F0F4FE08F1280204214046B4
:10965000FAF7D2FD4FF4803340F6384440F6904795
:10966000C2F20107C8F81830C8F81C30C8F820301A
:10967000C8F82430059340F60856234644F2441AAD
:10968000C2F20106C2F20103C0F2020A07F1280287
:10969000042138461C46C8F800A00493FAF7ACFD34
:1096A000059B019606F11C0230460121C7F800A077
:1096B000BB61FB613B627B62FAF79EFD019B44F25A
:1096C000381A9E462246059BCEF81830C0F2020A90
:1096D0001C320121204640F67C56CEF800A0FAF755
:1096E0008BFD059BA361C2F2010642F69053C0F2C6
:1096F000020306F118010022022033604FF000033C
:109700003372707231610B46C4F800A0F2601146EA
:10971000304600E0036943F82210747A013240F6C3
:109720007C539442C2F20103F4DC039A126848F2BB
:109730009041C2F201010AB90EE21A465369002BA8
:10974000FBD15661002440F67C5040F2482A44F296
:109750007453C0F20203C2F2010A7461B480F4804F
:10976000B472C2F20100336012F0C0F850468AE8C9
:10977000000A8AF808408AF80940CAF80C408AF8BA
:10978000104040F25C2B0FF057FD4DF6682240F67A
:109790008D11C2F2010BC2F20002C0F2000150466C
:1097A00018F0F8FA5846CBF80090CBF804808BF804
:1097B00008408BF80940CBF80C408BF8104040F281
:1097C000702A0FF039FD4DF6682240F68D11C2F275
:1097D000010AC2F20002C0F20001584618F0DAFA9B
:1097E0005046CAF800908AF808408AF80940CAF83A
:1097F0000C408AF81040CAF8047040F6F0490FF0A7
:109800001BFD4DF6682240F68D11C2F20109C2F22D
:109810000002C0F20001504618F0BCFA4FF0010BF4
:10982000484689E8200189F80840C9F80C4089F8C1
:10983000104089F809B040F2882A0FF0FDFC4DF67F
:10984000682240F68D11C2F2010AC2F20002C0F293
:109850000001484618F09EFA022350468AF8093063
:1098600005938AE8A0008AF80840CAF80C408AF8F4
:10987000104040F29C290FF0DFFC4DF6682240F6C4
:109880008D11C2F20109C2F20002C0F2000150467D
:1098900018F080FA4846C9F80080C9F8045089F8E1
:1098A000084089F80940C9F80C4089F8104040F296
:1098B000B0250FF0C1FC4DF6682240F68D11C2F2C2
:1098C0000105C2F20002C0F20001484618F062FA37
:1098D0002846C5F800802C72EC602C746F6085F807
:1098E00009B040F668580FF0A7FC4DF6682240F624
:1098F0008D11C2F20108C2F20002C0F20001284636
:1099000018F048FA019BC8F80430404688F808402F
:1099100088F80940C8F80C4088F81040C8F8007072
:1099200040F2CC250FF088FC4DF6682240F68D11F0
:10993000C2F20105C2F20002C0F20001404618F076
:1099400029FA049B6B6028462C726C72EC602C74B4
:109950002F6040F2E0280FF06FFC4DF6682240F6D1
:109960008D11C2F20108C2F20002C0F200012846C5
:1099700018F010FA4046C8F8046088F8084088F8E3
:109980000940C8F80C4088F81040C8F8007040F250
:1099900044150FF051FC4DF6682240F68D11C2F2CD
:1099A0000105C2F20002C0F20001404618F0F2F9CF
:1099B00028466E602C72EC602C7485F809B02F601C
:1099C00040F63C560FF038FC4DF6682240F68D11FB
:1099D000C2F20106C2F20002C0F20001284618F0ED
:1099E000D9F9059B737242F6905306F11801C0F243
:1099F0000203224633603472F460204631610B4624
:109A0000344600E0236943F82200717A013240F6BF
:109A10003C539142C2F20103F4DC039A126848F20B
:109A20009041C2F201010AB998E01A465369002B2D
:109A3000FBD15661002440F63C5044F25013C0F272
:109A400002037461B480F480B472C2F2010040F287
:109A50005817C2F2010733600AF0B8FC019B3C7250
:109A6000384687E848007C72FC603C740FF0E4FBE9
:109A70004DF6682240F68D11C0F200013846C2F260
:109A8000000240F6B45518F085F9C2F20105049AB7
:109A90002C720123284685E844006B72EC602C741C
:109AA0000FF0CAFB4DF6682240F68D11C0F200019E
:109AB0002846C2F2000218F06DF940F26C13C2F2AF
:109AC000010344F21012C0F202021A604FF40A704D
:109AD0000A221A7210F056FD4AF64441064605F075
:109AE0005FF9029F3B680793079D3B680893089CBA
:109AF0003B68099340F66450C2F2010040F66C7175
:109B000040F2442240F6B053C2F20101C2F2010217
:109B1000C2F20103066009980D601460186010F02D
:109B2000E5FF029F3B680A930A9D3B680B9340F256
:109B3000781140F62C5240F28423C2F20101C2F2A5
:109B40000102C2F201030B9C086015601C600DB09D
:109B5000BDE8F08F1A6059E50B60F3E50B6069E72B
:109B60004FF07E520021416702678267704700BF55
:109B700070B507EE901A2DED048BB8EEE79AB7EEAC
:109B8000008A88EE097A4FF46043C4F22B730025F3
:109B900000260446866305638561C561C5608560EE
:109BA0004560056007EE903A80ED057A87EE897A88
:109BB0000562456380ED049A17EE100A17F04EFD1A
:109BC00041EC100B15F024F851EC100B18F092F842
:109BD00049F6AB03C3F6B44308EE900A07EE903A99
:109BE00068EEA77A40F6DB7388EE277AC4F2490361
:109BF00006EE903A2369C4ED097A05EE903AB6EE86
:109C0000006ABAEE040AA5EE860A636907EE903A86
:109C100020EE260A84ED0A7A20EE270A14F0A6FD2B
:109C20004BF60B43C3F6324307EE103A0023C4F25F
:109C3000FC2307EE903A68EE878A87EE897A012343
:109C400023660023CBF6807384F854606566A566AE
:109C5000E364A364C8EE287A38EE478AC4ED168A16
:109C600084ED1B8ABDEC048B84ED0B0AC4ED177ADE
:109C700070BD00BFF8B50B6806EE903A436E07EE74
:109C8000903AC36E07EE103A836E76EEE77A06EEF0
:109C9000103AE7EE067A02F18047012A2DED108B8B
:109CA00007F1FF37C1ED007AC0ED196A19DD01EB4C
:109CB00087040B465D6807EE905A37EEE67A06EEAB
:109CC000905AC56E06EE105A1D6805EE905AA6EE23
:109CD000257A17EE105A43F8045FA342C0ED197AB3
:109CE000E8D1846FBF0007EE904ACB19B7EE007A37
:109CF000F4EE477A1B688366F1EE10FA11D0002A61
:109D00000FDD3C1D0C440B4602E0856F07EE905AB8
:109D10001D6807EE105A67EE277AE3EC017AA3423A
:109D2000F3D1036F07EE903AB7EE007AF4EE477A7C
:109D3000F1EE10FA00F0FB80C36C07EE103A436FAF
:109D4000F4EE477AF1EE10FA16460D46044600EEA0
:109D5000103A40F0EF80836C07EE903AB4EE670A59
:109D6000F1EE10FA40F0E680C36B0CEE903AF7EE9D
:109D700000BA3CEEABDA002E8CEE8DBA40F3D78001
:109D800040F6DB73C4F249030437A66B2F440AEE96
:109D9000103A2BEE0B8A46F26663C3F6E6630DEECD
:109DA000903A28EE0B8A4CF67743C3F22B2309EE48
:109DB000903A8BEE8D9AF2EE0E8A28EE0B8A10E026
:109DC000022E00F02981032E40F02281F0EE6B7A02
:109DD000ECEE2D7A67EEAA7AE5EC017AAF4200F05C
:109DE000A6802B6807EE903AE36905EE903AA369E6
:109DF00006EE103AE36A04EE103A23680AEE903A4F
:109E000063680EEE103AA3680FEE103AE3680EEEA8
:109E1000903A236A0CEE103A636907EE103A27EE87
:109E2000287A37EEE55A27EE0A7AF0EE4E3A25EE1A
:109E3000075A37EE2B7AEBEE2A3A636AC5EE076AC9
:109E4000B0EE4F7A75EEA65AABEE237AE5EEED7AD8
:109E500074EE2B4A77EEC67AB0EE6E5A67EE847ACD
:109E6000ABEE075A87EEA47A29EE455A36EE076A1A
:109E7000F0EE6B3AF0EE467AE5EE0C7AECEE083A4C
:109E800076EEA55AC7EEA36A37EE066A76EEA96AA1
:109E900007EE903A76EEEA6AC4ED075AEBEE26AA90
:109EA00084ED066AB0EE6A0AABEE260A20EE270AB7
:109EB00014F0E6FA7AEECE7AA36A67EEAC7A07EE91
:109EC000103A27EE000A87EE8D7A012E84ED000A03
:109ED00077EE0E7A37EECF6A37EE277A26EE2C6AC7
:109EE00084ED017AC6EE0D6A36EE8F7A77EE6E5A01
:109EF00076EE876A65EEAC5AC4ED026A85EE8D6A2D
:109F000076EE2E6A36EE266A84ED036A74D03FF749
:109F100057AF002E7CD1636B06EE103A66EE077ADF
:109F20003BEEC66AE6EE267AF0EE67AA4EE7BDEC97
:109F3000108BF8BD4BF61423B7EE008AC4F23F0332
:109F400009EE103A38EE400AF3EE038A20EE090AD1
:109F500014F0BEFE30EE480A4BF22D2380EE286A44
:109F6000C3F67D7307EE103A002307EE903AE6EE53
:109F7000077A236FF0EE0C6A77EE677A06EE103AF6
:109F800027EEA67A26EE090AC4ED107A84ED087A47
:109F900014F09EFE30EE480A4FF4784380EE286AB3
:109FA000C4F2936306EE903A0023C4F2702307EEE6
:109FB000903A40F6DB73C4F24903E6EE267A07EEE8
:109FC000103A636906EE903A27EEA60A20EE070AD9
:109FD00014F0CCFB216C226F636F84ED0F0A07EE47
:109FE000901A38EE678AF0EE40CABDEEC88AE26485
:109FF000A36484ED188ABAE6636B06EE903A66EEC7
:10A00000A77A7BEEE66AE6EE877AF0EE67AADDE6EF
:10A0100000230AEE903AD9E6636B06EE903A6AEEB8
:10A02000A6AA7BEEE66AE6EEA7AACFE610B403681E
:10A0300041681A780C78417A037A0C4202EA0302EA
:10A040001AD0837A03F003030AB143F0040343F008
:10A0500008039A10082B82722AD8072B22D2032BCE
:10A060002ED011D9042B13D0062B14D1C3685DF860
:10A07000044B023BC3607047837A03F00303002A5A
:10A08000E7D043F00403E4E7012B0BD0022B02D10D
:10A09000C368013BC3605DF8044B70470D2BF7D0DC
:10A0A0000E2BF8D1C3685DF8044B0133C3607047D1
:10A0B0000C2B05D0F2D8092BD8D00B2BE8D0EAE72F
:10A0C000C3685DF8044B0233C360704730EE600A2A
:10A0D00032EE612A31EE601A20EE022A82EE010A87
:10A0E00030EE210A704700BF00B583B00FF0E4FEE8
:10A0F00048F21C52C2F2010241F26003126801925E
:10A10000C2F20103019A1A6003B05DF804FB00BFBC
:10A110002DE9F0434DF67068C2F200082DED028B78
:10A12000D8ED027A9FED748A9FED746AF6EE008A8C
:10A13000F0EE686AE7EE886A48F21C53C2F2010347
:10A14000B2EE0E7A26EE877A4FF61147C7EE087AFE
:10A1500091B0C2F200071B6803933A78039941F269
:10A160006003C2F20103012A196077EE867AFCEEE1
:10A17000E77ACDED017A9DF8046000F0E08140F6C9
:10A180005C70C2F201000EF073FD43F2A473C0F2E2
:10A19000020393E803000AAC00254FF0203363600C
:10A1A000A360E5602561A38125750A9040F65C7087
:10A1B0002A46ADF82C10C2F2010029460EF014FD1B
:10A1C000204618F07DFA024640F65C702146C2F245
:10A1D00001000FF0FBFB4EF200202B460A2229461D
:10A1E000C2F200000FF078FC43F290200121C0F28F
:10A1F000020013F0E3FA4EF200202B460A22294611
:10A20000C2F200000FF068FC43F26C500321C0F270
:10A21000020013F0D3FA204618F052FA0146204605
:10A2200013F0CCFA43F240100121C0F2020013F007
:10A23000C5FA4EF20020C2F200000FF03BFC40F6DF
:10A240005C702A2301223146C2F201000A95656042
:10A25000A560E560256125758DF828300EF0C4FCF9
:10A26000204618F02DFA024640F65C702146C2F2F4
:10A2700001000FF0ABFB4EF200202B460A22012119
:10A28000C2F200000FF028FC43F290200121C0F23E
:10A29000020013F093FA4EF200202B460A223146B8
:10A2A000C2F200000FF018FC43F26C500321C0F220
:10A2B000020013F083FA204618F002FA0146204605
:10A2C00013F07CFA43F240100121C0F2020013F0B7
:10A2D00075FA4EF20020C2F200000FF0EBFBD8ED51
:10A2E000027AF0EE686A41F26408E7EE886AC2F228
:10A2F000010888F8006003E00000C8420000000088
:10A30000FDEEE67A0A2217EE900A04A917F094FDF2
:10A31000054618F0D5F9C0B20328024628BF03222B
:10A32000C2F1030043F23003C0F230032946204457
:10A3300000250A956560A560E56025612575ADF885
:10A340002830A37018F02AFA40F65C702A460D21D6
:10A35000C2F201000EF048FC204618F0B1F90246A6
:10A3600040F65C702146C2F201000FF02FFB4EF266
:10A3700000202B460A222946C2F200000FF0ACFB57
:10A3800043F290200121C0F2020013F017FA4EF2BE
:10A3900000202B460A220D21C2F200000FF09CFB88
:10A3A00043F26C500321C0F2020013F007FA20467A
:10A3B00018F086F90146204613F000FA43F24010E7
:10A3C0000121C0F2020013F0F9F94EF20020C2F2AE
:10A3D00000000FF06FFB98F8003041F26408B342C0
:10A3E000C2F2010800F0A48040F65C702A2301222A
:10A3F0003146C2F201000A956560A560E5602561FD
:10A4000025758DF828300EF0EFFB204618F058F92E
:10A41000024640F65C702146C2F201000FF0D6FA07
:10A420004EF200202B460A220121C2F200000FF05A
:10A4300053FB43F290200121C0F2020013F0BEF959
:10A440004EF200202B460A223146C2F200000FF0E5
:10A4500043FB43F26C500321C0F2020013F0AEF94B
:10A46000204618F02DF90146204613F0A7F943F2D3
:10A4700040100121C0F2020013F0A0F94EF20020BA
:10A48000C2F200000FF016FB98F800900A9540F613
:10A490005C70202349460122C2F201006560A5607C
:10A4A000E560256125758DF828300EF09DFB20466E
:10A4B00018F006F9024640F65C702146C2F201002F
:10A4C0000FF084FA4EF200202B460A220121C2F23C
:10A4D00000000FF001FB43F290200121C0F20200C6
:10A4E00013F06CF94EF200202B460A224946C2F2C4
:10A4F00000000FF0F1FA43F26C500321C0F20200A9
:10A5000013F05CF9204618F0DBF80146204613F002
:10A5100055F943F240100121C0F2020013F04EF948
:10A520004EF20020C2F200000FF0C4FA88F800607A
:10A5300001233B7011B0BDEC028BBDE8F08341F20A
:10A540006408C2F201080AACDAE600BF2DE9F04364
:10A550004FF61147C2F200078DB03B78002B40F058
:10A5600094854DF67066C2F2000669460A2230797B
:10A5700017F062FC044618F0A3F8C0B202280246A5
:10A5800028BF0222C2F1020006AB21461844002473
:10A5900043F2300306940794ADF8183008940994F8
:10A5A0000A948DF82C4018F0F9F840F65C702246B9
:10A5B0002146C2F201000EF017FB06A818F080F841
:10A5C000024640F65C7006A9C2F201000FF0FEF9E7
:10A5D0004EF2002023460A222146C2F200000FF06C
:10A5E0007BFA43F290200121C0F2020013F0E6F85A
:10A5F0004EF2002023460A222146C2F200000FF04C
:10A600006BFA43F26C500321C0F2020013F0D6F84B
:10A6100006A818F055F8014606A813F0CFF843F243
:10A6200040100121C0F2020013F0C8F84EF20020E1
:10A63000C2F200000FF03EFA40F65C7022460221A2
:10A64000C2F201004FF0200906940794089409947F
:10A650000A948DF82C408DF818900EF0C5FA06A8D3
:10A6600018F02EF8024640F65C7006A9C2F201000E
:10A670000FF0ACF94EF2002023460A222146C2F226
:10A6800000000FF029FA43F290200121C0F20200ED
:10A6900013F094F84EF2002023460A220221C2F25F
:10A6A00000000FF019FA43F26C500321C0F20200CF
:10A6B00013F084F806A818F003F8014606A813F072
:10A6C0007DF843F240100121C0F2020013F076F849
:10A6D0004EF20020C2F200000FF0ECF933794FF691
:10A6E000244003EB43024DF66E6803EB8203C2F293
:10A6F000000040F6A051C2F200081844C2F2010165
:10A7000005F0E4FE98F8005040F65C7015F0FD0589
:10A71000C2F2010000F0D082224602210694079482
:10A72000089409940A948DF82C408DF818900EF036
:10A730005BFA06A817F0C4FF024640F65C7006A953
:10A74000C2F201000FF042F94EF2002023460A2225
:10A750002146C2F200000FF0BFF943F29020012120
:10A76000C0F2020013F02AF84EF2002023460A221B
:10A770000221C2F200000FF0AFF943F26C50032146
:10A78000C0F2020013F01AF806A817F099FF01466C
:10A7900006A813F013F843F240100121C0F20200A2
:10A7A00013F00CF84EF20020C2F200000FF082F914
:10A7B00040F6A050C2F2010017F082FFC2B2082A90
:10A7C00040F6A05128BF08224FF02033C2F2010109
:10A7D00006A8069307940894CDF81B3009940A94B0
:10A7E0008DF82C4017F0DAFF40F65C70224603210A
:10A7F000C2F201000EF0F8F906A817F061FF024658
:10A8000040F65C7006A9C2F201000FF0DFF84EF2CC
:10A81000002023460A222146C2F200000FF05CF914
:10A8200043F290200121C0F2020012F0C7FF4EF265
:10A83000002023460A220321C2F200000FF04CF947
:10A8400043F26C500321C0F2020012F0B7FF06A8D9
:10A8500017F036FF014606A812F0B0FF43F2401091
:10A860000121C0F2020012F0A9FF4EF20020C2F254
:10A8700000000FF01FF940F65C7022460B21C2F277
:10A88000010006940794089409940A948DF82C40CA
:10A890008DF818900EF0A8F906A817F011FF0246DF
:10A8A00040F65C7006A9C2F201000FF08FF84EF27C
:10A8B000002023460A222146C2F200000FF00CF9C4
:10A8C00043F29020C0F20200012112F077FF2346EC
:10A8D0004EF200200A220B21C2F200000FF0FCF819
:10A8E00043F26C500321C0F2020012F067FF06A889
:10A8F00017F0E6FE014606A812F060FF43F2401092
:10A900000121C0F2020012F059FF4EF20020C2F203
:10A9100000000FF0CFF8707969460A22013017F075
:10A920008BFA044617F0CCFEC0B20228024628BFBC
:10A930000222C2F1020006AB21461844002443F271
:10A94000300306940794ADF81830089409940A94DB
:10A950008DF82C4017F022FF40F65C702146012252
:10A96000C2F201000EF040F906A817F0A9FE024657
:10A9700040F65C7006A9C2F201000FF027F84EF213
:10A98000002023460A220121C2F200000FF0A4F8A1
:10A9900043F290200121C0F2020012F00FFF4EF2AC
:10A9A000002023460A222146C2F200000FF094F84C
:10A9B00043F26C500321C0F2020012F0FFFE06A821
:10A9C00017F07EFE014606A812F0F8FE43F2401092
:10A9D0000121C0F2020012F0F1FE4EF20020C2F29C
:10A9E00000000FF067F840F65C7001220221C2F20D
:10A9F0000100202506940794089409940A948DF880
:10AA00002C408DF818500EF0EFF806A817F058FEFD
:10AA1000024640F65C7006A9C2F201000EF0D6FFB5
:10AA20004EF2002023460A220121C2F200000FF05C
:10AA300053F843F290200121C0F2020012F0BEFE52
:10AA40004EF2002023460A220221C2F200000FF03B
:10AA500043F843F26C500321C0F2020012F0AEFE44
:10AA600006A817F02DFE014606A812F0A7FE43F235
:10AA700040100121C0F2020012F0A0FE4EF20020B0
:10AA8000C2F200000FF016F898F8008008F0FD08F8
:10AA90004DF6706640F65C70B8F1010FC2F2000628
:10AAA000C2F2010000F0E78101220221069407941E
:10AAB000089409940A948DF82C408DF818500EF0E3
:10AAC00093F806A817F0FCFD024640F65C7006A954
:10AAD000C2F201000EF07AFF4EF2002023460A2255
:10AAE0000121C2F200000EF0F7FF43F29020012195
:10AAF000C0F2020012F062FE4EF2002023460A224B
:10AB00000221C2F200000EF0E7FF43F26C50032175
:10AB1000C0F2020012F052FE06A817F0D1FD014665
:10AB200006A812F04BFE43F240100121C0F20200D1
:10AB300012F044FE4EF20020C2F200000EF0BAFF06
:10AB4000727940F6F05302EB820602EB4606C2F23F
:10AB500001031E44304617F0B3FDC2B20A2A28BFD3
:10AB60000A224FF02033314606A806930793089433
:10AB700009940A948DF82C408DF8205017F00EFEA1
:10AB800040F65C7001220321C2F201000EF02CF8A5
:10AB900006A817F095FD024640F65C7006A9C2F2C1
:10ABA00001000EF013FF4EF2002023460A2201217D
:10ABB000C2F200000EF090FF43F290200121C0F29B
:10ABC000020012F0FBFD4EF2002023460A22032170
:10ABD000C2F200000EF080FF43F26C500321C0F27D
:10ABE000020012F0EBFD06A817F06AFD014606A868
:10ABF00012F0E4FD43F240100121C0F2020012F015
:10AC0000DDFD4EF20020C2F200000EF053FF40F6D0
:10AC10005C7001220E21C2F2010006940794089490
:10AC200009940A948DF82C408DF818500DF0DCFF33
:10AC300006A817F045FD024640F65C7006A9C2F270
:10AC400001000EF0C3FE4EF2002023460A2201212D
:10AC5000C2F200000EF040FF43F290200121C0F24A
:10AC6000020012F0ABFD4EF2002023460A220E2114
:10AC7000C2F200000EF030FF43F26C500321C0F22C
:10AC8000020012F09BFD06A817F01AFD014606A867
:10AC900012F094FD43F240100121C0F2020012F0C4
:10ACA0008DFD4EF20020C2F200000EF003FF0023E3
:10ACB0003B700DB0BDE8F0835B232A460221069568
:10ACC00007958DF81830089509950A958DF82C5040
:10ACD0000DF08AFF06A817F0F3FC024640F65C7000
:10ACE00006A9C2F201000EF071FE4EF200202B46C2
:10ACF0000A222946C2F200000EF0EEFE43F2902036
:10AD00000121C0F2020012F059FD4EF200202B4644
:10AD10000A220221C2F200000EF0DEFE43F26C5065
:10AD20000321C0F2020012F049FD06A817F0C8FC8A
:10AD3000014606A812F042FD43F240100121C0F284
:10AD4000020012F03BFD4EF20020C2F200000EF0B5
:10AD5000B1FE40F6A050C2F2010017F0B1FCC2B241
:10AD6000082A40F6A05128BF08224FF02033C2F233
:10AD7000010106A8069307950895CDF81B300995A3
:10AD80000A958DF82C5017F009FD40F65C702A46A4
:10AD90000321C2F201000DF027FF06A817F090FC76
:10ADA000024640F65C7006A9C2F201000EF00EFEEB
:10ADB0004EF200202B460A222946C2F200000EF075
:10ADC0008BFE43F290200121C0F2020012F0F6FC4B
:10ADD0004EF200202B460A220321C2F200000EF0A0
:10ADE0007BFE43F26C500321C0F2020012F0E6FC3D
:10ADF00006A817F065FC014606A812F0DFFC43F236
:10AE000040100121C0F2020012F0D8FC4EF20020E6
:10AE1000C2F200000EF04EFE40F65C705D232A4642
:10AE20000B21C2F20100069507958DF818300895A0
:10AE300009950A958DF82C500DF0D6FE06A817F04E
:10AE40003FFC024640F65C7006A9C2F201000EF01B
:10AE5000BDFD4EF200202B460A222946C2F2000018
:10AE60000EF03AFE43F29020C0F20200012112F0EF
:10AE7000A5FC2B462CE55B23424602210694079451
:10AE80008DF81830089409940A948DF82C400DF030
:10AE9000ABFE06A817F014FC024640F65C7006A94B
:10AEA000C2F201000EF092FD4EF2002023460A226B
:10AEB0004146C2F200000EF00FFE43F290204146E0
:10AEC000C0F2020012F07AFC4EF2002023460A2261
:10AED0000221C2F200000EF0FFFD43F26C5003218C
:10AEE000C0F2020012F06AFC06A817F0E9FB014666
:10AEF00006A812F063FC43F240104146C0F2020083
:10AF000012F05CFC4EF20020C2F200000EF0D2FD06
:10AF1000727940F6F05302EB820602EB4606C2F26B
:10AF200001031E44304617F0CBFBC2B20A2A28BFE9
:10AF30000A224FF02033314606A80693079308945F
:10AF400009940A948DF82C408DF8205017F026FCB7
:10AF500040F65C7042460321C2F201000DF044FE4F
:10AF600006A817F0ADFB024640F65C7006A9C2F2D7
:10AF700001000EF02BFD4EF2002023460A2241462E
:10AF8000C2F200000EF0A8FD43F290204146C0F24C
:10AF9000020012F013FC4EF2002023460A22032185
:10AFA000C2F200000EF098FD43F26C500321C0F293
:10AFB000020012F003FC06A817F082FB014606A867
:10AFC00012F0FCFB43F240104146C0F2020012F0C6
:10AFD000F5FB4EF20020C2F200000EF06BFD40F6D1
:10AFE0005C705D2342460E21C2F201000694079474
:10AFF0008DF81830089409940A948DF82C400DF0BF
:10B00000F3FD06A817F05CFB024640F65C7006A94B
:10B01000C2F201000EF0DAFC4EF2002023460A22B2
:10B020004146C2F200000EF057FD43F29020414627
:10B03000C0F2020012F0C2FB4EF2002023460A22A8
:10B040000E21C2F200000EF047FD43F26C500321C6
:10B05000C0F2020012F0B2FB06A817F031FB014665
:10B0600006A812F0ABFB43F240104146C0F20200CA
:10B0700012F0A4FB4EF20020C2F200000EF01AFD06
:10B0800000233B700DB0BDE8F08340F65C70C2F267
:10B0900001000DF0EDFDFFF764BA00BF2DE9F041AE
:10B0A0004FF61146C2F200068CB03378032B00F045
:10B0B0003E8340F65C70C2F201000DF0D9FD43F210
:10B0C000AC73C0F2020393E8030006AC00254FF016
:10B0D0002033A3606360E5602561C4F80B302575FB
:10B0E000069040F65C702A46ADF81C10C2F20100D2
:10B0F00029460DF079FD204617F0E2FA024640F6A7
:10B100005C702146C2F201000EF060FC4EF200209D
:10B110002B460A222946C2F200000EF0DDFC43F263
:10B1200090200121C0F2020012F048FB4EF20020F4
:10B130002B460A222946C2F200000EF0CDFC43F253
:10B140006C500321C0F2020012F038FB204617F0C9
:10B15000B7FA0146204612F031FB43F240100121BC
:10B16000C0F2020012F02AFB4EF20020C2F20000F0
:10B170000EF0A0FC46F2525340F65C70C3F6732307
:10B1800029460122C2F201006560A560E5602561E3
:10B19000257506930DF028FD204617F091FA02461A
:10B1A00040F65C702146C2F201000EF00FFC4EF238
:10B1B00000202B460A220121C2F200000EF08CFC76
:10B1C00043F290200121C0F2020012F0F7FA4EF291
:10B1D00000202B460A222946C2F200000EF07CFC19
:10B1E00043F26C500321C0F2020012F0E7FA20464D
:10B1F00017F066FA0146204612F0E0FA43F24010DA
:10B200000121C0F2020012F0D9FA4EF20020C2F27F
:10B2100000000EF04FFC47F2435340F65C70C3F65B
:10B22000742301220821C2F201006560A560E56077
:10B230002561257506930DF0D7FC204617F040FADE
:10B24000024640F65C702146C2F201000EF0BEFBE1
:10B250004EF200202B460A220121C2F200000EF01D
:10B260003BFC43F290200121C0F2020012F0A6FA4A
:10B270004EF200202B460A220821C2F200000EF0F6
:10B280002BFC43F26C500321C0F2020012F096FA3C
:10B29000204617F015FA0146204612F08FFA43F2C5
:10B2A0004010C0F20200012112F088FA4EF2002094
:10B2B000C2F200000EF0FEFB40F6ED53C2F20103B5
:10B2C0004FF2CB081B7803EB830303EB8303C2F637
:10B2D0008D089B0088FB0320DB17C3EB2010694619
:10B2E0000A2216F0A9FD054617F0EAF9C0B20228B5
:10B2F000024628BF0222C2F10200294643F230076B
:10B300000025204406956560A560E56025612575EA
:10B31000ADF8187017F042FA40F65C700122052172
:10B32000C2F201000DF060FC204617F0C9F9024698
:10B3300040F65C702146C2F201000EF047FB4EF26F
:10B3400000202B460A220121C2F200000EF0C4FBAD
:10B3500043F290200121C0F2020012F02FFA4EF2C7
:10B3600000200A222B460521C2F200000EF0B4FB99
:10B3700043F26C500321C0F2020012F01FFA204683
:10B3800017F09EF90146204612F018FA43F24010D9
:10B390000121C0F2020012F011FA4EF20020C2F2B6
:10B3A00000000EF087FB4FF61043C2F2000369461F
:10B3B0001B7803EB830303EB83039B0088FB0320D1
:10B3C000DB17C3EB20100A2216F036FD804617F07B
:10B3D00077F9C0B20228024628BF0222C2F1020059
:10B3E0004146204406956560A560E56025612575A8
:10B3F000ADF8187017F0D2F940F65C7001220D21FB
:10B40000C2F201000DF0F0FB204617F059F9024698
:10B4100040F65C702146C2F201000EF0D7FA4EF2FF
:10B4200000202B460A220121C2F200000EF054FB3C
:10B4300043F290200121C0F2020012F0BFF94EF257
:10B4400000202B460A220D21C2F200000EF044FB20
:10B4500043F26C500321C0F2020012F0AFF9204613
:10B4600017F02EF90146204612F0A8F943F24010D9
:10B470000121C0F202004DF66E6712F09FF9C2F290
:10B4800000074EF20020C2F200000EF013FB97F806
:10B49000008040F65C70B8F1040FC2F2010000F0C9
:10B4A0004881012204214FF0200806956560A560BF
:10B4B000E560256125758DF818800DF095FB204617
:10B4C00017F0FEF8024640F65C702146C2F2010019
:10B4D0000EF07CFA4EF200202B460A220121C2F225
:10B4E00000000EF0F9FA43F290200121C0F20200B0
:10B4F00012F064F94EF200200A222B460421C2F217
:10B5000000000EF0E9FA43F26C500321C0F2020091
:10B5100012F054F9204617F0D3F80146204612F0F5
:10B520004DF943F240100121C0F2020012F046F939
:10B530004EF20020C2F200000EF0BCFA40F65C7041
:10B540000695C2F201006560A560E560256125757C
:10B55000012207218DF818800DF046FB204617F0D8
:10B56000AFF8024640F65C702146C2F201000EF0D0
:10B570002DFA4EF200202B460A220121C2F20000D1
:10B580000EF0AAFA43F290200121C0F2020012F05C
:10B5900015F94EF200202B460A220721C2F20000C4
:10B5A0000EF09AFA43F26C500321C0F2020012F03E
:10B5B00005F9204617F084F80146204612F0FEF8FF
:10B5C00043F240100121C0F2020012F0F7F84EF2EF
:10B5D0000020C2F200000EF06DFA3B7840F65C707D
:10B5E000052B4FF00005C2F2010000F0FE800122A1
:10B5F0000C21202706956560A560E560256125750D
:10B600008DF818700DF0F0FA204617F059F8024640
:10B6100040F65C702146C2F201000EF0D7F94EF2FE
:10B6200000202B460A220121C2F200000EF054FA3B
:10B6300043F290200121C0F2020012F0BFF84EF256
:10B6400000200A222B460C21C2F200000EF044FA20
:10B6500043F26C500321C0F2020012F0AFF8204612
:10B6600017F02EF80146204612F0A8F843F24010D9
:10B670000121C0F2020012F0A1F84EF20020C2F245
:10B6800000000EF017FA40F65C700695C2F2010059
:10B690006560A560E5602561257501220F218DF8A3
:10B6A00018700DF0A1FA204617F00AF8024640F68D
:10B6B0005C702146C2F201000EF088F94EF20020C3
:10B6C0002B460A220121C2F200000EF005FA43F2D5
:10B6D00090200121C0F2020012F070F84EF200201A
:10B6E0002B460A220F21C2F200000EF0F5F943F2B8
:10B6F0006C500321C0F2020012F060F8204616F0F0
:10B70000DFFF0146204612F059F843F240100121B4
:10B71000C0F2020012F052F84EF20020C2F2000015
:10B720000EF0C8F9032333700CB0BDE8F08106AC0D
:10B73000C2E55B230122414606956560A560E56090
:10B74000256125758DF818300DF04EFA204616F05B
:10B75000B7FF024640F65C702146C2F201000EF0CF
:10B7600035F94EF200202B460A220121C2F20000D8
:10B770000EF0B2F943F290200121C0F2020012F063
:10B780001DF84EF200202B460A224146C2F200006C
:10B790000EF0A2F943F26C500321C0F2020012F045
:10B7A0000DF8204616F08CFF0146204612F006F8F0
:10B7B00043F240100121C0F2020011F0FFFF4EF2EF
:10B7C0000020C2F200000EF075F940F65C705D23B7
:10B7D0000695C2F201006560A560E56025612575EA
:10B7E000012207218DF81830B6E65B2301220C21D7
:10B7F00006956560A560E560256125758DF81830B2
:10B800000DF0F2F9204616F05BFF024640F65C7040
:10B810002146C2F201000EF0D9F84EF200202B466C
:10B820000A220121C2F200000EF056F943F29020E4
:10B830000121C0F2020011F0C1FF4EF200202B46A0
:10B840000A220C21C2F200000EF046F943F26C50BD
:10B850000321C0F2020011F0B1FF204616F030FFC4
:10B860000146204611F0AAFF43F240100121C0F228
:10B87000020011F0A3FF4EF20020C2F200000EF011
:10B8800019F940F65C705D230695C2F2010065600F
:10B89000A560E5602561257501220F218DF818301E
:10B8A000FFE600BFF0B548F21C53C2F201034FF6A9
:10B8B00011468FB0C2F200061B68019332780199DD
:10B8C00041F26003C2F20103022A196000F0D18044
:10B8D00040F65C70C2F201000DF0CAF943F2B47395
:10B8E000C0F2020393E8070008AC00254FF02033B4
:10B8F000E560C4F80B3084E8070040F65C702A4627
:10B900002946C2F20100256125750DF06DF920462A
:10B9100016F0D6FE024640F65C702146C2F20100E7
:10B920000EF054F84EF200202B4629460A22C2F2AD
:10B9300000000EF0D1F843F290200121C0F2020085
:10B9400011F03CFF4EF200202B460A222946C2F29B
:10B9500000000EF0C1F843F26C500321C0F2020067
:10B9600011F02CFF204616F0ABFE0146204611F0E8
:10B9700025FF43F240100121C0F202004DF670672E
:10B9800011F01CFFC2F200074EF20020C2F20000CC
:10B990000EF090F83D7C002D73D00A2202A92846B3
:10B9A00016F04AFA054616F08BFEC0B2022802468F
:10B9B00028BF0222C2F1020043F23003294620448C
:10B9C000002508956560A560E56025612575ADF8E1
:10B9D000203016F0E3FE40F65C7029460122C2F2E8
:10B9E00001000DF001F9204616F06AFE024640F60D
:10B9F0005C702146C2F201000DF0E8FF4EF200201B
:10BA00002B460A220121C2F200000EF065F843F233
:10BA100090200121C0F2020011F0D0FE4EF2002071
:10BA20002B460A222946C2F200000EF055F843F2D6
:10BA30006C500321C0F2020011F0C0FE204616F047
:10BA40003FFE0146204611F0B9FE43F240100121AD
:10BA5000C0F2020011F0B2FE4EF20020C2F200006D
:10BA60000EF028F83F7C012F60D0022333700FB016
:10BA7000F0BD4DF67067C2F2000708AC3D7C002DAA
:10BA80008BD144F64F5340F65C70C4F64E132946F2
:10BA90000122C2F201006560A560E560256125759F
:10BAA00008930DF0A1F8204616F00AFE024640F673
:10BAB0005C702146C2F201000DF088FF4EF20020BA
:10BAC0002B460A220121C2F200000EF005F843F2D3
:10BAD00090200121C0F2020011F070FE4EF2002011
:10BAE0002B460A222946C2F200000DF0F5FF43F270
:10BAF0006C500321C0F2020011F060FE204616F0E7
:10BB0000DFFD0146204611F059FE43F240100121AD
:10BB1000C0F2020011F052FE4EF20020C2F200000C
:10BB20000DF0C8FF022333700FB0F0BD40F65C701B
:10BB300042F220033A460221C2F2010008956560F4
:10BB4000A560E56025612575ADF820300DF04CF855
:10BB5000204616F0B5FD024640F65C702146C2F262
:10BB600001000DF033FF4EF200202B460A22394629
:10BB7000C2F200000DF0B0FF43F290203946C0F24F
:10BB8000020011F01BFE4EF200202B460A22022179
:10BB9000C2F200000DF0A0FF43F26C500321C0F28E
:10BBA000020011F00BFE204616F08AFD01462046E9
:10BBB00011F004FE43F240103946C0F2020011F0C9
:10BBC000FDFD4EF20020C2F200000DF073FF0223D3
:10BBD00033700FB0F0BD00BF2DE9F0414FF61146B4
:10BBE000C2F200068CB03378042B00F0F88440F6E3
:10BBF0005C70C2F201000DF03BF843F2C473C0F276
:10BC0000020393E8030006AC00256560A560E560CB
:10BC100025612575069040F65C702A468DF81C104B
:10BC2000C2F2010029460CF0DFFF204616F048FD65
:10BC3000024640F65C702146C2F201000DF0C6FEDD
:10BC40004EF200202B460A222946C2F200000DF0D7
:10BC500043FF43F290200121C0F2020011F0AEFD3B
:10BC60004EF200202B460A222946C2F200000DF0B7
:10BC700033FF43F26C500321C0F2020011F09EFD2D
:10BC8000204616F01DFD0146204611F097FD43F2B7
:10BC900040100121C0F2020011F090FD4EF2002090
:10BCA000C2F200000DF006FF40F65C7043F654232C
:10BCB0002A460621C2F2010006956560A560E5608E
:10BCC00025612575ADF818300CF08EFF204616F072
:10BCD000F7FC024640F65C702146C2F201000DF00E
:10BCE00075FE4EF200202B460A222946C2F20000C1
:10BCF0000DF0F2FE43F290200121C0F2020011F09B
:10BD00005DFD4EF200202B460A220621C2F2000001
:10BD10000DF0E2FE43F26C500321C0F2020011F07C
:10BD20004DFD204616F0CCFC0146204611F046FDA4
:10BD300043F240100121C0F2020011F03FFD4EF22B
:10BD40000020C2F200000DF0B5FE40F65C7047F234
:10BD50006D332A460E21C2F2010006956560A5608A
:10BD6000E56025612575ADF818300CF03DFF2046E3
:10BD700016F0A6FC024640F65C702146C2F20100B5
:10BD80000DF024FE4EF200202B460A222946C2F274
:10BD900000000DF0A1FE43F290200121C0F202004C
:10BDA00011F00CFD4EF200202B460A220E21C2F2A9
:10BDB00000000DF091FE43F26C500321C0F202002E
:10BDC00011F0FCFC204616F07BFC0146204611F0E9
:10BDD000F5FC43F240100121C0F2020011F0EEFC2C
:10BDE0004EF20020C2F200000DF064FE43F2CC736C
:10BDF000C0F2020340F65C701B6806951F0C2946D2
:10BE00000122C2F201006560A560E560256125752B
:10BE1000ADF818308DF81A700CF0E6FE204616F0DA
:10BE20004FFC024640F65C702146C2F201000DF064
:10BE3000CDFD4EF200202B460A220121C2F2000065
:10BE40000DF04AFE43F290200121C0F2020011F0F1
:10BE5000B5FC4EF200202B460A222946C2F2000011
:10BE60000DF03AFE43F26C500321C0F2020011F0D3
:10BE7000A5FC204616F024FC0146204611F09EFC4D
:10BE800043F240100121C0F2020011F097FC4EF283
:10BE90000020C2F200000DF00DFE46F6567340F68B
:10BEA0005C70C3F66C2301220821C2F201006560B8
:10BEB000A560E5602561257506930CF095FE20468A
:10BEC00016F0FEFB024640F65C702146C2F201000D
:10BED0000DF07CFD4EF200202B460A220121C2F219
:10BEE00000000DF0F9FD43F290200121C0F20200A4
:10BEF00011F064FC4EF200202B460A220821C2F207
:10BF000000000DF0E9FD43F26C500321C0F2020085
:10BF100011F054FC204616F0D3FB0146204611F0E8
:10BF20004DFC43F24010C0F20200012111F046FC2A
:10BF30004EF20020C2F200000DF0BCFD40F24012B3
:10BF4000C2F201024FF49663107848F21F57C5F20F
:10BF5000EB1703FB00F387FB0320DB17C3EB201079
:10BF600069460A2215F068FF054616F0A9FBC0B223
:10BF70000428024628BF0422C2F104004FF03033E7
:10BF80002946204400256560A560E560256125758A
:10BF9000069316F003FC40F65C702A460921C2F2B3
:10BFA00001000CF021FE204616F08AFB024640F606
:10BFB0005C702146C2F201000DF008FD4EF2002037
:10BFC0002B460A222946C2F200000DF085FD43F2FD
:10BFD00090200121C0F2020011F0F0FB4EF200208F
:10BFE0000A222B460921C2F200000DF075FD43F232
:10BFF0006C500321C0F2020011F0E0FB204616F065
:10C000005FFB0146204611F0D9FB43F240100121AD
:10C01000C0F2020011F0D2FB4EF20020C2F200008A
:10C020000DF048FD40F6EC53C2F201034AF2EB007A
:10C030001B7803EB430303EB4313CEF60E2080FB88
:10C0400003201844DB17C3EB601069460A2215F081
:10C05000F3FE804616F034FBC0B20228024628BF29
:10C060000222C2F102004146204443F23008069504
:10C070006560A560E56025612575ADF8188016F04E
:10C080008DFB40F65C7001220421C2F201000CF02D
:10C09000ABFD204616F014FB024640F65C702146CC
:10C0A000C2F201000DF092FC4EF200202B460A2253
:10C0B0000121C2F200000DF00FFD43F2902001219A
:10C0C000C0F2020011F07AFB4EF200200A222B4649
:10C0D0000421C2F200000DF0FFFC43F26C5003217A
:10C0E000C0F2020011F06AFB204616F0E9FA0146A0
:10C0F000204611F063FB43F240100121C0F2020020
:10C1000011F05CFB4EF20020C2F200000DF0D2FCF8
:10C1100040F67073C2F2010369461B7803EB4303D8
:10C1200003EB431387FB0320DB17C3EB20100A222A
:10C1300015F082FE074616F0C3FAC0B20228024686
:10C1400028BF0222C2F102003946204406956560EC
:10C15000A560E56025612575ADF8188016F01EFB19
:10C1600040F65C7001220D21C2F201000CF03CFD92
:10C17000204616F0A5FA024640F65C702146C2F24F
:10C1800001000DF023FC4EF200202B460A22012173
:10C19000C2F200000DF0A0FC43F290200121C0F299
:10C1A000020011F00BFB4EF200202B460A220D215B
:10C1B000C2F200000DF090FC43F26C500321C0F27B
:10C1C000020011F0FBFA204616F07AFA01462046EA
:10C1D00011F0F4FA43F240100121C0F202004DF6D2
:10C1E0006E6711F0EBFAC2F200074EF20020C2F2C5
:10C1F00000000DF05FFC3B7840F65C70062BC2F24D
:10C20000010000F04A822A4608214FF020080695D6
:10C210006560A560E560256125758DF818800CF0D6
:10C22000E3FC204616F04CFA024640F65C702146CC
:10C23000C2F201000DF0CAFB4EF200202B460A228A
:10C240002946C2F200000DF047FC43F29020012184
:10C25000C0F2020011F0B2FA4EF200200A222B4680
:10C260000821C2F200000DF037FC43F26C500321AC
:10C27000C0F2020011F0A2FA204616F021FA01469F
:10C28000204611F09BFA43F240100121C0F2020057
:10C2900011F094FA4EF20020C2F200000DF00AFCF8
:10C2A00040F65C700695C2F201006560A560E5602D
:10C2B000256125752A460D218DF818800CF094FC17
:10C2C000204616F0FDF9024640F65C702146C2F2A7
:10C2D00001000DF07BFB4EF200202B460A2229467E
:10C2E000C2F200000DF0F8FB43F290200121C0F2F1
:10C2F000020011F063FA4EF200202B460A220D21B3
:10C30000C2F200000DF0E8FB43F26C500321C0F2D2
:10C31000020011F053FA204616F0D2F901462046E9
:10C3200011F04CFA43F240100121C0F2020011F06A
:10C3300045FA4EF20020C2F200000DF0BBFB3B7844
:10C3400040F65C70072B4FF00005C2F2010000F0D0
:10C350004881012203214FF0200806956560A56001
:10C36000E560256125758DF818800CF03DFC2046B0
:10C3700016F0A6F9024640F65C702146C2F20100B2
:10C380000DF024FB4EF200202B460A220121C2F2BE
:10C3900000000DF0A1FB43F290200121C0F2020049
:10C3A00011F00CFA4EF200200A222B460321C2F2B1
:10C3B00000000DF091FB43F26C500321C0F202002B
:10C3C00011F0FCF9204616F07BF90146204611F0E9
:10C3D000F5F943F240100121C0F2020011F0EEF92C
:10C3E0004EF20020C2F200000DF064FB40F65C70DB
:10C3F0000695C2F201006560A560E56025612575BE
:10C40000012206218DF818800CF0EEFB204616F074
:10C4100057F9024640F65C702146C2F201000DF069
:10C42000D5FA4EF200202B460A220121C2F200006A
:10C430000DF052FB43F290200121C0F2020011F0F6
:10C44000BDF94EF200202B460A220621C2F200005E
:10C450000DF042FB43F26C500321C0F2020011F0D8
:10C46000ADF9204616F02CF90146204611F0A6F948
:10C4700043F240100121C0F2020011F09FF94EF288
:10C480000020C2F200000DF015FB3B7840F65C7016
:10C49000082B4FF00005C2F2010000F05A81012282
:10C4A0000C21202706956560A560E560256125754E
:10C4B0008DF818700CF098FB204616F001F9024632
:10C4C00040F65C702146C2F201000DF07FFA4EF298
:10C4D00000202B460A220121C2F200000DF0FCFAD6
:10C4E00043F290200121C0F2020011F067F94EF2F0
:10C4F00000200A222B460C21C2F200000DF0ECFABB
:10C5000043F26C500321C0F2020011F057F92046AB
:10C5100016F0D6F80146204611F050F943F24010CB
:10C520000121C0F2020011F049F94EF20020C2F2DE
:10C5300000000DF0BFFA40F65C700695C2F20100F3
:10C540006560A560E5602561257501220F218DF8E4
:10C5500018700CF049FB204616F0B2F8024640F67F
:10C560005C702146C2F201000DF030FA4EF200205C
:10C570002B460A220121C2F200000DF0ADFA43F26F
:10C5800090200121C0F2020011F018F94EF20020B3
:10C590002B460A220F21C2F200000DF09DFA43F251
:10C5A0006C500321C0F2020011F008F9204616F089
:10C5B00087F80146204611F001F943F240100121AD
:10C5C000C0F2020011F0FAF84EF20020C2F20000B0
:10C5D0000DF070FA042333700CB0BDE8F08106ACA6
:10C5E000ACE45B230122032106956560A560E5604C
:10C5F000256125758DF818300CF0F6FA204616F0F6
:10C600005FF8024640F65C702146C2F201000DF070
:10C61000DDF94EF200202B460A220121C2F2000071
:10C620000DF05AFA43F290200121C0F2020011F0FD
:10C63000C5F84EF200202B460A220321C2F2000068
:10C640000DF04AFA43F26C500321C0F2020011F0DF
:10C65000B5F8204616F034F80146204611F0AEF841
:10C6600043F240100121C0F2020011F0A7F84EF28F
:10C670000020C2F200000DF01DFA40F65C705D2350
:10C680000695C2F201006560A560E560256125752B
:10C69000012206218DF81830B6E65B232A460821D0
:10C6A00006956560A560E560256125758DF81830F3
:10C6B0000CF09AFA204616F003F8024640F65C7039
:10C6C0002146C2F201000DF081F94EF200202B4606
:10C6D0000A222946C2F200000DF0FEF943F2902032
:10C6E0000121C0F2020011F069F84EF200202B4641
:10C6F0000A220821C2F200000DF0EEF943F26C505C
:10C700000321C0F2020011F059F8204615F0D8FFBD
:10C710000146204611F052F843F240100121C0F2C8
:10C72000020011F04BF84EF20020C2F200000DF0B2
:10C73000C1F940F65C705D230695C2F201006560A8
:10C74000A560E560256125752A460D218DF8183014
:10C75000B4E55B2301220C2106956560A560E560C8
:10C76000256125758DF818300CF03EFA204615F03D
:10C77000A7FF024640F65C702146C2F201000DF0B0
:10C7800025F94EF200202B460A220121C2F20000B8
:10C790000DF0A2F943F290200121C0F2020011F045
:10C7A0000DF84EF200202B460A220C21C2F20000A6
:10C7B0000DF092F943F26C500321C0F2020010F028
:10C7C000FDFF204615F07CFF0146204610F0F6FFE5
:10C7D00043F240100121C0F2020010F0EFFF4EF2D0
:10C7E0000020C2F200000DF065F940F65C705D2398
:10C7F0000695C2F201006560A560E56025612575BA
:10C8000001220F218DF81830A3E600BF2DE9F04F6B
:10C810002DED068B48F21C57C2F2010789B041F298
:10C8200060023B680493C2F20102049B116840F667
:10C83000B7325B1A934207D94FF61143C2F2000395
:10C840001B78002B40F0488140F6C848C2F201082E
:10C8500040F66C733A680592C2F2010341F28732E6
:10C860001968059B5B1A934208D94DF66E63C2F2B4
:10C8700000031A78911E012940F2E28040F6C84474
:10C88000C2F2010440F6CC534FF618464BF6836AC9
:10C8900004F10C02C2F201039FEDD08A9FEDD09A01
:10C8A000DFEDD08A9FEDD0AADFEDD09ACDF80480DD
:10C8B000C2F200060093C2F6A07A0025904603EB70
:10C8C000051B58460BF0FAFF58465FFA85F90CF045
:10C8D0003BF838B13B68069340F6B053C2F201030F
:10C8E000069A1A6058460CF025F8A0B340F6B053EB
:10C8F0003A680792C2F201031A68079B9B1AB3F5C4
:10C90000FA7F00F223814FF61143C2F20003B9F11E
:10C91000010F1B7800F0D580012B00F07284C0F06D
:10C920001183022B00F08784AB4643F2FC70072191
:10C93000C0F2020010F042FF4EF200205946C2F24F
:10C94000000000230A220DF0C7F84EF20020C2F2C8
:10C9500000000DF0AFF8237C012B40F2498172B644
:10C96000E36862B6002B56F8042BB8BF0333B2EB72
:10C97000A30F5CD0B9F1010F6DD14FF61142C2F295
:10C9800000021378012B00F0AE82C0F06983032B04
:10C9900000F0FA81042B0FD14DF66E63C2F2000352
:10C9A0001B78072B00F0E986082B00F0CB84062BC0
:10C9B00000F05387FFF710F943F648100821C0F242
:10C9C000020010F0FBFE4EF2002000230A2229464E
:10C9D000C2F200000DF080F843F22C50C0F20200C9
:10C9E000022110F0EBFE237C012B40F2068372B68D
:10C9F000E16862B60029B8BF03314EF20020891009
:10CA0000C2F200000CF0F8FF4EF20020C2F200006B
:10CA10000DF050F8237C012B40F2C48272B6E3681B
:10CA200062B6002BB8BF03339B1046F8043C0135B7
:10CA3000022D04F1140408F1140807D0009B3EE70E
:10CA4000032A40F0008101221A7017E709B0BDECFB
:10CA5000068BBDE8F08F4FF61143C2F200031B783E
:10CA6000012B40F2F380022BA6D1237C012B40F254
:10CA7000D28772B6E36862B6032B40F35185237CFC
:10CA8000012B41F2508072B6E36862B63F2B03DDA2
:10CA900072B64023E36062B6237C012B40F28F879D
:10CAA00072B6E36862B64DF67062002BC2F2000205
:10CAB000B8BF03339B101374F9F754FFFEF7F2FE6F
:10CAC0007AE7002B00F02982033B012B4FF0040191
:10CAD00040F23883CB4628E7033B012B7FF6B4AE08
:10CAE0004DF67063C2F2000393ED027ADFED3B6A0C
:10CAF000DFED3B7A9FED3B6A27EE267A27EE277A19
:10CB0000C7EE267A77EE867AFDEEE77A17EE903A50
:10CB10009B0072B640F6C848C2F20108C8F80C3053
:10CB200062B698F81030012B40F2388372B6D8F80C
:10CB30000C3062B64FF61842002BC2F20002B8BFAA
:10CB400003339B101360FDF701FD81E643F2D070C3
:10CB50002921C0F2020010F031FE4EF20020002325
:10CB60000A222946C2F200000CF0B6FF4EF2002065
:10CB7000C2F200000CF09EFFB9F1010FAB467FF44A
:10CB8000D4AE4FF61143C2F200031B78032B00F022
:10CB9000FC84042B00F0DA84002B7FF4C6AE4DF643
:10CBA0006E6240F6ED53C2F20002C2F201030421AC
:10CBB00011701B7872B69B00E36062B6237C012B78
:10CBC00041F2158372B6E36862B6002BB8BF033337
:10CBD0009B103360FEF762FAA7E600BF0000C84270
:10CBE00000002C420000000000000C4200FEFF4646
:10CBF00072B694E80C0010781978637A227A194298
:10CC000002EA000200F0B780A37A03F003030AB13E
:10CC100043F0040343F008039A10082BA27200F2B9
:10CC20001482072B80F03483032B00F0368340F20C
:10CC3000AF81042B00F0B281062B7FF491AEE36844
:10CC4000023BE3608DE600221A7017E6237C012B7D
:10CC500040F2898672B6E36862B6032B40F36684BD
:10CC6000237C012B40F28B8772B6E36862B6AB2B54
:10CC700003DD72B6AC23E36062B6237C012B40F285
:10CC8000228772B6E36862B6002B227CB8BF0333FA
:10CC90009B10012A46F8043C40F2E98672B6E3682C
:10CCA00062B6002BB8BF03339A10642303FB02F370
:10CCB0008AFB0312DB17C3EBE20307EE903AF8EEB0
:10CCC000E77A4DF6706387EE887AC2F2000340F689
:10CCD0003459C2F2010943F6040014221C21C0F2A7
:10CCE0000200A9F804200293D3ED027A77EE677A66
:10CCF000F3EE046A87EEA67A89ED007A10F05EFD05
:10CD0000029B986814F0AAFC41EC100B4EF2002034
:10CD10000521C2F200000CF01FFF43F624000E2193
:10CD2000C0F2020010F04AFD4EF20020B9F80410E3
:10CD3000C2F200000CF060FE43F634000E21C0F297
:10CD4000020010F03BFDD9F8000014F087FC41EC24
:10CD5000100B4EF200200521C2F200000CF0FCFE88
:10CD60004EF20020C2F200000CF0A4FEF9F7FAFD2A
:10CD7000FDF7CEF920E6A37A03F00303002A3FF47F
:10CD80004BAF43F0040347E74DF66E63C2F2000376
:10CD90001B78042B00F02084052B40F0A180237C1D
:10CDA000012B41F2E68272B6E36862B6032B40F3D0
:10CDB000E887237C012B41F2AB8472B6E36862B64C
:10CDC000B3F5C87F04DB72B64FF4C873E36062B694
:10CDD000237C012B41F2A18272B6E36862B6002B7C
:10CDE000227CB8BF03339B10012A46F8043C41F271
:10CDF000688272B6E36862B64FF61042002B217C5F
:10CE0000B8BF0333C2F200029B100129137041F234
:10CE1000528272B6E36862B6002BB8BF03339B1030
:10CE200007EE903AB8EEE77A40F6645BC7EE087A10
:10CE3000C2F2010B40F2C429DBF80030C2F2010952
:10CE400043F6A40014222321C0F20200A9F8042012
:10CE5000B7EE007A37EE677AD3ED497A77EE677AE4
:10CE6000F3EE046A87EEA67A89ED007A10F0A6FC4C
:10CE7000DBF80030D3F8240114F0F0FB41EC100B88
:10CE80004EF200200521C2F200000CF065FE43F6D0
:10CE9000C8001521C0F2020010F090FC4EF20020F4
:10CEA000B9F80410C2F200000CF0A6FD43F6E00051
:10CEB000C0F20200152110F081FCD9F8000014F036
:10CEC000CDFB41EC100B4EF20020C2F20000052118
:10CED0000CF042FE4EF20020C2F200000CF0EAFD1F
:10CEE000FEF7DCF868E54DF6706340F65C70C2F260
:10CEF00000030021C2F201000293039311700BF0B2
:10CF0000B7FE029B5B7972B6019A9B00136262B610
:10CF1000F9F728FDFDF71AFB4EE54DF66E62C2F2F9
:10CF200000021378012B00F01484C0F0E182022B80
:10CF300000F0DE82032B00F00C84FDF707FB4FF0BE
:10CF4000010BF2E44DF67063C2F2000393ED027A36
:10CF500027EE087A27EE097AC7EE087A77EEA87AE4
:10CF6000FDEEE77A17EE903A9B0072B6E36062B688
:10CF7000237C012B40F2108772B6E36862B6002B67
:10CF8000B8BF03339B103360AB46FDF7C1F8CCE468
:10CF9000012B00F07D81022B7FF4E2ACE368013BC2
:10CFA000E360DEE472B694E80C0010781978637AD6
:10CFB000227A194202EA000200F09680A37A03F076
:10CFC00003030AB143F0040343F008039A10082B4B
:10CFD000A27200F2A880072B80F0AF81032B00F033
:10CFE000B08240F26681042B00F0A880062B7FF40B
:10CFF00016ADE368023BE36012E572B694E80C00FC
:10D0000010781978637A227A194202EA000274D001
:10D01000A37A03F003030AB143F0040343F00803C7
:10D020009A10082BA27270D8072B80F07B81032BFB
:10D0300000F0828240F23681042B70D0062B7FF400
:10D04000D7ACE1680239E160D3E40C2B00F0258114
:10D0500000F21881092B3FF4F2AD0B2B9ED07FE438
:10D060004DF66E63C2F200031A78012A00F057856C
:10D07000C0F0FB81022A00F0FA81032A31D1237C1F
:10D08000012B40F2B18772B6E36862B6032B40F31E
:10D090001586237C012B41F2A38272B6E36862B647
:10D0A0007F2B4DF67063C2F2000307DD1A79622A06
:10D0B00041F2A68172B67C22E26062B6227C012A2D
:10D0C00040F2BC8772B6E26862B6002AB8BF03328B
:10D0D000C2F38702114618795A7103F0FDFCF9F783
:10D0E00041FCFDF733FA67E4A37A03F00303002A57
:10D0F0003FF46CAF43F0040368E7A37A03F0030343
:10D10000002A8DD043F004038AE70C2B00F0148230
:10D1100000F20281092B94D00B2B7FF469ACE168FB
:10D120000139E16065E40C2B00F00B8200F2FF8016
:10D13000092B3FF45EAF0B2B7FF471ACE368013B2E
:10D14000E3606DE44DF66E63C2F200031A78062ABE
:10D1500000F0558500F2BD80042A00F05785052AAD
:10D1600040F0F38240F6ED52C2F2010219701378DA
:10D1700072B69B00E36062B6237C012B41F25B82B6
:10D1800072B6E36862B6002BB8BF03339B103360FE
:10D190004FF0010BFDF782FFFFF7C7BB72B6D8F85F
:10D1A0000030D8F804101A78087898F8091098F820
:10D1B0000830084202EA030200F0828098F80A3040
:10D1C00003F003030AB143F0040343F008039A1089
:10D1D000082B88F80A2000F28D82072B80F0018549
:10D1E000032B00F0058540F23585042B00F08D827D
:10D1F000062B7FF49CACD8F80C30023BC8F80C30FE
:10D2000097E44DF67063C2F200031B7C72B69B007C
:10D21000E36062B6237C012B40F2218672B6E3689C
:10D2200062B6002BB8BF03339B103360AB46FEF7EA
:10D2300039FBFFF77ABB4DF67063C2F2000393ED42
:10D24000027A27EE087A27EE097AC7EE087A77EE97
:10D25000A87AFDEEE77A17EE903A9B0072B6E3608B
:10D2600062B6237C012B40F2CD8572B6E36862B6CC
:10D27000002BB8BF03339B103360AB46FDF766F954
:10D28000FFF753BB0D2B3FF489AE0E2B7FF468AB39
:10D29000E3680133E360FFF764BBE3680233E360F4
:10D2A000FFF75FBB012B3DD0022B3FF438AFFFF7F8
:10D2B0009FBB012B41D0022B3FF440AFFFF7AFBB28
:10D2C00098F80A3003F00303002A80D043F00403E7
:10D2D0007DE7072A00F02082082A40F0368240F2DB
:10D2E0004012C2F2010206211278197072B6930040
:10D2F000E36062B6237C012B41F2808172B6E36861
:10D3000062B6002BB8BF03339B1033604FF0010BA4
:10D31000FEF762FCFFF709BB0D2B3FF400AF0E2BAD
:10D320007FF466ABE1680131E160FFF762BB0D2B72
:10D330003FF404AF0E2B7FF472ABE3680133E3607C
:10D34000FFF76EBB237C012B41F2CC8172B6E36800
:10D3500062B6032B40F3DE85237C012B41F2308241
:10D3600072B6E36862B6CB2B03DD72B6C823E36006
:10D3700062B6237C012B41F2AF8172B6E36862B6DC
:10D38000002BB8BF0333C3F3870307EE903A9FED3A
:10D39000907AF8EE676A40F67079C6EE877AC2F244
:10D3A000010989F80030B7EE007A77EEA87A37EEF7
:10D3B000677AB4EEE97AF1EE10FA00F33B84DFED20
:10D3C000826AB4EEE67AF1EE10FA00F1F585F0EE3D
:10D3D000476AFEEEC86A16EE903A40F69042C2F2F4
:10D3E0000102F4EEE97AF1EE10FA936100F31D8484
:10D3F0009FED757AF4EEC77AF1EE10FA00F1EA8546
:10D40000B0EE677ABEEEC87A17EE103AF4EEE97A1B
:10D41000F1EE10FAD36101F39E849FED6B7AF4EE86
:10D42000C77AF1EE10FA00F1D085B0EE677ABEEE61
:10D43000C87A17EE103A43F62C101921C0F20200F8
:10D44000136210F0BBF94EF2002099F8001000238F
:10D450000A22C2F200000CF03FFB4EF20020C2F2A2
:10D4600000000CF027FBFFF7A5BA02221A70237CFC
:10D47000012B40F2388672B6E36862B6032B40F3A4
:10D480002A8440F6C859237CC2F20109012B99F87D
:10D4900000B041F2F68072B6E36862B6002BB8BF06
:10D4A0000333BBEBA30F06DC99F80030013B9B0074
:10D4B00072B6E36062B6237C012B40F2EA8572B655
:10D4C000E36862B61A1EB8BF03324DF67063C2F34A
:10D4D0008702C2F2000310461A71029303F014F897
:10D4E000029B5979187903F0F7FAF9F73BFAF8E556
:10D4F0004DF67063C2F2000301215B79117072B6C0
:10D500009B00E36062B6237C8B4240F2318172B6AD
:10D51000E36862B6002BB8BF03339B1033600CE5A1
:10D5200072B60023E36062B6FFF7B6BA72B60023A4
:10D53000E36062B6FFF7A1BBE1680231E160FFF78B
:10D5400058BAE3680233E360FFF76ABA4DF66E62D9
:10D550004DF67063C2F20002C2F2000382F800903E
:10D560005B7972B69B00E36062B6237C012B40F2CC
:10D57000118672B6E36862B6002BB8BF03339B1006
:10D580003360FCF7E3FFFFF7D0B94DF66E6240F26F
:10D590004013C2F20002C2F20103062111701B788F
:10D5A00072B69B00E36062B6237C012B40F2C58516
:10D5B00072B6E36862B6002BB8BF03339B103360CA
:10D5C000FEF70AFBFFF7B1B900FEFFC60000964464
:10D5D0000000484279783042237C012B40F23F869C
:10D5E00072B6E36862B6032B40F3D183237C012B30
:10D5F00041F24D8072B6E36862B6B3F5C87F04DBD2
:10D6000072B64FF4C873E36062B6237C012B40F21C
:10D61000788772B6E36862B6002B227CB8BF03330A
:10D620009B10012A46F8043C40F2138772B6E36867
:10D6300062B640F6ED52002B217CB8BF0333C2F234
:10D6400001029B100129137040F22F8772B6E36824
:10D6500062B6002BB8BF03339B1007EE903AF8EE8A
:10D66000E77A40F6645B87EE887AC2F2010B40F2FB
:10D670003819DBF80030C2F2010943F644001422E5
:10D680002621C0F20200A9F80420F7EE007A37EE56
:10D69000C77AD3ED4A7A77EE677AF3EE046A87EEBB
:10D6A000A67A89ED007A10F089F8DBF80030D3F81B
:10D6B000280113F0D3FF41EC100B4EF2002005219E
:10D6C000C2F200000CF048FA43F66C001821C0F2D8
:10D6D000020010F073F84EF20020B9F80410C2F204
:10D6E00000000CF089F943F68800C0F2020018210E
:10D6F000FFF7E1BB0C2B00F07B8200F26C82092B60
:10D700003FF479AD0B2B7FF412AAD8F80C30013B13
:10D71000C8F80C30FFF70DBA40F67072C2F2010281
:10D7200008211278197072B69300E36062B6237C08
:10D73000012B41F27F8172B6E36862B6002BB8BF5D
:10D7400003339B103360FEF747FA4FF0010BFFF7EE
:10D75000ECB84DF67063C2F2000300211B79117022
:10D7600072B69B00E36062B6237C012B3FF6CFAE1E
:10D7700072B62046FCF75AFCCAE6237C012B40F225
:10D780008C8772B6E36862B6032B40F3CD83237CAB
:10D79000012B41F23D8072B6E36862B68F2B03DD48
:10D7A00072B68C23E36062B6237C012B40F28E8735
:10D7B00072B6E36862B6002BB8BF0333C3F38703C6
:10D7C00007EE903AB8EE677A40F6EC59C7EE0A7A5F
:10D7D000C2F2010989F8003077EEA87AF4EEE97A0E
:10D7E000F1EE10FA00F31D821FED897AF4EEC77A8C
:10D7F000F1EE10FA00F1E583B0EE677ABEEEC87A7A
:10D8000017EE103A40F65842C2F2010243F61010E9
:10D810001B21C0F20200D3610FF0D0FF99F8003055
:10D8200007EE903AF8EE677A87EE8A7A77EE287AF2
:10D8300017EE900A13F012FF41EC100B4EF200208D
:10D840000221C2F200000CF087F94EF20020C2F271
:10D8500000000CF02FF9FFF7ADB8237C012B40F24C
:10D860002F8772B6E36862B6032B40F34E83237CA6
:10D87000012B40F2DC8772B6E36862B6CB2B03DD86
:10D8800072B6C823E36062B6237C012B40F2128794
:10D8900072B6E36862B6002BB8BF0333C3F38703E5
:10D8A00007EE903AB8EE677A5FEDB87A5FEDB86A46
:10D8B00067EE277A40F2401987EEA67AC2F2010994
:10D8C00089F8003077EE287AF5EEC07AF1EE10FA9A
:10D8D00000F126835FEDC16AB6EE007AA7EEA67A64
:10D8E0004FF4FC53C0F20103FCEEC77A17EE90EA46
:10D8F0009E4540F274839E464FF4107040F2F4232C
:10D90000C2F201031A7ED10700F19981D98BC3F8C5
:10D9100020E0814242F0010238BFD8831A7643F6F4
:10D92000F8001721C0F202000FF048FF99F800102C
:10D930004FF4966348F21F5203FB01F3C5F2EB125A
:10D9400082FB03124EF20020D917C1EB2211C2F262
:10D9500000000CF051F84EF20020C2F200000CF072
:10D96000A9F8FFF727B872B694E80C001078197878
:10D97000637A227A194202EA000200F08481A37AD3
:10D9800003F003030AB143F0040343F008039A10C1
:10D99000082BA27200F2A581072B80F02785032BAC
:10D9A00000F0528540F21486042B00F0A581062B6E
:10D9B0007FF451A9E368023BE360FFF74DB972B60B
:10D9C00094E80C0010781978637A227A194202EAF6
:10D9D000000200F04F81A37A03F003030AB143F081
:10D9E000040343F008039A10082BA27200F29981F5
:10D9F000072B80F0F084032B00F0BA8540F2F68507
:10DA0000042B00F09981062B7FF44BA8E368023BBE
:10DA1000E360FFF747B872B694E80C001078197805
:10DA2000637A227A194202EA000200F03E81A37A68
:10DA300003F003030AB143F0040343F008039A1010
:10DA4000082BA27200F27D81072B80F0F384032B58
:10DA500000F0E58440F20586042B00F07D81062B62
:10DA60007FF408A8E368023BE360FFF704B872B6EE
:10DA700094E80C0010781978637A227A194202EA45
:10DA8000000200F00981A37A03F003030AB143F016
:10DA9000040343F008039A10082BA27200F23181AC
:10DAA000072B80F06085032B00F0A58440F2AC8545
:10DAB000042B00F03181062B7FF4F1A8E368023BD0
:10DAC000E360FFF7EDB872B694E80C0010781978AF
:10DAD000637A227A194202EA000200F0C280A37A35
:10DAE00003F00303002A41F03B8143F008039A103E
:10DAF000082BA27200F23581072B80F0AB83032B39
:10DB000000F09D8440F2B585042B00F03581062B92
:10DB10007FF4B8A8E368023BE360FFF7B4B80322E0
:10DB20001A70FFF7ACBA72B694E80C001078197846
:10DB3000637A227A194202EA000200F0BD81A37AD8
:10DB400003F003030AB143F0040343F008039A10FF
:10DB5000082BA27200F2B981072B80F0E585032B18
:10DB600000F0E78540F2FC85042B00F0B981062B1C
:10DB70007EF48AAFE368023BE360FEF786BF72B6CD
:10DB800094E80C0010781978637A227A194202EA34
:10DB9000000200F02E81A37A03F003030AB143F0E0
:10DBA000040343F008039A10082BA27200F29D812F
:10DBB000072B80F0A385032B00F0A58540F2D785C5
:10DBC000042B00F09D81062B7FF44FA8E368023BF5
:10DBD000E360FFF74BB80D2B3FF497AD0E2B7EF4AF
:10DBE000A6AFD8F80C300133C8F80C30FEF7A1BF4F
:10DBF000D8F80C300233C8F80C30FEF79ABF40F664
:10DC0000EC52C2F201020721FFF76EBB4FF6104241
:10DC1000C2F2000205211278197072B69300FFF764
:10DC2000A9BA0023C7F6FF73ECE50023C7F6FF731C
:10DC3000D36100E40023C7F6FF73FFF7CEBB196A78
:10DC40008E4540F27681DA8BC3F820E0824238BFFD
:10DC5000D88364E6012BC4D0022B3FF456ADFEF707
:10DC600066BFA37A03F00303002A3FF440AF43F0FA
:10DC700004033CE7A37A03F00303002A3FF4B3AEA6
:10DC800043F00403AFE6A37A03F00303002A3FF452
:10DC90007EAE43F004037AE6A37A03F00303002A7E
:10DCA0003FF4F9AE43F00403F5E6A37A03F003036F
:10DCB000002A3FF4C4AE43F00403C0E64DF670639F
:10DCC000C2F200031A79002A40F0ED8472B6E260D5
:10DCD00062B6FFF7F3B972B60023E36062B6FFF7EE
:10DCE000EABB0C2B00F0B08300F27A83092B3FF4DF
:10DCF00061AE0B2B7EF4AFAFE368013BE360FEF750
:10DD0000ABBF0C2B00F0778300F22784092B3FF484
:10DD1000D5AE0B2B7EF4C3AFE368013BE360FEF7A7
:10DD2000BFBF0C2B00F0248400F24F83092B3FF47B
:10DD30006DAE0B2B7EF4B5AEE368013BE360FEF7FE
:10DD4000B1BE0C2B00F06B8300F26E83092B3FF405
:10DD500089AE0B2B7EF48EAEE368013BE360FEF7E9
:10DD60008ABE0C2B00F06B8300F26E82092B3FF40D
:10DD7000D1AE0B2B7EF486AFE368013BE360FEF788
:10DD800082BF72B60023E36062B6FFF721B872B6B5
:10DD90000023E36062B638E472B658F80C2C63686E
:10DDA00010781978637A227A194202EA000200F0A8
:10DDB000ED83A37A03F00303002A40F0E58743F0E4
:10DDC00008039A10082BA27200F2F283072B80F04E
:10DDD0005586032B00F03B8640F23286042B00F080
:10DDE000F283062B7FF4C9A8E368023BE360FFF7E8
:10DDF000C5B8A37A03F00303002A3FF4D4AE43F07E
:10DE00000403D0E672B658F80C2C636810781978C1
:10DE1000637A227A194202EA000200F0AE83A37A02
:10DE200003F003030AB143F0040343F008039A101C
:10DE3000082BA27200F20584072B80F04186032B89
:10DE400000F0338640F22A86042B00F00584062B6E
:10DE50007FF40CAAE368023BE360FFF708BA72B6EE
:10DE600058F80C2C636810781978637A227A194272
:10DE700002EA000200F09383A37A03F003030AB1DD
:10DE800043F0040343F008039A10082BA27200F237
:10DE9000C283072B80F0FD85032B00F0E48540F260
:10DEA000DB85042B00F0C283062B7FF4B8A9E3685E
:10DEB000023BE360FFF7B4B9A37A03F00303002A3F
:10DEC0003FF445AE43F0040341E60C2B00F03184EF
:10DED00000F22484092B3FF44DAE0B2B7EF4D4AD1D
:10DEE000E368013BE360FEF7D0BD0C2B00F00B8430
:10DEF00000F2FE83092B3FF469AE0B2B7EF4B5AE26
:10DF0000E368013BE360FEF7B1BE72B60023E36055
:10DF100062B6B9E472B60023E36062B6FFF729BACD
:10DF200001204FF0000EE9E472B60023E36062B610
:10DF30003AE49107C3F820E006D5596A7F31C90950
:10DF40000131884238BF0846510706D5996A7F31AA
:10DF5000C9090131884238BF0846110706D5D96A78
:10DF60007F31C9090131884238BF0846D10606D53C
:10DF7000196B7F31C9090131884238BF08469106C3
:10DF800006D5596B7F31C9090131884238BF08462F
:10DF9000510606D5996B7F31C9090131884238BFD6
:10DFA0000846D20906D0DA6B7F32D209013290429C
:10DFB00038BF1046D883B2E40023C8F20103FFF74C
:10DFC0000CBA0023C8F201031CE40023C8F20103C9
:10DFD000FFF731BA0023C8F20103FFF717BA0EF1B9
:10DFE0007F00C009013089E472B694E80C00107813
:10DFF0001978637A227A194202EA000240F0BE835D
:10E00000A37A03F00303002A40F0C2869A10082B7B
:10E01000A27200F21284072B80F01086032B00F00E
:10E02000DC8540F2D385042B00F01284062B7FF4AC
:10E030002BA8E368023BE360FFF727B872B694E8C9
:10E04000060091F800E01078627A217A10420EEA18
:10E05000010140F07383A27A02F00302002940F02C
:10E0600083869110082AA17200F2F783072A80F0B4
:10E07000CF85032A00F0358640F22C86042A00F072
:10E08000F783062A7FF41FA8E268023AE260FFF7EE
:10E090001BB872B694E80C0010781978637A227A6B
:10E0A000194202EA000240F05283A37A03F003030C
:10E0B000002A40F05D869A10082BA27200F270834D
:10E0C000072B80F07285032B00F07B8540F2728570
:10E0D000042B00F07083062B7FF4F2A9E368023B67
:10E0E000E360FFF7EEB972B694E80C001078197887
:10E0F000637A227A194202EA000240F04883A37A46
:10E1000003F00303002A40F047869A10082BA272FE
:10E1100000F26E83072B80F0B185032B00F023857E
:10E1200040F21985042B00F06E83062B7FF4A4A91E
:10E13000E368023BE360FFF7A0B972B658F80C2C15
:10E14000636810781978637A227A194202EA000229
:10E1500000F04583A37A03F003030AB143F00403FC
:10E1600043F008039A10082BA27200F22384072BB5
:10E1700080F0C084032B00F0C98440F2C084042BDB
:10E1800000F02384062B7FF414AAE368023BE360CB
:10E19000FFF710BA72B658F80C2C6368107819782B
:10E1A000637A227A194202EA000200F00F83A37A0E
:10E1B00003F003030AB143F0040343F008039A1089
:10E1C000082BA27200F2CD83072B80F07385032BFE
:10E1D00000F0658540F25C85042B00F0CD83062BB2
:10E1E0007FF4C8A9E368023BE360FFF7C4B972B6E5
:10E1F00058F80C2C636810781978637A227A1942DF
:10E2000002EA000200F00A83A37A03F003030AB1D2
:10E2100043F0040343F008039A10082BA27200F2A3
:10E220004583072B80F0AA84032B00F0B38440F2CF
:10E23000AA84042B00F04583062B7EF4C4ACE3686B
:10E24000023BE360FEF7C0BC0D2B3FF495AD0E2BF7
:10E250007EF418ADE3680133E360FEF714BD72B6D7
:10E2600094E80C0010781978637A227A194202EA4D
:10E27000000200F0BF83A37A03F00303002A40F0FA
:10E280007B8543F008039A10082BA27200F2A28348
:10E29000072B80F04684032B00F0F58440F226859E
:10E2A000042B00F0A283062B7FF49BA9E368023BBA
:10E2B000E360FFF797B972B62046FBF7B7FEFEF7AB
:10E2C000A9BD72B694E80C0010781978637A227AA6
:10E2D000194202EA000200F0D082A37A03F003039D
:10E2E000002A40F04D8543F008039A10082BA272D3
:10E2F00000F2CC82072B80F07B84032B00F07D841E
:10E3000040F20A85042B00F0CC82062B7EF472AD1D
:10E31000E368023BE360FEF76EBD72B694E80C0062
:10E3200010781978637A227A194202EA000200F022
:10E330003883A37A03F003030AB143F0040343F0E4
:10E3400008039A10082BA27200F21B83072B80F09F
:10E350008584032B00F0878440F2D084042B00F0E6
:10E360001B83062B7EF439ADE368023BE360FEF7C6
:10E3700035BD72B694E80C0010781978637A227A69
:10E38000194202EA000200F0E382A37A03F00303D9
:10E390000AB143F0040343F008039A10082BA27259
:10E3A00000F2C682072B80F03E84032B00F04B84E2
:10E3B00040F2AB84042B00F0C682062B7EF4F4AC52
:10E3C000E368023BE360FEF7F0BC0D2B3FF4B4AC16
:10E3D0000E2B7EF466ABE3680133E360FEF762BBAD
:10E3E0000D2B3FF489AC0E2B7EF435ACE368013382
:10E3F000E360FEF731BCE3680233E360FEF750BC34
:10E4000072B60022E26062B61A790132D2B21046C8
:10E410001A71029302F078F8029BFEF74FBEE36890
:10E420000233E360FEF727BB0D2B3FF495AC0E2BB8
:10E430007EF420ABE3680133E360FEF71CBBE368C6
:10E440000233E360FEF71FBCE3680233E360FEF7CC
:10E4500003BC72B694E80C0010781978637A227ABB
:10E46000194202EA000200F0CE82A37A03F003030D
:10E470000AB143F0040343F008039A10082BA27278
:10E4800000F22482072B80F05783032B00F059837E
:10E4900040F25184042B00F02482062B7FF4C7A89D
:10E4A000E368023BE360FFF7C3B872B694E80C0080
:10E4B00010781978637A227A194202EA000200F091
:10E4C0002E82A37A03F003030AB143F0040343F05E
:10E4D00008039A10082BA27200F29E82072B80F08C
:10E4E000FE82032B00F0F18240F22D84042B00F019
:10E4F0009C82062B7FF4ABA8E368023BE360FFF746
:10E50000A7B872B694E80C0010781978637A227A6A
:10E51000194202EA000200F0F981A37A03F0030332
:10E520000AB143F0040343F008039A10082BA272C7
:10E5300000F2DC81072B80F0C883032B00F00683F8
:10E5400040F2F283042B00F0DC81062B7FF462A8FA
:10E55000E368023BE360FFF75EB80D2B3FF4DCABF2
:10E560000E2B7EF49CABE3680133E360FEF798BBAF
:10E57000E3680233E360FEF795BAA37A03F003037E
:10E58000002A3FF454AC43F0040350E4A37A03F0B0
:10E590000303002A3FF415AC43F0040311E4A37A0B
:10E5A00003F00303002A3FF46FAC43F004036BE471
:10E5B0000C2B00F04C8200F25B82092B3FF414AC70
:10E5C0000B2B7EF4DAACE368013BE360FEF7D6BCCC
:10E5D000012B3FF40BAF022B3FF48EABFEF73BBB9E
:10E5E00072B62046FBF722FDFEF758BD012B3FF423
:10E5F000F2AE022B3FF4A0ABFEF753BA72B6204640
:10E60000FBF714FDFEF77BBE012BACD0022B3FF4D1
:10E6100083ABFEF744BB0C2B00F0258200F2338263
:10E62000092B3FF444AC0B2B7EF4F9ADE368013BBE
:10E63000E360FEF7F5BD72B62046FBF7F7FCFEF788
:10E64000A0BD0C2B00F0318200F23482092B3FF484
:10E6500001AC0B2B7EF40AAEE368013BE360FEF7EE
:10E6600006BE012B3FF4E6AE022B3FF475ABFEF77E
:10E6700001BA012B3FF4EEAD022B3FF47DABFEF768
:10E6800001BB72B62046FBF7D1FCFEF705BF72B6A0
:10E690002046FBF7CBFCFEF7AEBF72B62046FBF779
:10E6A000C5FCFFF76FB872B67C22E26062B61A79D9
:10E6B000013AABE672B62046FBF7B8FCFFF7E9B8C3
:10E6C00072B62046FBF7B2FCFFF7CCB872B6204614
:10E6D000FBF7ACFCFFF76DB872B62046FBF7A6FC63
:10E6E000FEF74CBE72B62046FBF7A0FCFEF72FBE2D
:10E6F0000D2B3FF405AC0E2B7EF4B7AAE368013373
:10E70000E360FEF7B3BAE3680233E360FEF7AEBA44
:10E7100072B62046FBF78AFCFEF750BB0D2B3FF488
:10E72000DFAB0E2B7EF4B0A9E3680133E360FEF7A4
:10E73000ACB9E3680233E360FEF7A7B9A27A02F04E
:10E74000030209B142F0040242F0080289E4A37A0C
:10E7500003F003030AB143F0040343F00803AAE4FF
:10E76000012BE1D0022B3FF4BBABFEF78DB9012B9F
:10E77000C4D0022B3FF4C4ABFEF777BAA37A03F000
:10E7800003030AB143F0040343F008033EE4A37A11
:10E7900003F003030AB143F0040343F00803B4E4B5
:10E7A0000C2B00F00E8200F2FA81092B3FF496AC9C
:10E7B0000B2B7EF485AEE368013BE360FEF781BE80
:10E7C00072B62046FBF732FCFEF7CBBDA37A03F00E
:10E7D0000303002A3FF4F3AC43F00403EFE4A37A0D
:10E7E00003F00303002A3FF4BDAC43F00403B9E493
:10E7F0000C2B00F0B88100F23B82092B3FF498AC5F
:10E800000B2B7EF439AEE368013BE360FEF735BEC7
:10E8100072B62046FBF70AFCFEF7BEBFA37A03F0F0
:10E820000303002A3FF4F8AC43F00403F4E472B6A7
:10E830002046FBF7FBFBFFF71FB80C2B00F0CD8148
:10E8400000F2F681092B3FF4F4AB0B2B7EF41CACE9
:10E85000E368013BE360FEF718BC0C2A00F041823C
:10E8600000F2D081092A3FF40FAC0B2A7EF42BACC6
:10E87000E268013AE260FEF727BCA37A03F00303E3
:10E88000002A3FF432AD43F004032EE50C2B00F0D8
:10E89000B48100F2A781092B3FF43AAD0B2B7EF433
:10E8A000A9AAE368013BE360FEF7A5BA0C2B00F0D0
:10E8B000718100F25D81092B3FF4C1AC0B2B7EF41A
:10E8C00082A9E368013BE360FEF77EB90C2B00F000
:10E8D000388100F22B81092B3FF4E2AD0B2B7EF443
:10E8E000A6AEE368013BE360FEF7A2BE0C2B00F08E
:10E8F0002D8100F2E481092B3FF42AAE0B2B7EF42C
:10E9000089AEE368013BE360FEF785BEA37A03F0BE
:10E910000303002A3FF409AE43F0040305E6A37A9B
:10E9200003F00303002A3FF4D4AD43F00403D0E521
:10E930000C2B00F0888100F27081092B3FF440AD70
:10E940000B2B7EF431AAE368013BE360FEF72DBA9E
:10E95000A37A03F00303002A3FF41FAD43F004033E
:10E960001BE50C2B00F09B8100F29E81092B3FF4EC
:10E9700039AC0B2B7EF4FEADE368013BE360FEF7A0
:10E98000FABD0C2B00F06F8100F26281092B3FF47D
:10E99000EBAC0B2B7EF421AAE368013BE360FEF7AE
:10E9A0001DBAA37A03F00303002A3FF4CAAC43F074
:10E9B0000403C6E40C2B00F0A98000F29580092B1B
:10E9C0003FF4E3AB0B2B7EF4F4ADE368013BE36073
:10E9D000FEF7F0BD0C2B00F0568100F29C80092B55
:10E9E0003FF464AC0B2B7EF4FCADE368013BE360C9
:10E9F000FEF7F8BDA37A03F00303002A3FF443AC0B
:10EA000043F004033FE4A37A03F00303002A3FF436
:10EA100034AD43F0040330E50C2B56D05AD8092B03
:10EA20003FF46AAD0B2B7EF412AEE368013BE3606A
:10EA3000FEF70EBE72B62046FBF7F8FAFEF77CBE74
:10EA4000012B1BD0022B3FF4BEADFEF796BAE36854
:10EA50000233E360FEF792BA012B1AD0022B3FF487
:10EA6000E5ADFEF7DCBBE3680233E360FEF7D8BB3D
:10EA70000D2B3FF4A8AD0E2B7EF47FAAE368013383
:10EA8000E360FEF77BBA0D2B3FF4D0AD0E2B7EF486
:10EA9000C6ABE3680133E360FEF7C2BB012B0FD0C6
:10EAA000022B3FF4D9ADFEF7E1BBE3680233E3602C
:10EAB000FEF7DDBB0D2B3FF4CFAD0E2B7EF4D6ABB6
:10EAC000E3680133E360FEF7D2BBE3680233E3603F
:10EAD000FEF7BEBD0D2BA8D00E2B7EF4B8ADE368BB
:10EAE0000133E360FEF7B4BD0D2B3FF46EAF0E2B88
:10EAF0007EF45FADE3680133E360FEF75BBD012B9D
:10EB0000F8D0022B3FF461AFFEF753BDE368023348
:10EB1000E360FEF74FBD0D2B3FF467AF0E2B7EF485
:10EB200060ADE3680133E360FEF75CBD0D2B3FF49D
:10EB3000D8AE0E2B7EF47BADE3680133E360FEF7C5
:10EB400077BDE3680233E360FEF772BDE36802332A
:10EB5000E360FEF760BD012B00F09080022B3FF4D4
:10EB600052AEFEF789BCE3680233E360FEF785BC72
:10EB70000D2B3FF4A6AE0E2B7EF425A8E3680133DF
:10EB8000E360FEF721B8012BF8D0022B3FF499AED9
:10EB9000FEF719B8E3680233E360FEF715B80D2BF2
:10EBA0003FF409AE0E2B7EF48BACE3680133E360D7
:10EBB000FEF787BC012BF8D0022B3FF4FCADFEF72B
:10EBC0007FBCE3680233E360FEF77BBC012B35D0EA
:10EBD000022B3FF43DAEFEF757BAE3680233E36021
:10EBE000FEF753BA0D2B3FF45CAE0E2B7EF402A958
:10EBF000E3680133E360FEF7FEB8E3680233E360E5
:10EC0000FEF7F9B80D2A3FF433AE0E2A7EF45BAA64
:10EC1000E2680132E260FEF757BA0D2B3FF493AE83
:10EC20000E2B7EF4C1A8E3680133E360FEF7BDB8A4
:10EC30000D2B3FF40DAE0E2B7EF426AAE3680133B4
:10EC4000E360FEF722BAE3680233E360FEF7ADB893
:10EC50000D2B3FF4A1AE0E2B7EF4BFA8E368013369
:10EC6000E360FEF7BBB8E3680233E360FEF7B6B8D3
:10EC70000D2B3FF4C8AD0E2B7EF4FEABE3680133E1
:10EC8000E360FEF7FABBE3680233E360FEF7AABC79
:10EC9000012B0FD0022B3FF46FAEFEF76BBCE36885
:10ECA0000233E360FEF767BC0D2B3FF465AE0E2B1D
:10ECB0007EF460ACE3680133E360FEF75CBC0D2BCF
:10ECC0003FF41FAE0E2B7EF4A5ACE3680133E36086
:10ECD000FEF7A1BC012A9BD0022A3FF4C9ADFEF782
:10ECE000F2B9E2680232E260FEF7EEB9012B3FF4BE
:10ECF00018AF022B3FF479AEFEF773BC012BADD0F9
:10ED0000022B3FF449AEFEF768B8012B8BD0022BE3
:10ED10003FF419AEFEF748B8012B3FF469AF022B60
:10ED20003FF4BFADFEF766B8012BCED0022B3FF407
:10ED3000E8ADFEF76FBC012B3FF4FEAE022B3FF4B3
:10ED4000D0ADFEF774BC012B3FF4C9AE022B3FF4EB
:10ED50006CAEFEF77CBC0023C7F6FF73FEF76BBBFF
:10ED600043F00403FEF7C1BE42F00402FFF779B995
:10ED700043F00403FFF79FB943F00403FFF781BAA0
:10ED800043F00403FFF7AFBA43F00403FFF717B8EB
:10ED900043F00403FFF73AB943F00403FFF7B5B9B2
:10EDA0002DE9F0432DED028B0446002683B000F1DF
:10EDB000B405284684F89D6084F89E6084F89F60BE
:10EDC00084F8A06084F8A16084F8A26084F8A3604D
:10EDD00084F8A46084F8A56084F8A66084F8A7602D
:10EDE00084F8A86084F8A96084F8AA6084F8AB600D
:10EDF00084F8AC6084F8906084F8916084F8926044
:10EE00000191FAF7ADFE43F65411AD22C0F20201B2
:10EE100004F598700BF072F90B2384F8DD3102F0E1
:10EE2000C9FE02F017FF03F0DDFBDDED017AB8EE5D
:10EE3000E78AA046B0EE480A03F0D4F9B0EE480ADB
:10EE400003F01CFAB0EE480A03F0F8FAB0EE480AF4
:10EE500002F0B2FC01992846FAF78AFE4FF40970D5
:10EE60000BF090FB0546F1F70BFBC4F820524FF472
:10EE700009700BF087FB42F67853C0F2020303607F
:10EE8000C4F824024FF409700BF07CFB43F62853BE
:10EE9000C0F20203C4F81C02036004F18409254691
:10EEA0004FF425700BF06EFB07460C3501F010FF98
:10EEB00045F8047C05F80A6C05F8096C05F8086C3F
:10EEC000A9454FF00003EBD194F89D209FEDD26A45
:10EED000DFEDD26A84F8DE3107EE902AB8EEE77AE9
:10EEE00094F89F20C4F8883067EE067A0B2067EE0E
:10EEF000A67A4FF40051FCEEE77AC4F88C30CDEDE1
:10EF0000017A84F8963084F8953084F8943084F847
:10EF1000933084F8923084F8913084F8903084F8FB
:10EF2000DD019DF80430C4F884100AB184F89030F3
:10EF300094F89E200AB184F8913094F8A0200AB188
:10EF400084F8923094F8A5309FEDB36ADFEDB36A90
:10EF500094F8A71007EE903AB8EEE77A67EE067AD3
:10EF600067EEA67AFCEEE77ACDED017A9DF80430E3
:10EF700031B194F89010994238BF194684F8901036
:10EF800094F8A61031B194F89110994238BF1946FF
:10EF900084F8911094F8A80030B194F892108B4244
:10EFA00038BF0B4684F8923094F8A1309FED9A6AEE
:10EFB000DFED9A6A94F8A31007EE903AB8EEE77A7C
:10EFC00067EE067A67EEA67AFCEEE77ACDED017A77
:10EFD0009DF8043031B194F89010994238BF194629
:10EFE00084F8901094F8A21031B194F891109942DD
:10EFF00038BF194684F8911094F8A41031B194F8F0
:10F000009250AB4238BF2B4684F8923094F8A93026
:10F010009FED816ADFED816A94F8AB5007EE903A7C
:10F02000B8EEE77A67EE067A67EEA67AFCEEE77A44
:10F03000CDED017A9DF8043035B194F890509D42A1
:10F0400038BF1D4684F8905094F8AA5035B194F812
:10F0500091509D4238BF1D4684F8915094F8AC50B1
:10F0600035B194F89260B34238BF334684F8923099
:10F070002AB921B918B915B97F2384F892303F23F2
:10F08000002584F89C30C4F8985004F2B91104F5B6
:10F09000017003F009F994F8E0310BB184F8E05104
:10F0A00094F8E231002584F8DF51002B00F0F7805E
:10F0B000D4F81C3284F8E251C4F8B03098F8043027
:10F0C0005BB1D8F8083088F80250184688F8045028
:10F0D00088F803500BB102F055FB08F10C08C1454C
:10F0E000ECD194F89D309FED4C6A94F89F1007EE98
:10F0F000903A94F89630B8EEE77A06EE903A67EEDA
:10F10000067AF8EEE66A002267EEA67A84F8922084
:10F11000FCEEE77A84F89120CDED017A9DF8043079
:10F1200084F8902009B184F8903094F89E200AB1B8
:10F1300084F8913094F8A0200AB184F8923094F8C1
:10F14000A5309FED356A94F8A71007EE903A94F831
:10F150009430B8EEE77A06EE903A67EE067AF8EE6B
:10F16000E66A67EEA67AFCEEE77ACDED017A9DF8C5
:10F17000043031B194F89010994238BF194684F8A0
:10F18000901094F8A61031B194F89110994238BFBC
:10F19000194684F8911094F8A80030B194F89210B0
:10F1A0008B4238BF0B4684F8923094F8A1309FED23
:10F1B0001A6A94F8A31007EE903A94F89530B8EED6
:10F1C000E77A06EE903A67EE067AF8EEE66A67EEC0
:10F1D000A67AFCEEE77ACDED017A9DF8043031B1E4
:10F1E00094F89010994238BF194684F8901094F81A
:10F1F000A21031B194F89110994238BF194684F8A1
:10F20000911094F8A41069B194F89250AB4238BFB1
:10F210002B4684F8923005E00AD7233C000000001A
:10F220000AD7233C94F8A9301FED036A94F8AB5039
:10F2300007EE903A94F89330B8EEE77A06EE903AFB
:10F2400067EE067AF8EEE66A67EEA67AFCEEE77AF3
:10F25000CDED017A9DF8043035B194F890509D427F
:10F2600038BF1D4684F8905094F8AA5035B194F8F0
:10F2700091509D4238BF1D4684F8915094F8AC508F
:10F2800035B194F89260B34238BF334684F8923077
:10F290002AB921B918B915B97F2384F892302046CC
:10F2A00003B0BDEC028BBDE8F08300BF2DE9F04F49
:10F2B0002DED028B8B00CDB00A3302AF23F0070394
:10F2C0007961ADEB030D90F8E1117A6002AB06466F
:10F2D0003B6139B390F8DD31DBB1002400F598755E
:10F2E00003E00134A4B2A34213D904EB440206EBB9
:10F2F000820108790028F4D04B78886816F822201B
:10F30000294602F005F8013496F8DD31A4B2A34293
:10F31000EBD806F2B91106F5017002F0C5FF002323
:10F3200086F8E1317B69002B00F0AB8007F12708FC
:10F330004FF6144406F501739FED588ABB6028F020
:10F340000F08C2F200044FF0000A3B694FF48072CC
:10F3500003EB8A090021404613F06AF800214FF4BC
:10F360008072484613F064F8BD68284602F0DEFF5C
:10F370008346284603F034F896F8DD11002955D06D
:10F38000C7F80CA00025824603E00135EDB28D429E
:10F390004AD205EB450306EB83031A79002AF4D021
:10F3A000986806F1840300935A465346414601F09B
:10F3B00067FEA8F1040308F1FC0E4A46F7EE006A66
:10F3C000BFEE006A00200DE0216801312160B7EE38
:10F3D000007AD2ED007A186037EE877A7345A2EC96
:10F3E000017A1BD053F8041F091121F3572149104A
:10F3F00007EE901AF8EEE77A87EE887AB4EEE67AAE
:10F40000F1EE10FAE0DCB4EEC67AF1EE10FAE0D5D7
:10F41000216801312160BFEE007ADAE796F8DD114C
:10F420000135EDB28D42B4D3D7F80CA07B690AF157
:10F43000400A1FFA8AFA534587D83C691D4606F1EF
:10F44000B4001A462146FAF715FC7A689FED137A44
:10F45000681E80B202EB40002146023AF1EC017ACC
:10F4600067EE877AFDEEE77A17EE903A22F8023FD0
:10F470008242F3D107F59677BD46BDEC028BBDE81D
:10F48000F08F39691A4606F1B400FAF7F3FB07F575
:10F490009677BD46BDEC028BBDE8F08F00FEFF46BF
:10F4A0002DE9F843064690F8C03190F8DD51002A66
:10F4B00000F0B080183BCF1890F8DE81FFB2002D2D
:10F4C00000F09F804FEA480909EB080300EB830333
:10F4D00041469C78CE46002C6ED0002402E0837812
:10F4E000002B69D00131013491FBF5F305FB1311B9
:10F4F000E4B24FEA410E0EEB0100AC4206EB800095
:10F500005FFA81F8EBD196F8E031002B4BD096F8FA
:10F51000DD31002B47D03279002A40F06281012B87
:10F5200041D9327C002A40F05E81022B3BD0327FF1
:10F53000002A40F06281032B35D096F82820002A5B
:10F5400040F05D81042B2ED096F83420002A40F044
:10F550004C81052B27D096F84020002A40F04781A7
:10F56000062B20D096F84C20002A40F04281072B31
:10F5700019D096F85820002A40F03D81082B12D06F
:10F5800096F86420002A40F03C81092B0BD096F8B5
:10F590007020002A40F037810A2B04D096F87C3086
:10F5A000002B40F0E9804FEA4809C84406EB880682
:10F5B00001233371BDE8F8838E444FEA8E0E01318A
:10F5C00006EB0E0991FBF5F305FB131586F8DE51EA
:10F5D00006F80E7089F8012096F8DF3189F80330BB
:10F5E0000121134689F80210D9F808003A4606F5B9
:10F5F000987101F087FB96F8B831002B53D1002C9D
:10F6000081D106F5017002F011FF96F8E031002B70
:10F61000C9D07CE7183BCF18FBB2002D41D0017850
:10F6200099427BD0012D3CD9327B9A4271D0022D78
:10F6300037D0327E9A4267D0032D32D096F82420FC
:10F640009A425BD0042D2CD096F830209A424FD0AD
:10F65000052D26D096F83C209A4243D0062D20D086
:10F6600096F848209A4237D0072D1AD096F85420A1
:10F670009A422BD0082D14D096F860209A421FD0C1
:10F68000092D0ED096F86C209A4213D00A2D08D07E
:10F6900096F878209A4204D196F87A30002B40F000
:10F6A0008280BDE8F883D9F8080002F06BF8002CDE
:10F6B000A7D028E796F86E20002AE7D0092773E044
:10F6C00096F86220002ADBD008276DE096F85620D5
:10F6D000002ACFD0072767E096F84A20002AC3D037
:10F6E000062761E096F83E20002AB7D005275BE0A8
:10F6F00096F83220002AABD0042755E096F8262051
:10F70000002A9FD003274FE0B27E002A94D0022720
:10F710004AE0B27B002A8AD0012745E0817800299F
:10F7200080D082701746804696F8E031E3B14FF002
:10F73000000E734671464FF0FF3203EB430306EBB6
:10F740008304481CA4782CB116F823309342C4BF1C
:10F750005AB28E4641B2A9420B46EEDB013203D0CB
:10F7600098F80430002B50D196F8DF3183B3012391
:10F7700088F80330BDE8F8830A2303EB43039B00BA
:10F78000F2189178C1B1F35CBB428AD24FEA4809C2
:10F7900009EB080306EB8303002111719868916857
:10F7A00001F09CFF01E70A2707EB470806EB8808F2
:10F7B000002388F80230B7E74FEA480909EB08034D
:10F7C00006EB830311719868916801F0A7FFECE6DE
:10F7D00007EB470206EB8206B068BDE8F84301F08C
:10F7E00083BD0023C9E70123C7E70423C5E7052339
:10F7F000C3E70623C1E70723BFE70223BDE70323CF
:10F80000BBE70823B9E70923B7E70EEB4E0E07EB7A
:10F81000470206EB8E03002106EB820288F80410F3
:10F82000012119719868916801F058FF9CE700BFA9
:10F83000F8B590F8C03190F8DD41183B1944002C20
:10F8400040D00378C9B28B423DD0012C3AD9037B1A
:10F850008B4200F09D80022C34D0037E8B4200F05E
:10F860009180032C2ED090F824308B4200F08380BE
:10F87000042C27D090F830308B4276D0052C21D044
:10F8800090F83C308B426AD0062C1BD090F8483060
:10F890008B425ED0072C15D090F854308B4252D05A
:10F8A000082C0FD090F860308B4246D0092C09D03C
:10F8B00090F86C308B423AD00A2C03D090F8783014
:10F8C0008B422ED0F8BD8378002BBED000258570EA
:10F8D000064690F8E0310746E3B100231A469C46FD
:10F8E0004FF0FF3E03EB430307EB8300511C80788E
:10F8F00030B117F823307345C4BF4FFA83FE9446E6
:10F900004AB2A2421346EDDBBEF1FF3F02D033798B
:10F91000002B52D197F8DF31002B45D00123F37033
:10F92000F8BD90F87A30002BCCD00A2535E090F85D
:10F930006E30002BC0D009252FE090F86230002BEC
:10F94000B4D0082529E090F85630002BA8D0072520
:10F9500023E090F84A30002B9CD006251DE090F85B
:10F960003E30002B90D0052517E090F83230002B68
:10F9700084D0042511E090F82630002B3FF478AFB6
:10F9800003250AE0837E002B3FF46BAF022504E0E1
:10F99000837B002B3FF45FAF012505EB450600EBB1
:10F9A00086060023B37094E705EB450507EB850059
:10F9B000BDE8F840806801F097BC0CEB4C0C05EBFF
:10F9C000450207EB8C03002107EB82023171012114
:10F9D00019719868916801F081FE9BE7012380F816
:10F9E000E131704790F8E0318B4218BF80F8E011A8
:10F9F000704700BF90F8DF318B4218BF80F8DF11ED
:10FA0000704700BF90F8DF01704700BF70B5044633
:10FA100000F18406002523793BB1A368A570184640
:10FA20002571E5700BB101F0ADFE0C34B442F2D19A
:10FA300070BD00BF90F89D309FED6C6ADFED6C6A81
:10FA400090F89F1007EE903AB8EEE77A70B467EE40
:10FA5000067A83B067EEA67A0023FCEEE77A4FF4CD
:10FA60000052CDED017AC0F88420C0F888309DF8AE
:10FA70000420C0F88C3080F8963080F8953080F8FB
:10FA8000943080F8933080F8923080F8913080F88C
:10FA9000903009B180F8902090F89E300BB180F83A
:10FAA000912090F8A01009B180F8922090F8A5302C
:10FAB0009FED4E6ADFED4E6A90F8A72007EE903A70
:10FAC000B8EEE77A67EE067A67EEA67AFCEEE77A9A
:10FAD000CDED017A9DF8043032B190F890209A4231
:10FAE00038BF1A4680F8902090F8A62032B190F8DE
:10FAF00091209A4238BF1A4680F8912090F8A84089
:10FB000034B190F89220934238BF134680F8923077
:10FB100090F8A1309FED356ADFED356A90F8A320AB
:10FB200007EE903AB8EEE77A67EE067A67EEA67AC5
:10FB3000FCEEE77ACDED017A9DF8043032B190F811
:10FB400090209A4238BF1A4680F8902090F8A22060
:10FB500032B190F891209A4238BF1A4680F891202D
:10FB600090F8A42032B190F89250AB4238BF2B46A7
:10FB700080F8923090F8A9309FED1C6ADFED1C6A86
:10FB800090F8AB5007EE903AB8EEE77A67EE067A57
:10FB900067EEA67AFCEEE77ACDED017A9DF80430A7
:10FBA00035B190F890509D4238BF1D4680F8905076
:10FBB00090F8AA5035B190F891509D4238BF1D463B
:10FBC00080F8915090F8AC5035B190F89260B34203
:10FBD00038BF334680F8923029B922B91CB915B91B
:10FBE0007F2380F8923003B070BC70470AD7233C63
:10FBF00000000000037913B18378002B60D1037CEF
:10FC000013B1837B002B58D1037F13B1837E002B6C
:10FC100050D190F828301BB190F82630002B45D1F8
:10FC200090F8343013B190F83230DBBB90F84030AC
:10FC300013B190F83E308BBB90F84C3013B190F874
:10FC40004A303BBB90F8583013B190F85630EBB9BE
:10FC500090F8643013B190F862309BB990F870302E
:10FC600013B190F86E304BB990F87C302BB190F80E
:10FC70007A3013B1002380F87A307047002380F87F
:10FC80006E30F1E7002380F86230E7E7002380F868
:10FC90005630DDE7002380F84A30D3E7002380F8B0
:10FCA0003E30C9E7002380F83230BFE7002380F8F8
:10FCB0002630B5E700238376ABE700238373A3E701
:10FCC000002383709BE700BF90F8DD01704700BF01
:10FCD0002DE9F04F054690F8B611D0F8B00085B088
:10FCE00002F0F4F895F8DD11002900F0C780C0F3A8
:10FCF000C0030093C0F3001300260193C0F3401328
:10FD0000344600F00108C0F3400BC0F3800A0293B0
:10FD100005F5F27703E00134E4B2A1427CD904EBAB
:10FD2000440305EB830999F80420002AF3D000214D
:10FD30002022384612F07CFB3946D9F8080001F041
:10FD40008FFCB8F1000F6BD0D5F8E41140F22D42D2
:10FD5000914269D895F8FC11A1F10401B1FA81F141
:10FD6000022049090122BBF1000F0AD0D5F8E82191
:10FD700040F22D4E724503D895F8FD21042A57D044
:10FD80000246BAF1000F0DD0D5F8EC0140F22D4E2D
:10FD900001327045D2B205D895F8FE01042804BF9F
:10FDA0000131C9B2009B6BB1D5F8F00140F22D4E84
:10FDB00001327045D2B205D895F8FF01042804BF7E
:10FDC0000131C9B2019B6BB1D5F8F40140F22D4E5F
:10FDD00001327045D2B205D895F80002042804BF5C
:10FDE0000131C9B2029B6BB1D5F8F80140F22D4E3A
:10FDF00001327045D2B205D895F80102042804BF3B
:10FE00000131C9B2914217D095F8DD110134E4B245
:10FE10000136A142F6B282D8304605B0BDE8F08F77
:10FE20000120424641469EE70220012200219AE736
:10FE30000131C9B20246A4E7002243F6042089F842
:10FE4000042089F8032089F802201021C0F2020062
:10FE500003920DF0B3FC039A4EF2002013462146A4
:10FE60000A22C2F2000009F037FE4EF20020C2F270
:10FE7000000009F01FFE95F8DD114CE70E46CBE7B8
:10FE80002DE9F04100F5987384B004460A4600F568
:10FE9000D775106856685E6018601089967A9E72F1
:10FEA0001881D07A00F00306C0F38100DE72187367
:10FEB000107BC0F3C30600F007001E755873507B1B
:10FEC000C0F3820600F00300DE739873907B187411
:10FED000D07BC0F3440600F001009E745874107C7F
:10FEE000D87415339D4202F11102D2D10B460A4655
:10FEF00053F8660FDFEDD75A5B68C4F8AE016B604C
:10FF000091F86E3003F01F0384F8B63191F86F302A
:10FF1000C3F3C00003F0070384F8B80184F8B731D5
:10FF20000B6FC4F8B93191F87430C3F30115C3F302
:10FF3000420003F0010384F8BF5184F8BE0184F845
:10FF4000BD3191F8753084F8C03152F8761F04F253
:10FF5000C1175368C4F8C1117B6013893B816322C8
:10FF60000123072184F8CB3184F8CC3184F8CD21EA
:10FF700084F8CF2184F8D12184F8D32184F8CE11DC
:10FF800084F8D01184F8D21184F8D41194F8941024
:10FF900084F8D63106EE101A94F8961084F8D7310A
:10FFA00006EE901A94F8951084F8D831B8EEC66A27
:10FFB000F8EEE66A07EE101A94F8931084F8D93137
:10FFC00026EE256A66EEA56A07EE901AB8EEC77AA5
:10FFD000BCEEC66AFCEEE66AF8EEE77A27EE257A12
:10FFE0008DED016ACDED026A9DF804009DF80810C0
:10FFF00084F8DA3167EEA57ABCEEC77A88428DEDD7
:020000021000EC
:10000000037AFCEEE77A38BF08469DF80C10CDED78
:10001000017A88429DF8045084F8DB3138BF0846E5
:10002000A842C4F88830C4F88C3084F89D2084F845
:100030009E3084F89F3084F8A03084F8A12084F8A2
:10004000A23084F8A33084F8A43084F8A52084F882
:10005000A63084F8A73084F8A83084F8A92084F862
:10006000AA3084F8AB3084F8AC30237938BF284606
:1000700000210B253F2284F8900084F8D511C4F8A4
:10008000981084F8DC5184F8910084F8920084F888
:100090009C201BB1A378002B40F08381237C1BB1F3
:1000A000A37B002B40F07A81237F1BB1A37E002B22
:1000B00040F0718194F8283023B194F82630002B59
:1000C00040F0658194F8343023B194F83230002B3D
:1000D00040F0598194F8403023B194F83E30002B21
:1000E00040F04D8194F84C3023B194F84A30002B05
:1000F00040F0418194F8583023B194F85630002BE9
:1001000040F0358194F8643023B194F86230002BCC
:1001100040F0298194F8703023B194F86E30002BB0
:1001200040F01D8194F87C3023B194F87A30002B94
:1001300040F011810B2384F8DD31254604F1840859
:1001400000262B793BB1AB68AE7018462E71EE706D
:100150000BB101F017FB0C354545F2D194F89D30F9
:100160009FED3D6A94F89F1007EE903A94F8963010
:10017000B8EEE77A06EE903A67EE067AF8EEE66AAF
:10018000002267EEA67A84F89220FCEEE77A84F8E3
:100190009120CDED017A9DF8043084F8902009B1CA
:1001A00084F8903094F89E20002A40F0148194F84E
:1001B000A0200AB184F8923094F8A5309FED266A09
:1001C00094F8A71007EE903A94F89430B8EEE77AD6
:1001D00006EE903A67EE067AF8EEE66A67EEA67AE1
:1001E000FCEEE77ACDED017A9DF8043031B194F858
:1001F0009010994238BF194684F8901094F8A610D0
:10020000002940F0E08094F8A81031B194F89200F1
:10021000834238BF034684F8923094F8A1309FEDB2
:100220000E6A94F8A30007EE903A94F89530B8EE71
:10023000E77A06EE903A67EE067AF8EEE66A67EE3F
:10024000A67AFCEEE77ACDED017A9DF8043060B134
:1002500004E000BFA3707D3F0AD7233C94F89000D0
:10026000984238BF184684F8900094F8A2000028FD
:1002700040F0A18094F8A40030B194F89250AB42C1
:1002800038BF2B4684F8923094F8A9301FED0E6ADF
:1002900094F8AB5007EE903A94F89330B8EEE77AC2
:1002A00006EE903A67EE067AF8EEE66A67EEA67A10
:1002B000FCEEE77ACDED017A9DF8043035B194F883
:1002C00090509D4238BF1D4684F8905094F8AA5033
:1002D000002D68D194F8AC5035B194F89260B342D7
:1002E00038BF334684F892302AB920B919B915B904
:1002F0007F2384F89230012540F650700A22394657
:1003000084F8E151C2F2010012F048FA43F61820D5
:100310000721C0F202000DF051FA40F65070C2F20F
:10032000010012F0CDF9014640F65070C2F2010012
:100330000DF044FA43F620200921C0F202000DF02E
:100340003DFA4EF20020C2F2000009F0B3FB28464D
:1003500004B0BDE8F081002384F87A30EAE6002397
:1003600084F86E30DEE6002384F86230D2E60023A3
:1003700084F85630C6E6002384F84A30BAE60023F3
:1003800084F83E30AEE6002384F83230A2E6002343
:1003900084F8263096E60023A3768BE60023A37329
:1003A00082E6A1707AE694F891509D4238BF1D46CE
:1003B00084F891508EE794F89100984238BF18461F
:1003C00084F8910056E794F89110994238BF194685
:1003D00084F8911017E784F89130E8E610B50446E8
:1003E00012F06EF901462046BDE810400DF0E6B966
:1003F00010B5044612F064F9014620460DF0DEF90E
:1004000004464EF20020C2F2000009F053FB2044E3
:1004100010BD00BF2DE9F04100262F270C468E604D
:100420000E604E60C1F80B600A2201F8017B804625
:1004300011F002FD204612F043F908EB48054FF693
:100440002442C2F2000208EB85051544431C2754E0
:100450002946E01812F0B8F84EF2002743F62C2097
:10046000C2F200072121C0F202000DF0A7F93346C5
:100470000A224146384609F02FFB43F650200A2154
:10048000C0F202000DF09AF9284612F019F901465F
:1004900028460DF093F943F26C500321C0F202009C
:1004A0000DF08CF9204612F00BF9014620460DF0B4
:1004B00085F943F24010C0F2020001210DF07EF9EF
:1004C0003846BDE8F04109F0F5BA00BF10B584B078
:1004D0000C460146684612F077F843F62821684634
:1004E000C0F2020112F08EF928B10146204612F046
:1004F0006BF804B010BD43F65C23C0F2020303CBDB
:100500002060616004B010BD2DE9F04194B0044654
:1005100004A804F083FB40F6F050C2F201004FF44F
:10052000B072002111F084FF40F63053C2F2010393
:100530001B7833B904A804F07FFB002014B0BDE899
:10054000F08148F21F53C5F2EB13A3FB04235B09B0
:10055000642000FB1340C0B26946FFF75BFF43F61F
:1005600064201E21C0F202000DF028F9684612F046
:10057000A7F8014668460DF021F943F24010012129
:10058000C0F202000DF01AF94EF20020C2F2000093
:1005900009F090FA48F2101101236A460CA8C2F241
:1005A000010104F017FC14AB9DF8344053F8131DFF
:1005B000CDF81D105A689E681D7B0E99CDF821203C
:1005C000139B9DF83C20CDF825600CA88DF8295090
:1005D0008DF8144006918DF81C200B9304F02CFB31
:1005E00004A804F043FB0028A4D004A804F03AFBBC
:1005F00041F2080398420DD043F684201A21C0F23C
:1006000002000DF0DBF84EF20020C2F2000009F00B
:1006100051FA8FE704A804F071FAF0280DD043F6E0
:10062000A0201F21C0F202000DF0C8F84EF20020F9
:10063000C2F2000009F03EFA7CE704A804F05EFA7A
:1006400043280DD043F6C0201C21C0F202000DF05B
:10065000B5F84EF20020C2F2000009F02BFA69E76B
:1006600041F2070104A804F0F3FA04A804F046FAE2
:10067000F72806D043F6E020C0F20200FFF7B8FEEC
:1006800058E7032104A804F0E3FA04A804F036FABA
:10069000092806D043F60030C0F20200FFF7A8FE9A
:1006A00048E741F2060104A804F0D2FA04A804F0D5
:1006B00025FA062146B204A804F0CAFA04A804F0F8
:1006C0001DFA002740F6F05502463C46B846C2F2F5
:1006D000010516E004F012FA04F07F0108EB88032C
:1006E00008EB43030246A1F1760009282B449CBF86
:1006F0005B1803F8762C7F2904BF08F101085FFA24
:1007000088F80134A4B2D2B2B4F5805F04A8A7EB94
:100710000207DFD143F62030C0F20200FFF75EFE91
:1007200007F07F074EF20020394600231022C2F264
:10073000000009F0D1F943F63430C0F20200FFF7AF
:100740004DFE4EF20020002310223146C2F200007E
:1007500009F0C2F943F24010C0F20200FFF748FE70
:10076000B7423FF4E7AE43F63C30C0F20200FFF779
:1007700035FE4EF20020394600231022C2F200005E
:1007800009F0AAF943F65C30C0F20200FFF726FE3A
:100790004EF20020314600231022C2F2000009F080
:1007A0009BF94EF20020C2F2000009F083F9C1E685
:1007B0002DE9F04192B002A804F030FA4FF624403F
:1007C000C2F2000040F21452002111F031FE40F656
:1007D0003053C2F201031C78002C00F09E804FF6CB
:1007E0002446C2F20006002408E00AA804F024FA15
:1007F00002A804F03BFA002800F08F802F23002588
:100800000A220DF10501204601958DF8043011F002
:1008100013FB48F21011C2F20101012301AA0AA838
:1008200004F0D8FA9DF82CE00C9D9DF834709DF8EA
:1008300036009DF837109DF838209DF839309DF826
:100840003AC09DF835808DF80CE004959DF83BE0AA
:100850008DF814709DF83D509DF83C708DF8160091
:100860008DF817109DF83E009DF83F108DF8182068
:100870008DF819309DF840209DF841308DF81F10FB
:100880008DF820208DF81AC08DF81BE08DF81E0021
:100890008DF815808DF81C708DF81D508DF8213065
:1008A0000AA8119B099304F0C7F902A804F0DEF925
:1008B000012202A988B30AA804F004FB0AA804F0E4
:1008C000BFF9002891D10AA804F0B8F904EB440557
:1008D00004EB850535440146284611F075FE43F6C4
:1008E00064300C21C0F202000CF068FF284611F0C1
:1008F000E7FE014628460CF061FF43F2401001215B
:10090000C0F202000CF05AFF4EF20020C2F20000CA
:10091000013409F0CFF8E4B267E702A804F08CF9DB
:10092000204612B0BDE8F0812DE9F0470E46904612
:10093000054604F097F941F2080398420FD043F6B8
:100940008420C0F202001A210CF038FF4EF2002081
:10095000C2F2000009F0AEF80020BDE8F08728469A
:1009600004F0CCF8F02805D043F6A020C0F2020035
:100970001F21E9E7284604F0C1F8432805D043F6D3
:10098000C020C0F202001C21DEE741F20701284628
:1009900004F05EF9284604F0B1F8F72805D043F6D4
:1009A000E020C0F202001D21CEE70321284604F01A
:1009B0004FF9284604F0A2F8092804D043F6003085
:1009C000C0F20200EFE741F20601284604F040F9C8
:1009D000284604F093F806214FFA80F9284604F0DF
:1009E00037F906F1010A00244FEACA1AF601274630
:1009F000284604F083F8B442C3B2A7EB030704DB34
:100A0000A31B5445B8BF08F803000134B4F5805F58
:100A1000EED143F620301221C0F202000CF0CEFEDF
:100A200007F07F074EF20020002310223946C2F261
:100A3000000009F051F843F634300421C0F20200FE
:100A40000CF0BCFE4EF20020002310224946C2F2F8
:100A5000000009F041F843F240100121C0F2020009
:100A60000CF0ACFE4EF20020C2F2000009F022F8B9
:100A70004F4508D14FF62043C2F2000300221A80EE
:100A80000120BDE8F08743F63C301F21C0F2020090
:100A90000CF094FE4EF20020394600231022C2F2E0
:100AA000000009F019F843F65C300621C0F202009C
:100AB0000CF084FE4EF20020494600231022C2F2C0
:100AC000000009F009F84EF20020C2F2000008F020
:100AD000F1FF0020BDE8F08730B540F63052C2F299
:100AE0000102B5B01378002B00F09C80044604A8E6
:100AF0000D4604F093F848F21F53C5F2EB13A3FB25
:100B000004235B09642000FB1340C0B26946FFF771
:100B100081FC48F2101101236A4614A8C2F20101B7
:100B200004F058F934AB9DF8544053F8732DCDF8C8
:100B30001D2059689A681B7BCDF82110CDF825201F
:100B400016999DF85C208DF8293014A81B9B8DF810
:100B5000144006918DF81C200B9304F06DF804A846
:100B600004F084F8044600BB43F674301021C0F250
:100B700002000CF023FE684611F0A2FD0146684613
:100B80000CF01CFE43F68830C0F2020008210CF085
:100B900015FE4EF20020C2F2000008F08BFF04A800
:100BA00004F04AF8204635B030BDDDF82130DDF8DC
:100BB0001D20CDF84130DDF82530CDF84530CDF899
:100BC0003D209DF82930069A8DF849300E929DF807
:100BD00014308DF8343044F2FC129DF81C308DF83E
:100BE0003C30C0F2020205F01F050B9B0C92294617
:100BF0000CA814AA1393FFF797FE04460CA804F060
:100C00001BF804BB43F6A4301A21C0F202000CF01A
:100C1000D5FD4EF20020C2F2000008F04BFF04A800
:100C200004F00AF843F6C0301321C0F202000CF0C1
:100C3000C5FD4EF20020C2F2000008F03BFF002488
:100C4000204635B030BD0A220DF1C6010CA811F0C6
:100C5000A5FD43F694300E21C0F202000CF0AEFD6B
:100C6000684611F02DFD014668460CF0A7FD43F2E1
:100C70008C600221C0F202000CF0A0FD05EB8503A0
:100C800040F6F05005EB4305C2F20100054428464A
:100C900011F016FD014628460CF090FD43F240107D
:100CA0000121C0F202000CF089FD4EF20020C2F2D8
:100CB000000008F0FFFE40F66453C2F2010314A9DD
:100CC0001868FFF7DDF8044669E700BF09F0F4B8DB
:100CD0000022C0F8A421C0F89C21C0F8B421C0F8BB
:100CE000AC21C0F8C421C0F8BC21C0F8D421C0F8A0
:100CF000CC21C0F8E421C0F8DC21C0F8F421C0F810
:100D0000EC2170472DE9F04F45F255541646C0F2DC
:100D1000150404FB06F49A4604F142732DED088B8A
:100D200008EE903A4FF04E530AEE103A4CF283031D
:100D3000CBF6CA6309EE903A43F27A63C3F6AB434B
:100D400009EE103A4DF20A73C3F623430BEE103A44
:100D50004AF63B23C4F6B83345F256550AEE903AAC
:100D600018EE903AC5F2555593B085FB022703F271
:100D700031733246A7EBE67743F61C4B08EE903A08
:100D80004FEA6A0303958146073F08930C460546E0
:100D9000C0F2020B0026099190464EE0BAF1000F16
:100DA00000F30F816FF0EE0101FB02F20732D21067
:100DB00000EB0213002F23EAE373627B40F3FF8012
:100DC0001F2FCCBFC2EB42127A43D21000920AA965
:100DD0000EAA09EB060000F007FD627CA37CE17C13
:100DE000207D002A7AD003F0030C4FF0640E40F609
:100DF00078031EFB0C11C0F2440303FB01F3072828
:100E00004FEAE301C3BF073843F291434343002352
:100E10000B44C5F86C22C5F83032A37B03F0030302
:100E200044365BF82330C5F85432B6F5CC7F04F174
:100E3000150405F1040500F0D4802078217962784A
:100E400063790A90A0780E910B92A179E2780F93C2
:100E50000C90E379207C0D921193109100F01EFE0E
:100E6000237AC3EB0803B3F1110200F18680039AE1
:100E7000217B94F80AE0103B82FB03C2A2EBE373F0
:100E800001B303291ED01F2BDBBF43F6AC42C0F2D7
:100E90000202FA23D35C03FB0EFE40F2491303FB6C
:100EA0000EF301294FEAE33316DD18447F28A8BF6B
:100EB0007F20BAF17F0F4FEA4010E27B7FF76EAFE1
:100EC0000F2171E703FB0EF340F2491202FB03F31B
:100ED00001294FEA2333E8DC5B42E6E7B8EEE88A13
:100EE000079028EE0A0A069120EE290A059304923B
:100EF0000DF0EEFE20EE090AF1EE0C7A80EE277A74
:100F00000798059B0699073843F62C4E03F01F03FC
:100F1000C0F2020E5EF8233007EE900A27EE087A40
:100F2000F8EEE77AA7EE278ABDEEC88A18EE102AF7
:100F30001A441346049A00293FF46BAF07EE901A47
:100F4000F8EEE77AB7EE000AA7EE8B0A05930DF0EC
:100F500041FFF6EE007AE0EE2A7A17EE900A10F0E2
:100F60007DFB41EC100B0DF08FF951EC100B10F0E4
:100F700079FE059B049A03444BE7039B94F809C050
:100F8000C2F10101E27A83FB013EAEEBE17102B3F3
:100F9000032A1ED01F29DBBF43F6AC4EC0F2020E5F
:100FA000FA211EF8011040F2491301FB0CF103FB7A
:100FB00001F3DB13012A3FF778AF5B4275E70022AC
:100FC00004E743F6D433C0F202030899595CEF39C1
:100FD000EAE601FB0CF140F2491303FB01F31B139A
:100FE000E8E7DDF8248098F87E5098F8824098F879
:100FF0007F3098F8830098F880600A950E9498F8EE
:10100000845098F881400B930F9098F88530119395
:101010000EAA0AA909F5FC700C9610950D9401F022
:1010200029FA98F88630C9F8883298F887302BB3B7
:10103000C3F10803C9F8503298F88B3003EB8303EF
:1010400003EB43139B11C9F88C3298F88F3043F6A9
:101050001442C0F2020203F00703D35CC9F89032D5
:1010600098F88C3003EB830303EB43139B11C9F80F
:10107000843213B0BDEC088BBDE8F08F1023D9E7A4
:101080002DE9F04F2DED048B89B0D0F89052DDF8AA
:10109000588007918146D0F88C0298F80DE09B4665
:1010A000A2F5000305FB03F500FB0BF0A0FB0567B1
:1010B000EB1700FB037714468EFB0523900B40EAE9
:1010C0008340FE1186EAE67380EAE072A2EBE072EA
:1010D000A3EBE6739342B8BF134609F5FC701E46B6
:1010E00001F000FAD8F80030002DB4BF4FF0FF3205
:1010F0000122B3F5005A06FB02001AD0D8F80820E6
:10110000002A40F0D980D8F804304FEACA2A07EE06
:1011100090AA07EE103AF8EEE77AB8EEC77AF2EE48
:10112000086A67EE877A87EEA67AFDEEC77A17EE31
:1011300090AA4FF05A5309EE103A45F62943C3F6E8
:101140008F53D9F8842298F80C1008EE903A43F2A5
:101150003333C4F2431308EE103A82FB0B23C4F17D
:1011600080744FEA122B4BEA036BE3170BFB03F27D
:1011700098F80E30002704FB07225B04ABFB0467E2
:1011800081FB0445C3F57E0BE30943EA45635B45F8
:1011900017444FEA166138BF5B4641EA0721D8F889
:1011A00014208B4238BF0B4692449B4600EB0A0347
:1011B00005934E4609F50C744F46002514E0504443
:1011C00001F040F8C6F8A001384600F065FB626AFD
:1011D00002BBC6F898010135062D07F1440706F158
:1011E000100604F1040452D098F818302B4113F083
:1011F000010344D0E36B2068002BE0D1059B184429
:1012000001F020F8C6F8A001384600F045FB626AFC
:10121000002ADED0D117ABFB0223CDE90223039ACB
:1012200006900BFB01230393DDE90201020E42EA63
:10123000012207EE902AF8EE677AB0EE480A67EED0
:10124000897AA7EEA80A0DF043FDFCEEC07A069855
:1012500017EE901AC3174FEA011E0EFB03F3090F96
:1012600000FB0131AEFB0023CDE902230B440393C5
:10127000029B1A0F039B42EA0312801AA9E7384621
:10128000029300F009FB029BC6F89831A3E7D8F857
:101290002C00D9F850120268D9F88832019109F56A
:1012A000127100919468079909F5CC72A04709B0B2
:1012B000BDEC048BBDE8F08F21230C21C8F20403A0
:1012C00091FBF2F202FB0AFA83FB0A1353444FEA42
:1012D000EA7ACAEB233A41F6FF7393FBF2F303FB7E
:1012E0000AFA4FEACA2A24E770B50646044600F512
:1012F000CC7520460021443400F080FBAC42F8D18C
:1013000006F5FC700021BDE8704001F039B900BF5E
:101310002DE9F04F45F255549246C0F2150404FBF6
:101320000AF4994604F142732DED088B08EE903AC9
:101330004FF04E530AEE103A4CF28303CBF6CA63D9
:1013400009EE903A43F27A63C3F6AB4309EE103AE2
:101350004DF20A73C3F623430BEE103A4AF63B23D1
:10136000C4F6B83345F256550AEE903A18EE903A64
:10137000C5F2555593B085FB0A2803F23173A8EBEB
:10138000EA7843F61C4B08EE903A4FEA690302955F
:10139000074607900891A8F1070809930C460546EF
:1013A000C0F2020B00262AE0B9F1000F00F312810F
:1013B0006FF0EE0101FB02F20732D21000EB0213D4
:1013C000B8F1000F23EAE373627B40F30181B8F1C7
:1013D0001F0FCCBFC2EB421208FB02F2D2100092E8
:1013E000384601360EAA0AA900F062FB062E04F167
:1013F000150405F1040507F1440700F0FB80627C49
:10140000A37CE17C207D002A71D003F0030C4FF017
:10141000640E40F678031EFB0C11C0F2440303FB7C
:1014200001F307284FEAE301C3BF073843F29143B2
:10143000434300230B44C5F83032A37BC5F86C222C
:1014400003F003035BF82330C5F854322078217988
:10145000627863790A90A0780E910B92A179E27874
:101460000F930C90E379207C0D921193109100F072
:1014700015FB237AC3EB0A03B3F1110200F1868056
:10148000029A217B94F80AE0103B82FB03C2A2EB94
:10149000E37301B303291ED01F2BDBBF43F6AC421D
:1014A000C0F20202FA23D35C03FB0EFE40F24913A2
:1014B00003FB0EF301294FEAE33316DD18447F28BE
:1014C000A8BF7F20B9F17F0F4FEA4010E27B7FF782
:1014D0006BAF0F216EE703FB0EF340F2491202FBE4
:1014E00003F301294FEA2333E8DC5B42E6E7B8EE79
:1014F000E88A069028EE0A0A059120EE290A04934C
:1015000003920DF0E5FB20EE090AF1EE0C7A80EE75
:10151000277A0698049B0599073843F62C4E03F06A
:101520001F03C0F2020E5EF8233007EE900A27EE8A
:10153000087AF8EEE77AA7EE278ABDEEC88A18EE99
:10154000102A1A441346039A00293FF474AF07EE99
:10155000901AF8EEE77AB7EE000AA7EE8B0A04932A
:101560000DF038FCF6EE007AE0EE2A7A17EE900ADB
:1015700010F074F841EC100B0CF086FE51EC100BDF
:1015800010F070FB049B039A034454E7029B94F809
:1015900009C0C2F10101E27A83FB013EAEEBE171C9
:1015A00002B3032A1ED01F29DBBF43F6AC4EC0F2A4
:1015B000020EFA211EF8011040F2491301FB0CF152
:1015C00003FB01F3DB13012A3FF778AF5B4275E7BA
:1015D000002204E743F6D433C0F202030999595CB0
:1015E000EF39E7E601FB0CF140F2491303FB01F38D
:1015F0001B13E8E7089A079992F88630C1F88832F9
:1016000092F887303BB3C3F1080308461446C0F88C
:10161000503294F88B3003EB830303EB43139B119D
:10162000C0F88C3294F88F3043F61442C0F20202B4
:1016300003F00703D35CC0F8903294F88C3003EBCE
:10164000830303EB43139B11C0F8843213B0BDEC4A
:10165000088BBDE8F08F102308461446D7E700BF7B
:101660002DE9F84F43F2680A804689460646A1F103
:10167000040B01F1180500F160070446C2F2010AEB
:10168000D4F8981101F172414A1340F2FE731340ED
:10169000581C5AF823205AF82000C1F30D0382FB8E
:1016A0000323920B42EA83420916C1F10601024468
:1016B0000A413046294610344BF8042F00F050FA06
:1016C000A74205F1010506F14406D9D109F11E0131
:1016D00008F5FC70BDE8F84F00F080BF2DE9F0413F
:1016E00004460F4600F5CC7806460D46394620469E
:1016F00000F03AFAD5F89C31C6F89C314434D5F85C
:10170000A431C6F8A431444507F1440705F110059A
:1017100006F11006EAD1BDE8F08100BFD1F8AC3186
:10172000D1F8A42110B4D1F89C41C0F89C41C0F874
:10173000A421C0F8AC31D1F8B431C0F8B431D1F83B
:10174000BC31C0F8BC31D1F8C431C0F8C431D1F8D3
:10175000CC31C0F8CC31D1F8D431C0F8D431D1F883
:10176000DC31C0F8DC31D1F8E431C0F8E431D1F833
:10177000EC31C0F8EC31D1F8F431C0F8F4315DF857
:10178000044B70470023C0F89C31C0F8A431C0F866
:10179000AC31C0F8B431C0F8BC31C0F8C431C0F8C5
:1017A000CC31C0F8D431C0F8DC31C0F8E431C0F835
:1017B000EC31C0F8F43170474FF48843C4F22C7315
:1017C00007EE103A87EE000A4FF0974307EE903A83
:1017D00020EE270A4DF68463BCEEC00AC2F2000375
:1017E00083ED000A704700BF30B40C6804601468D1
:1017F00004614D684560556845618D6885609568F0
:101800008561C968C160D268C261132C4FF00002C3
:1018100082624263DBBF43F6D042C0F202021C3454
:1018200052F824400362641003EB8413A3F585533C
:10183000026802994162102B02EB8204B8BF1023A8
:1018400002EBC4021B04002B01EBA212D4BF002444
:10185000012401253E2A80F84050C36280F83040C0
:1018600016DC02F0030392100433083203FA02F28A
:10187000D3174DF68461C2F200010968A1FB02454D
:1018800001FB0355230E43EA0523836330BC7047F5
:101890004FF060720023ECE7426B022AF0B403467B
:1018A00005DD032A66D190F84010002962D193F833
:1018B000301071B9986A996BDC6A401AA04298623C
:1018C00059DC511C03299C6259635BDD2046F0BC46
:1018D00070474FF6FF70996AC0F2B36081424CDDE9
:1018E000C1F1885000169D6BDC6A05FB0010A04218
:1018F000986240DB511C03299C625963E6DC03EBD0
:10190000820251691329DBBF43F6D040C0F20200C6
:1019100001F11C0550F82150196A586A6D1001EB4D
:101920008511A1F585511029B8BF102109048C42F9
:10193000ACBF00250125D96283F83050526802EB14
:10194000820102EBC10200EBA2123E2A4CDD4FF0F5
:10195000607600274DF68462C2F2000220461268CB
:10196000A2FB064502FB0755220E42EA05229A63B6
:10197000F0BC7047986AF0BC70470021C0F2B461B7
:101980000A20B0E703EB820251691329DBBF43F65B
:10199000D040C0F2020001F11C0550F82150196A34
:1019A000586A6D1001EB8511A1F585511029B8BF5A
:1019B000102109048C42ACBF00250125D96283F8AF
:1019C0003050526802EB820102EBC10200EBA21020
:1019D0003E28BCDC00F0030680100436083006FA0E
:1019E00000F00646C717B5E702F00306921004366A
:1019F000083206FA02F21646D717ABE790F84030E5
:101A00008B4241D000290CBF0323002330B49D003A
:101A1000421980F8401043631369816A132BDBBFBE
:101A200043F6D042C0F2020203F11C0452F82340F4
:101A3000036A426A641003EB8413A3F58553102BE9
:101A4000B8BF10231B048B42D4BF0021012180F8B2
:101A50003010C362435903EB830103EBC10302EB74
:101A6000A3123E2A11DD4FF0607200234DF684610F
:101A7000C2F200010968A1FB024501FB0355230ED8
:101A800043EA052330BC8363704702F003039210DE
:101A90000433083203FA02F2D317E7E71328DBBF57
:101AA00043F6D043C0F202031C3053F820007047C5
:101AB00030B40C680460146804614C684460546875
:101AC00044618C68846094688461C968C16090F8DE
:101AD0004010D568029AC56103624262002934D081
:101AE000132CDBBF43F6D041C0F202011C3451F885
:101AF00024408568816A641003EB8413A3F5855341
:101B0000102BB8BF102305EB85041B0405EBC4059F
:101B10008B4202EBA512D4BF0021012102243E2AF0
:101B2000C36280F83010446311DD4FF0607200230F
:101B30004DF68461C2F200010968A1FB024501FB78
:101B40000355230E43EA0523836330BC704702F03C
:101B5000030322410433083203FA02F2D317E7E702
:101B6000436B0B70704700BF0A680B69036102602A
:101B70004B6843604B6943618B6883608B69836109
:101B8000CB68C360F0B5CB69C3610B6A4F6A8E6ADC
:101B9000CD6A91F830E04C6B8A6B036291F840306B
:101BA00047628662C56280F830E04463826380F8F1
:101BB0004030F0BD70B54FF09D432DED048B08EE25
:101BC000103A41F23063002143F26804C3F6807397
:101BD0000020C4F2D01108EE903AC2F201040025B0
:101BE000B6EE009A0BE078EE097A17EE900A0FF045
:101BF00035FD41EC100B0CF047FB51EC100B6E0067
:101C000010F030F801360135B5F5806F28EE288ADE
:101C100044F82600E7D1002340F2FF355A00D11CDA
:101C2000501C54F8211054F820000133091AAB421B
:101C300043F2680044F82210C2F20100EED141F6EE
:101C4000FC73BDEC048BC35841F6F872C3F100433A
:101C5000835070BD002207EE902A4FF0974202EEAB
:101C6000102A4FF06C5204EE902A4FF06E5202EEA2
:101C7000902A4AF6AB22C3F62A2241F2680303EE09
:101C8000102AC2F201030022F6EE003AB7EE006A13
:101C9000B0EE004AF0EE465AE7EEE75A03EBC20117
:101CA0000132B0EE677AA5EEA47AB2F5806FB0EE9D
:101CB000465AA7EE475AF0EE636AE7EE826AB0EE44
:101CC000677AA5EE247AFDEEE66AC1ED016AF0EED0
:101CD000466AE7EE476AB0EE677AA6EEA27A76EE3B
:101CE000856AB0EE465AA7EE475A35EE257AA6EE3B
:101CF000847AE7EE037ACDD130B4002240F2FF358A
:101D00005100C81C4C1C53F8200053F824400132E9
:101D1000001BAA4241F2680443F82100C2F2010408
:101D2000EED14FF0974306EE903AB6EE007AA7EE6A
:101D3000A67A41F6FC7341F6F872E358FDEEC77AD5
:101D400017EE901ACB1AA35030BC7047704700BFF3
:101D50002DE9F04F43F6345491B003EB4303C0F246
:101D6000020404EBC3041546069007910FCC0AAE9B
:101D70000FC694E80300002386E803004FF0010833
:101D800043F268060AAF05F160098DF824808DF8EA
:101D900025308DF82630C2F2010605973BE00AF1A6
:101DA000FF30069B00EB001003EB0010133020F017
:101DB0000F0095E8084003F1724B4FEA6B3340F295
:101DC000FE721A40531C56F8222056F82340CBF3DB
:101DD0000D0382FB0323920B4FEA2B6B42EA8342F3
:101DE000CBF1060B144444FA0BF4BEF58C6F6C6017
:101DF0001CDAB4F58C6F19DABCF1000F03D110AB0B
:101E00009A440AF81CCCEB68AA6803EB8213EB60D7
:101E10001035A9452FD0059B53F8041B059311F0ED
:101E2000030A01F0040CBAD10798C2E710AB9A4438
